:10000000544649530001000068160300B60F3C3700
:100010001773022520102713445631591773010115
:10002000201027134456315917730201201027134B
:100030004456315903000000000000000000000099
:1000400054464353002000001CD202000000000070
:10005000008001100121000025210000D53602009A
:10006000292100002B2100002D2100003D2100004E
:100070003D2100003D2100003D2100002F21000016
:10008000312100003D21000033210000996F000064
:1000900063730000372100003D21000071700010E3
:1000A00037210000995000009D500000937200001D
:1000B00037210000D76B0000C9620000A15000008A
:1000C000916900003721000037210000E55D000044
:1000D0000000000000000000000000000000000020
:1000E0000000000000000000000000000000000010
:1000F0000000000000000000000000000000000000
:1001000000000000000000000000000000000000EF
:1001100000000000000000000000000000000000DF
:1001200000000000000000000000000000000000CF
:1001300000000000000000000000000000000000BF
:1001400000000000000000000000000000000000AF
:1001500000F003F800F020F8FEE70D480168890878
:100160008900002001C101C101C101C17047000027
:1001700094790010FEE7FEE7FEE7FEE7FEE7FEE704
:10018000FEE7FEE7FEE703480047FEE7FEE7000064
:10019000202100003D21000000F002F800F068F886
:1001A0000AA090E8000C82448344AAF10107DA45D2
:1001B00001D100F05DF8AFF2090EBAE80F0013F0BC
:1001C000010F18BFFB1A43F00103184764540200E3
:1001D000C45402000A444FF0000C10F8013B13F025
:1001E000070408BF10F8014B1D1108BF10F8015B90
:1001F000641E05D010F8016B641E01F8016BF9D183
:1002000013F0080F1EBF10F8014BAD1C0C1B09D1D9
:100210006D1E58BF01F801CBFAD505E014F8016B4B
:1002200001F8016B6D1EF9D59142D6D370470000DD
:10023000103A24BF78C878C1FAD8520724BF30C812
:1002400030C144BF04680C607047000000230024E4
:1002500000250026103A28BF78C1FBD8520728BFD6
:1002600030C148BF0B6070471FB51FBD10B510BD32
:10027000DFF80CD0FFF7F8FF07F0F0FA21F044FAAE
:100280000080011003B4FFF7F1FF03BC21F044FA32
:1002900008B500200346024600900121022000F02C
:1002A0006EFB08BD38B5FF4D0024FF48AC81EC81E2
:1002B0002C8240698047E861FF202872FB480023B8
:1002C0001A46046044608460C4600461012068725E
:1002D0002C70AC7001460220009400F050FB01200D
:1002E00038BD38B5EF4D02282C7A22460DD00528AE
:1002F00010D0A24208BF38BD002003460246214666
:10030000009000F03CFB2C7238BD022914BF012480
:100310000224EEE7022914BF04240824E9E708B503
:10032000009313460A460146012000F028FB08BD51
:1003300008B50346009103220221012000F01FFBB3
:1003400008BD38B500240EF06FFB002818BF01244B
:1003500013F05FF8002818BF0224D2480178A142A8
:1003600008BF38BD047000200346022100902246D9
:10037000084600F004FB38BD38B5CA4D044668781D
:10038000A04208BF38BD07F083FA6C70002C0CBF88
:10039000052106210020034602460090022000F0BD
:1003A000EEFA38BD08B500210B4602460091072140
:1003B000022000F0E4FA08BD08B500210B46024611
:1003C00000910821022000F0DAFA08BD08B50021EA
:1003D0000091002814BF01220022002303210220E3
:1003E00000F0CDFA08BD08B5002003460246009093
:1003F0000421022000F0C3FA08BDAA4B0028DA78D5
:1004000014BF01210021D9708A4208BF7047021C25
:1004100018BF012208B50020034600900A210220DF
:1004200000F0ADFA08BD9F4B00289A7814BF012157
:10043000002199708A4208BF7047021C18BF012230
:1004400008B50020034600900921022000F097FA29
:1004500008BD94488078002818BF0120704701200B
:100460009049087170478F48007970478D49002086
:10047000087170472DE9F04104460127002503F07B
:100480000700884E8846012804BF0020308248D0EB
:10049000022846D1308A844904280BD2002818BF8C
:1004A000B06902D148688047B06110F8011B217023
:1004B000B0612FE0062809D288688047318A80B26F
:1004C000C1F10501C900C840207023E0082808D206
:1004D00008698047318AC1F10701C900C84020700E
:1004E00018E00C2808D248698047318AC1F10B0115
:1004F000C900C84020700DE00E2808D288698047E6
:10050000318AC1F10D01C900C840207002E0FF200E
:1005100020700027308A401C80B230820E2828BF0D
:10052000012588F800503846BDE8F08130B403F06A
:1005300007000024DFF86CC1012804BFACF80C40B0
:10054000ACF810401BD013F0070F18D1554BBCF876
:1005500010009B89022805D2120242EA1322ACF84D
:100560000C2009E003449D1EB5F5806F04DADCF829
:100570001C502B4403F8022C401CACF810000C70EB
:1005800030BC00207047F0B40746002003F0070499
:10059000444D0646012C04BF2E826E6125D0DFF843
:1005A00004C1022CBCF80EC003D013F0070F0DD00D
:1005B0001BE02A8A0CEB0203B3F5806F15D2E869C1
:1005C000C05C3870501C288201200EE0120242EA02
:1005D0001C22EA816B69012B05D1B2F5806F24BF23
:1005E00040F2FF32EA815A1C6A610E70F0BC70471B
:1005F00038B503F0070000240D46012809D1294829
:1006000000231A460482848119460220009400F0D7
:10061000B6F92C70002038BD2DE9F04182B01746A4
:100620000C0005464FF0000800F0028126782049B2
:10063000012E18BF022E05D0032E5AD0002E00F036
:10064000F780BDE06078421E05EB001000F8102C2A
:10065000607805EB001000F80F6C08686288438D25
:10066000C08C5A4392FBF0F0627805EB021222F83C
:100670000E0C0868A288018D808C514391FBF0F02C
:10068000617805EB011121F80C0C6178A07905EB7C
:10069000011121F80A0C6178207A05EB011121F88B
:1006A000080C07E00084001090740200848A001097
:1006B000B08900106178607A05EB011121F8060C11
:1006C0006178A07B05EB011121F8040CE079052885
:1006D000607805EB001010F8021C0CBF41F001011E
:1006E00021F0010100F8021C002E69D102B0BDE822
:1006F000F0816078421E05EB001000F8102C627843
:10070000032005EB021202F80F0C08686288438D83
:10071000C08C5A4392FBF0F0627805EB021222F88B
:100720000E0C0868A288018D808C514391FBF0F07B
:10073000617805EB011121F80C0C07F0A9F80528E8
:1007400021D107B36178B87905EB011121F80A0CC2
:100750006178387A05EB011121F8080C6178787A14
:1007600005EB011121F8060CF8790528607805EBF6
:10077000001010F8021C0CBF41F0010121F0010132
:1007800000F8021C17E0607805EB001020F80A8CD6
:10079000607805EB001020F8088C607805EB0010FD
:1007A00020F8068C607805EB001010F8021C21F090
:1007B000010100F8021C607805EB001020F8048CA1
:1007C000012E18BF032E06D00DF042FE002804BFF4
:1007D00002B0BDE8F08107F05BF805281CBF02B04D
:1007E000BDE8F081012E04BFC0208DF8000005D0C7
:1007F000022E0CBFC220C1208DF8000060788DF859
:10080000010060880123000A8DF80200A0788DF8AD
:100810000300A0880622000A8DF8040020798DF8D4
:1008200005006946072011F024FD02B0BDE8F08103
:1008300085F8008085F80180A5F80280A5F804807D
:10084000A5F80680A5F80880A5F80A80A5F80C8010
:10085000A87B20F00100A87302B0BDE8F0814D49EB
:100860000020487170474B4840797047002818BFF6
:1008700001204849887170474648807970470028B0
:1008800018BF01204349C87170474248C07970477A
:100890004049488170473F48408970473D490120A1
:1008A000487170473C4B03EB80004254704730B5B1
:1008B00085B001788DF8001042788DF8012082789B
:1008C0008DF80220C2788DF8032002798DF804207B
:1008D00042798DF8052080798DF8060000200125E9
:1008E0002C4C8DF8070002900390522905D1A07975
:1008F00088B9A57106F089FB60819DF80000462843
:1009000001BF9DF801000128E079002803D1E571BD
:1009100006F07BFB608107F0EDF801280CD120F098
:1009200011FF012801BF9DF8000046289DF8010035
:10093000012804BF05B030BD684620F008FF05B0AF
:1009400030BD70471349002818BF01204872704716
:100950001048407A7047012818BF70470F48012996
:1009600004BF416841F4007105D0002906BF416809
:1009700021F400717047416070470948704708B51D
:10098000DDF808C0CDF800C0DFF818C0DCF800C002
:10099000E04708BD00840010848A00100010004069
:1009A000606F0200907402007047F648D0F8500360
:1009B00000F00100704770B5F24D04000AD002F05B
:1009C000B9FA38B9D5F8500310F0010F1CBF002058
:1009D000A86005D10120A860002C08BF00202DD000
:1009E000D5F8600310F0010F0BD1D5F8600340F08B
:1009F0000100C5F86003D5F8600320F00100C5F8D8
:100A00006003E148016811F0010F07D1016841F06E
:100A100001010160016821F00101016004F078FB2F
:100A200000281CBFD5F8500310F0010F05D004F0CA
:100A300069FB002818BF04F077FB0120286270BD15
:100A4000D048006A002818BF01207047C00000F19C
:100A5000804000F5A04041637047C00000F1804035
:100A600000F5A040006B00F4807070471021C000BA
:100A700000F1804000F5A0404163704730B4820926
:100A8000C24B00F00F0000EB400053F822404FF43F
:100A9000847505EB8015D1F800C044F805C053F803
:100AA00022204FF4867303EB80104968115030BC4C
:100AB00070478209B54850F82200D0F8402161F310
:100AC0000D22C0F840217047B049800951F820003C
:100AD000D0F84001C0F305207047AA49D1F8402161
:100AE00060F31742C1F840217047A648D0F8400192
:100AF000C0F3074070474FF4A072C0F3011302EB3C
:100B00008312DFF888C200F00F03800903EB430370
:100B10005CF82000002900EB8310815814BF41F0DD
:100B2000010121F0010181507047984A810952F872
:100B3000212000F00F0101EB410102EB8111C0F314
:100B400001104FF4A07202EB8010085800F0010071
:100B500070478E4A810952F82110D1F8E01100F057
:100B60000F00012201F0070102FA00F0084018BF4F
:100B7000012070474FF4A072C0F3011302EB8312FF
:100B8000DFF808C200F00F03800903EB43035CF8B1
:100B90002000002900EB8310815814BF41F00201AE
:100BA00021F0020181507047784A810952F82120D2
:100BB00000F00F0101EB410102EB8111C0F30110C4
:100BC0004FF4A07202EB80100858C0F34000704749
:100BD00081096F4A01EB410102EBC10100F00F02F4
:100BE00001EBC201C0F3011051F8200070476849C1
:100BF00082091CD00122B2EB901F18BF70476548D4
:100C00000068C0F30800886163480268C2F30842C4
:100C10000A620068C0F30800486260480268C2F3D4
:100C200008428A620068C0F30800C86270475548ED
:100C3000D0F82421C2F308020A60D0F8E421C2F3FC
:100C400008428A60D0F8E421C2F30802CA60D0F8F2
:100C5000A422C2F308420A61D0F8A402C0F308003B
:100C6000486170472DE9F0030122830900F00F016C
:100C7000C0F3011CC0F3011622EA0C0C00290BBFC3
:100C800002254D1E00224FEA0C124FF0080404EB1F
:100C9000CC043F4F03EB430C07EBCC0C0CEBC10136
:100CA000DFF8E88051F826604FF4587C58F823109C
:100CB0000CEBC50551F805C000F00F001CF0010F4A
:100CC00000EB40004FF4927C0CEB801C40F2FF17CD
:100CD00029D02C48D0F844034FF032090005000D0C
:100CE00006FB09F60EBF0120B6FBF0F0401CFF2802
:100CF00088BFFF204E594FF0FF0909FA04F9C0B22E
:100D000026EA0906A0403043485158F8230050F81D
:100D10000C3007FA02F123EA0102114340F80C10EB
:100D2000BDE8F003704751F80C0007FA02F398434E
:100D3000C6F3080303FA02F2104341F80C00BDE8C1
:100D4000F003704710B50020FFF78CFF0120FFF77C
:100D500089FF1120FFF786FF0220FFF783FF122093
:100D6000FFF780FF4020FFF77DFF4120FFF77AFF6C
:100D70005120FFF777FF4220FFF774FFBDE81040D6
:100D800052206FE700500040605B00407C6F020023
:100D9000388B001024590040E4590040A45A004008
:100DA0002DE9F04707464FEA9016FF480D0050F82E
:100DB00026404FF000002062C4F84001C4F8000251
:100DC000C4F84002C4F8C002C4F8000308BFBDE87C
:100DD000F0872868206068686060616801200029E9
:100DE00008BF6060F1490860A868A060E868E0603A
:100DF0002869A0616869E061E8696062286AE06268
:100E000021206063E063686A2064A86A6064E86A1D
:100E1000A064286BE064686B2066A86BA066E86B32
:100E20006067286CA067686CE067A86CC4F88000F5
:100E3000E86CC4F88400286DC4F88800686DC4F8B4
:100E40008C00A86DC4F89000E86DC4F8A400286E6A
:100E5000C4F8A800686EC4F8AC00A86EC4F8B0006E
:100E6000E86EC4F8B400286FC4F8B800686FC4F81E
:100E7000BC004FF0FF30C4F8E400A86FC4F8F000E5
:100E8000E86FC4F8F400D5F88000C4F8FC004FF413
:100E9000107205F1840104F5807020F05DFCD5F836
:100EA000C40220F48030C4F84003D5F8C802C4F866
:100EB0004C03D5F8CC02C4F85003D5F8D002C4F8DE
:100EC0005403D5F8D402C4F85803D5F8D802C4F8AE
:100ED0005C03002005EBC002D2F8DC3204EBC00159
:100EE000C1F86033D2F8E022C1F86423401C032823
:100EF000F0DBD5F8F402C4F87803D5F8F802C4F8AA
:100F00007C03D5F8FC02C4F80004D5F80003C4F84B
:100F10000404D5F80403C4F80804D5F80803C4F899
:100F20000C04D5F80C03C4F810040022002104EBD3
:100F3000C20805EBC20000EB8103D3F8109308EB65
:100F4000810CCCF83094D3F83893CCF85894D3F87B
:100F50006033CCF88034491C0229ECDB05EB8200BD
:100F6000D0F8883304EB8201C1F8A834D0F89C3360
:100F7000C1F8BC34D0F8B003C1F8D004521C052A23
:100F8000D4DB002E14BF8A488A48006830F0FF0185
:100F900005D1D4F8901060F30301C4F89010D4F890
:100FA000500320F00100C4F85003D4F8600320F08F
:100FB0000100C4F86003D4F8680320F00100C4F80D
:100FC0006803D4F8700320F00100C4F870033846B9
:100FD000BDE8F0470BE678480078704776484078DF
:100FE00070477549887070477348807870477349B7
:100FF000D1F8542360F30902C1F8542370476F48B5
:10100000D0F85403C0F3090070476B49486070473B
:1010100069484068704768498860704766488068DA
:1010200070476648D0F8440340F20F12C0F30B013A
:1010300053003C20A1F20F1CBCF1000F4CBF521A10
:101040006246A1F21E2CBCF1000F4CBF591AA1F24E
:101050001E219142B8BF1E2070475749C860704793
:101060002DE9F05F04460027384614F4803F18BF8E
:10107000012014F4003F18BF40F0040014F4802F46
:1010800018BF40F0020014F4002F18BF40F0100009
:1010900014F4001F18BF40F0400014F4800F18BF74
:1010A00040F0080014F4000F18BF40F02000DFF8F3
:1010B0000881DFF8089198F8021010EA0105D9F8C4
:1010C000400320F48030C9F8400336D0D8F80C60D3
:1010D000D9F84803002740F00100C9F84803D9F8BF
:1010E000480320F00100C9F84803D9F8400340F450
:1010F0008030C9F840034FF0630ADFF8C4B016E04F
:1011000004F04DF95046D9F8481311F0010F0AD0F8
:10111000D9F844030005000D1CBFBBFBF0F0C8F874
:101120000800012703E0011EA0F10100EBDC301EE6
:10113000A6F1010601DD002FE2D0D9F8500320F01E
:101140000100C9F85003D9F8600320F00100C9F884
:101150006003D9F8680320F00100C9F86803D9F8E2
:10116000700320F00100C9F87003164A106820F0DF
:10117000010010601448016821F001010160134969
:101180000B6823F001030B60EFB315F0010F05D0DE
:10119000D9F8503343F00103C9F8503315F0040F68
:1011A0001AD0D9F8703313E07C6F02000458004065
:1011B000F0FE0400E0FE0400208400100050004017
:1011C00080F0FA02605B0040685B0040705B0040AA
:1011D00043F00103C9F8703315F0020F05D0D9F8B8
:1011E000603343F00103C9F8603315F0100F05D0E8
:1011F000D9F8683343F00103C9F8683315F0400F9C
:1012000005D00B6800E01CE043F001030B6015F013
:10121000080F03D0116841F00101116015F0200F93
:1012200003D0016841F00101016088F801500120FC
:1012300088F80000D9F8400340F48030C9F8400332
:1012400021E0002088F80100ADB1022088F80000FC
:10125000D9F8400340F48030C9F84003D9F8480376
:1012600040F00100C9F84803D9F8480320F0010014
:10127000C9F8480307E0D9F8401321F48031C9F8D0
:10128000401388F80000D9F8400114F0010F20F055
:101290000D0018BF40F0010014F0040F18BF40F01B
:1012A000040014F0020F18BF40F00800C9F8400114
:1012B000D9F8000214F0100F14BF40F0010020F024
:1012C0000100C9F80002D9F8400214F0200F14BF41
:1012D00040F0010020F00100C9F84002D9F8C00236
:1012E00014F0400F14BF40F0010020F00100C9F8D5
:1012F000C002D9F8000314F0800F14BF40F00100C1
:1013000020F00100C9F80003FF4814F4805F016871
:1013100014BF41F0010121F001010160FB4814F408
:10132000005F016814BF41F0010121F0010101607B
:10133000F74814F4804F016814BF41F0010121F017
:1013400001010160F34814F4004F016814BF41F03B
:10135000010121F001010160EF49086814F4807F68
:1013600020F00D0018BF40F0010014F4806F18BF8A
:1013700040F0040014F4007F18BF40F0080008603B
:101380000020FFF76FFC0120FFF76CFC1120FFF736
:1013900069FC0220FFF766FC1220FFF763FC402087
:1013A000FFF760FC4120FFF75DFC5120FFF75AFC7E
:1013B0004220FFF757FCBDE8F05F522052E42DE9D0
:1013C000F04F840900F00F0343EA8411D34D4FEA34
:1013D000911CC1F3011855F82C6003EB430C06EB8C
:1013E0008C174FF4A07606EB8818024657F8087061
:1013F000002017F0010F10D141F010018F09C1F347
:10140000011155F8277006EB811107EB8C177958FD
:1014100011F0010F08BFBDE8F08F55F82410CF6917
:1014200007F0080801EB8C17D7F80011DFF8F0A2DD
:1014300004EB440C0AEBCC0C1FFA81F902F00F0507
:10144000002103EB43060CEBC505C2F3011A43EA86
:10145000011242EA8412DFF8C4C2C2F3811B5CF8B5
:101460002BC0C2F3011B4FF4A0720CEB861C02EBE5
:101470008B125CF8022012F0010F1AD007EB811CCE
:1014800055F82A20DCF844B1B8F1000FCBF3080B73
:101490000EBF4FF0000CDCF844C1CCF3023C02EB71
:1014A000C20E0EEB021200EB42000BFA0CF202FB32
:1014B0000900491C0229CAD3BDE8F08F2DE9F0418B
:1014C0008509AA0195489309002450F82300D0F813
:1014D000401111F0010F34D0914E03EB430306EBA2
:1014E000C30302F00F0603EBC603C2F3011211F0AF
:1014F000040F53F82220D0F8003101F0080C9EB2FE
:10150000D0F84431C3F3080318BFC1F30744C769D7
:10151000C1F3052117F0080F1ABFD0F84401C0F33A
:1015200002300020BCF1000F18BF491C03FA00F084
:1015300001FB004002EBC201704301EB021100EB22
:101540004104012040EA8510FFF739FF06460220DA
:1015500040EA8510FFF733FFA1190844BDE8F08188
:1015600010B50020FFF7AAFF4FF47A7148434CF200
:101570005031B0FBF1F010BD6A484068C0F30C0078
:10158000704770B504460020FFF798FF05464020DD
:10159000FFF794FF35B3634BB0B141F28831084493
:1015A000A84211D9421B186800F01F0104FB01F08A
:1015B00000EBC00C0CEB0010B2EB400F04D9322052
:1015C0004843B2FBF0F0441CB4F5005F28BF41F67D
:1015D000FF7402D2002C08BF0124586864F30C0089
:1015E000586070BDB4F5005F28BF41F6FF7402D2A9
:1015F000002C08BF01244C48016864F30C01016011
:1016000070BD2DE9F041474F0646386810F01F05C0
:1016100008BF01250020FFF751FFDFF810810446C5
:10162000002E18BF002C3FD0414900204A68002AF4
:1016300008BF01223309B3FBF2F1D7F850C31CF005
:10164000010F1BD0B3EB420F1DD33A49B1FBF2F3AC
:10165000B6FBF2F10A09B3FBF4F1102928BF0F2100
:101660008A4298BF114639B1012984BF01FB143069
:10167000B0FBF1F007D908E0012109E0B8FBF6F270
:10168000A24288BF101B0029F6D0102988BF0F2165
:10169000D7F85C2361F30302C7F85C233221694366
:1016A000B0FBF1F0FFF76DFF7868C0F30C00684302
:1016B00000EBC00101EB001004EB4000B8FBF0F0C0
:1016C000BDE8F08170B5174D0024D5F8500310F037
:1016D000010F08D01648D5F85C13406801F00F01DF
:1016E000484304012EE00020FFF7E8FE0246286888
:1016F000696800F01F00C1F30C01414301EBC10018
:1017000000EB011018E00000005A0040405A004071
:10171000C05A0040005B0040405900407C6F02000E
:10172000388B001000500040045800400008AF2FD4
:101730002084001080F0FA0212EB40001CBFFD492B
:10174000B1FBF0F4204670BD002818BF0120FA4913
:10175000D1F85C2360F30302C1F85C237047F648BC
:10176000D0F85C0300F00F0070478109F34A00F0E5
:101770000F0000EB400052F821104FF4807202EB92
:1017800080100858EE4980B2B1FBF0F0401C4008D0
:1017900070472DE9F041E94B8209DFF8A4C353F803
:1017A000223000F00F0731B1BCFBF1F1491C4A08AF
:1017B000B2F5004F01D347F6FF72BCFBF2F1491CB2
:1017C0004D08D3F880104FEA520C01F00704D3F80B
:1017D0008010DA4B4FEA9018C1F3031600F00F01A6
:1017E00053F8283001EB410103EB81112FB3D1F8FD
:1017F0000431F61C74439BB2A2EB4404D1F800619F
:1018000024F0010462F30F06C1F80061D1F8002151
:101810006CF31F42C1F80021D1F8042163F30F02D9
:10182000C1F80421D1F8182164F30F02C1F818217E
:1018300001F0C9F82846BDE8F081F61CACF10E03B2
:101840007443A3EB4404D9E710B48309BB4C10F0F4
:101850000F0F00F00F0054F8233000EB40004FF45E
:10186000807404EB801018584FEA10401CBF10BC65
:101870007047D3F880C00CF00704D3F880C0401A3A
:10188000D3F80411CCF3031C60F30F01C3F8041167
:10189000012A1CBF10BC70470CF103016143A0EB8F
:1018A0004100D3F8181120F0010060F30F01C3F8D4
:1018B000181110BC70478109A04A00F00F0000EB1E
:1018C000400052F821104FF4807202EB801008584B
:1018D000000C7047830910F00F02984850F823005D
:1018E00002EB420300EB8313D3F800C161F31F4CFA
:1018F000C3F800C118BF7047D0F8802002F007037A
:10190000D0F88020C2F30312D21C5A430E39A1EB47
:101910004202D0F8043122F0010261F30F03C0F853
:101920000431D0F8181162F30F01C0F81811704794
:10193000824A810952F8212000F00F0101EB410198
:1019400002EB8111C0F301104FF4A27202EB801080
:101950000858C0F308007047F0B4784B840900F0D1
:101960000F0C53F824300CEB4C0503EB8516C0F339
:101970000112D6F81C5106EB82164D1BD6F84471A5
:1019800061F30807C6F844714CEA021141EA841178
:1019900001F00F02C1F3011101EB4201694A03F5A5
:1019A000C07352F821104A08C90753F822C0C90E63
:1019B00040F2FF148C402CEA040CAD1EC5F3080461
:1019C00004FA01F14CEA010143F82210F0BC00F0E6
:1019D000FABF830900F00F01C0F30112574850F815
:1019E0002300C36901EB410100EB811013F0100FDC
:1019F000D0F8281100EB8210C9B2D0F84401C0F32E
:101A0000080008BF0021401A0004000C08BF012094
:101A1000704703091B0203EB810101F1405101F5FD
:101A200000310007C00E0B6802FA00F0184308608E
:101A300070470209120202EB810101F1405101F5E8
:101A4000003100070968C00E21FA00F000F0030021
:101A5000704770B4DFF8E4C0820900F00F035CF84F
:101A6000225003EB4303C0F301104FF4A87605EBBB
:101A7000831506EB80160C68AC515CF8222049688F
:101A800002EB83124FF4AA7303EB8010115070BC69
:101A9000704730B4DFF8A4C0820900F00F035CF88F
:101AA000224003EB4303C0F301104FF4A87504EB8D
:101AB000831405EB801564590C605CF8222002EB5E
:101AC00083124FF4AA7303EB80101058486030BCA7
:101AD00070471A4910B4820983B051F8222000F0EF
:101AE0000F0101EB410102EB8111C0F301104FF432
:101AF000A87202EB80128A5800924FF4AA7202EB8D
:101B0000801008580190002001466A4601234FEAE0
:101B1000511C01F01F0452F82CC003FA04F41CEA13
:101B2000040F18BF401C491C2629F0D303B010BC79
:101B3000704700000008AF2F005000407C6F02008B
:101B4000A0860100846F020030B4002210F00F0F55
:101B500006D000F00F02C0F3011303EB4202521E45
:101B6000FE4B80094FF4866553F8204005EBC20513
:101B7000D1F800C044F805C053F8200040F23443C7
:101B800003EBC2024968815030BC704710B4002298
:101B900010F00F0F06D000F00F02C0F3011303EB9B
:101BA0004202521EED4B80094FF4866453F820C068
:101BB00004EBC2045CF804C0C1F800C053F8200074
:101BC00040F2344303EBC2028058486010BC7047B7
:101BD000E348C06870470022E049830951F82310A8
:101BE000CB6913F0080F0ED000F00F0202EB420297
:101BF00001EB8211C0F301104FF4A27202EB8010CE
:101C00000858C0F3023210467047DFF850C310B4D2
:101C100082095CF82230DC6944F00804DC615CF87D
:101C2000223000F00F0202EB420203EB8212C0F3FB
:101C300001134FF4A27000EB8310135861F30E33BD
:101C4000135010BC70470022C449830951F8231077
:101C5000CB6913F0080F0ED000F00F0202EB420226
:101C600001EB8211C0F301104FF4A47202EB80105B
:101C70000858C0F3024210467047B84A830952F828
:101C8000233000F00F0202EB420203EB8212C0F39A
:101C900001134FF4A47000EB8310135861F3124347
:101CA00013507047042988BF70472DE9F0030027BF
:101CB000DFF8A882840958F82430DA69C0F3011CDF
:101CC00012F0080F4FF4A27202EB8C1C00F00F020E
:101CD00002EB420205D003EB821555F80C50C5F318
:101CE0000237DD69002615F0080F4FF4A475C0F324
:101CF000011005EB801504D003EB82104059C0F3AE
:101D00000246C91B7018042803DD081A011D0420AF
:101D100003E00028BCBF014400207E18D96941F0CF
:101D20000801D96158F8241001EB821151F80C30E8
:101D300066F30E3341F80C3058F8241001EB821191
:101D40004A5960F312424A51BDE8F0037047834A92
:101D50008009002952F82000816914BF41F0080170
:101D600021F00801816170477C49800951F8200009
:101D70008069C0F3C0007047784A8009002952F892
:101D80002000816914BF41F0020121F0020181614C
:101D900070477249800951F820008069C0F3400003
:101DA00070476E4B820953F8223000F00F0202EBAD
:101DB000420203EB8212C0F301104FF4A67303EB4F
:101DC000801011507047654A810952F8212000F0B7
:101DD0000F0101EB410102EB8111C0F301104FF43F
:101DE000A67202EB8010085870475D4A10B4D2F812
:101DF000400110F0010F0BD0D2F84C01D2F8441181
:101E00000028C1F302311EBF0029C043C2F84C01B3
:101E10000123002003EB43018C0104EB801101F14D
:101E2000804101F5A041D1F8402112F0010F0CD002
:101E3000D1F84C21D1F844C1002ACCF3023C1EBF9A
:101E4000BCF1000FD243C1F84C21401C0228E4D35E
:101E50005B1C032BDDD310BC704700223F49830974
:101E600051F82310CB6913F0080F0ED000F00F02C9
:101E700002EB420201EB8211C0F301104FF4A47295
:101E800002EB80100858C0F3005210467047012042
:101E900070472DE9F04F82B0022ADDE90B49DDF8E9
:101EA000348026BF921E4FEA520C4FF0000C022BDA
:101EB00026BF9A1E530800232A4AA2FB0442170990
:101EC000B8F1000F14BF012200220192B9F1020FF4
:101ED00016BF5FEA09024FF0010B4FF0000B8209B9
:101EE0001E4C00F00F0606EB460554F822404FF456
:101EF000B27E04EB851AC0F301140EEB841ECDF8FC
:101F000000A05AF80EA061F35C6A6BF3186A05D161
:101F100067F3174A63F3CA1A6CF3C60A019969F3A7
:101F2000420A61F3000A0099DFF8309041F80EA0F0
:101F300059F822204FF4B471C0F3011A01EB8A1151
:101F400002EB8512B8F1000F555814BF45F080051B
:101F500025F080055550012506E000007C6F020049
:101F600000500040CDCCCCCCB5EB901F1CBF02B0D4
:101F7000BDE8F08F04EB4600FC4951F820201831F1
:101F800011F8208006EB4600800100EB841000F180
:101F9000804000F5A040D0F85049F549FF26A1FB4C
:101FA00002914908A1EB81094A44D2009640FFB250
:101FB00097404FEA8802002003F00F0393400CF093
:101FC0000F0C4FF00F090CFA02FC09FA02F24FEA6B
:101FD000810805FA00F1214222D008EBC00101F18D
:101FE000804101F5A041D1F8809C29EA060949EA1F
:101FF0000709C1F8809C810001F1804101F5A041F1
:10200000D1F8A89C29EA020949EA0309C1F8A89C69
:10201000D1F8BC9C29EA020949EA0C09C1F8BC9C28
:10202000401C0528D5D302B0BDE8F08F2DE9F04F54
:1020300084B0DDE90EA8DDF834C0B8F1000F14BF9C
:10204000012400240294BAF1020F16BF5FEA0A04C9
:102050004FF0010B4FF0000B8409C64D00F00F0745
:1020600007EB470655F824504FF4B27E05EB86196E
:10207000C0F301150EEB851ECDE9009E59F80E90B8
:1020800061F35C696BF318697ED002996AF34209C7
:1020900061F30009DDE9001BDFF8D8A241F80B90DD
:1020A0004FF4B4715AF82440C0F3011901EB8911BF
:1020B00004EB8614B8F1000F665814BF46F0800692
:1020C00026F0800666500126B6EB901F1CBF04B0B8
:1020D000BDE8F08F05EB4700A449A74C51F820104C
:1020E00054F8204007EB4700800100EB851000F119
:1020F000804000F5A040D0F850099D4DFF26A5FB7B
:1021000001756D08A5EB850739444FEAC1090090B8
:1021100006FA09FE00200F21A400A1404FEA850B1A
:10212000012505FA00F6009D2E4241D01568022DCA
:1021300026BFAD1E6D080025121D1E68022E26BF8B
:10214000B61E760800265CF8048B8C4FA7FB088728
:102150004FEA07580BEBC00707F1804707F5A04788
:10216000D7F880AC4FEA18682AEA0E0A08FA09F88C
:102170004AEA0808C7F8808C870007F1804707F50E
:10218000A047D7F8A88C00E018E006F00F0628EA70
:102190000108A64048EA0606C7F8A86CD7F8BC6C48
:1021A00005F00F058E43A5403543C7F8BC5C1B1DE9
:1021B000401C0528B4D304B0BDE8F08F1168022993
:1021C00026BF891E49080021D3F800B0BBF1020FD9
:1021D00026BFABF1020B4FEA5B0B4FF0000BCDF8C3
:1021E0000CB0DFF898B1DCF800E0ABFB0EEB4FEA87
:1021F0001B1B6BF31749DDF80CB06BF3CA1961F3C5
:10220000C60942E72DE9F00F5A4D84094FF4B2791F
:1022100055F8244000F00F0505EB450604EB861445
:10222000C0F3011609EB8619DDE9098754F8094066
:10223000DDF820C0C4F3436BC4F3410904F0010A84
:10224000002918BFC1F800B0B8F1000F18BFC8F8D6
:102250000090002F18BFC7F800A081094FF00108B7
:102260005BD0B8EB901F1CBFBDE8F00F704706EBCA
:1022700045003E49404C51F8201054F820B005EB81
:102280004500800100EB861000F1804000F5A04081
:10229000D0F850A9364C0020A4FB015464084FEA42
:1022A0008409A4EB84042144CF004FEA8B0508FA8B
:1022B00000F111EA0A0F2AD009EBC00101F18041B7
:1022C00001F5A041D1F8801CF940840004F180445C
:1022D00004F5A044C9B2D4F8A86CD4F8BC4CEE40C4
:1022E00006F00F06EC4004F00F041AB16400A41CC1
:1022F00042F8044B1BB17400A41C43F8044BBCF11E
:10230000000F04D001EB810189004CF8041B401C34
:102310000528CCD3BDE8F00F7047C4F30740C4F3E1
:10232000C311C4F3C30412B16400A41C146013B13C
:102330004900891C1960BCF1000F04BFBDE8F00F13
:10234000704700EB80008000CCF80000BDE8F00F83
:102350007047084A8009002952F82000C16914BF5B
:1023600041F0200121F02001C16170479C6F020003
:10237000ABAAAAAA7C6F0200B46F0200CDCCCCCC71
:10238000F749800951F82000C069C0F34010704738
:1023900030B490B000224FF48045EC466C1001E060
:1023A000082A05D2531C03EB8303B5FBF3F304E0C7
:1023B000D31F03EB8303B4FBF3F35B1A48BF5B4209
:1023C0004CF82230521C102AEAD30023009C012131
:1023D0005CF82120A242BCBF14460B46491C1029C0
:1023E000F6D300F00F0202EB42014FEA8111C0F375
:1023F000011C01EB8C1101F18041840901F5A04120
:102400002AD00124B4EB901F1EBF10B030BC70471F
:102410000CEB4200D1F850C9D24A12F820200F2507
:10242000910000208D4003F00F028A4004FA00F171
:1024300011EA0C0F0AD0810001F1804101F5A041A1
:10244000D1F8D03CAB431343C1F8D03C401C052825
:10245000ECD310B030BC7047D1F8680163F30300CF
:10246000C1F8680110B030BC704781091CBF002062
:10247000704700F00F0101EB41018901C0F3011029
:1024800001EB801000F1804000F5A040D0F8680119
:1024900000F00F00082834BF401CC01F00EB800074
:1024A00034BF4FF480414FF40051B1FBF0F070475E
:1024B0002DE9F0074FF0010991B0B9EB901F1EBF55
:1024C00011B0BDE8F007704700F00F02C0F3011033
:1024D00000EB420302EB4202920102EB8010DFF8B4
:1024E00084C200F1804000F5A0405CF82330D0F8B1
:1024F00050A90F204FEA83084FF0000C4FF480469C
:102500006C4600FA08F709FA0CF010EA0A0F36D008
:1025100051F8043B00204FF4005501E0082805D293
:10252000421C02EB8202B6FBF2F204E0C21F02EB95
:102530008202B5FBF2F2D21A48BF524244F8202080
:10254000401C1028EAD30025009B012054F82020CD
:102550009A42BCBF13460546401C1028F6D34FEAEA
:102560008C0000F1804000F5A040D0F8D02C05F0A0
:102570000F03BA4303FA08F31A43C0F8D02C0CF146
:10258000010CBCF1050FBED311B0BDE8F0077047D8
:1025900070B40124B4EB901F1CBF70BC704700F0F6
:1025A0000F02C0F3011000EB420302EB4202920162
:1025B000DFF8B0C102EB801000F1804000F5A040D0
:1025C0005CF82330D0F850C900209B004FF48045C0
:1025D0006E1004FA00F212EA0C0F16D0820002F11B
:1025E000804202F5A042D2F8D02CDA4002F00F026D
:1025F000082A34BF521CD21F02EB820234BFB5FB43
:10260000F2F2B6FBF2F241F8042B401C0528E0D3AD
:1026100070BC704700F00F02C0F3011303EB4202DD
:10262000504B8009A3F1380C53F822205CF82000AD
:1026300001230029D0F8101403FA02F214BF114349
:102640009143C0F81014704700F00F01C0F301135C
:1026500003EB4101434B0022800913F82110383B62
:1026600053F82000D0F81004012303FA01F10842C6
:1026700018BF01221046704770B410F0300F14BF1D
:10268000012300238609DFF8D8C000F00F024FEACB
:1026900090104FF49A7502EB42025CF820004FF064
:1026A000010405EB821214D085584FEA430C5B42BB
:1026B0000CEB43039B1C04FA03F35B1E03FA0CF4BC
:1026C000194025EA040401FA0CF12143815070BC41
:1026D00070470029815804FA03F31ABF1943815047
:1026E0009943F3D070BC704730B410F0300118BF7C
:1026F000012184094FEA9013194D00F00F0000EBFF
:1027000040004FF49A7202EB801255F823004FF00C
:10271000010C0CD082584800C240494200EB4100F5
:10272000801C0CFA00F0401E30BC104070478058EE
:102730000CFA01F1084018BF012030BC7047084B6B
:10274000800953F820C0CCF8741053F820C01168E9
:10275000CCF8781053F820005168C167704700002A
:102760007C6F0200B46F0200C0490028D1F8AC00B1
:1027700014BF40F0020020F00200C1F8AC00704726
:10278000BA490028D1F8AC0014BF40F0010020F095
:102790000100C1F8AC007047B448D0F8E000B4497B
:1027A000096808437047B149C1F8E400B1490860BD
:1027B0007047AE48D0F89800AF49096840EA410038
:1027C000704770B44FEA0075860900F00F044FEAB5
:1027D000D565C0F30110A5F1020502F0010C054416
:1027E0004FEA8C334FEA520012D001EB41017CB327
:1027F00005EB4502D20002EB8C3202EB810101EBCA
:10280000800000F1405000F5C030406A70BC704755
:1028100001EB410202EB01117CB198226A4302EB09
:102820008C3202EB810101EB800000F1405000F599
:102830008030D0F88C0E70BC704703EB810101EB47
:10284000800000F1405000F58030006870BC704797
:10285000FFE703EB810101EB800000F1405000F540
:10286000C030006870BC7047F0B44FEA007687094A
:1028700000F00F044FEAD666C0F30110A6F102067D
:1028800002F0010C06444FEA8C354FEA520012D098
:1028900001EB41017CB306EB4602D20002EB8C3225
:1028A00002EB810101EB800000F1405000F5C030E7
:1028B0004362F0BC704701EB410202EB01117CB1B5
:1028C0009822724302EB8C3202EB810101EB800013
:1028D00000F1405000F58030C0F88C3EF0BC7047ED
:1028E00005EB810101EB800000F1405000F58030E4
:1028F0000360F0BC7047FFE705EB810101EB80004E
:1029000000F1405000F5C0300360F0BC704783090F
:1029100000F00F02C0F301100CD0002A08BF574886
:1029200005D0012A17D000280CBF5548554800EBA8
:1029300081307047002A08BF4FF04050F7D0012A7D
:1029400004D000280CBF50485048F0E7002814BFBE
:102950004F485048EBE7002814BF4F484F48E6E780
:1029600010B44FEA007C840900F00F034FEADC6CDE
:10297000C0F30110ACF1020C604410D0002B08BF72
:1029800047481CD000EB4000C00000EB813002EB58
:10299000420100EB8100434910BC08447047002B02
:1029A00008BF41480BD09823584300EB813002EB1D
:1029B000420101EB021100EB81003C49ECE710BC45
:1029C00000EB813070472DE9F0074FEA901C00F0D2
:1029D0000F04374804EB440150F82C0000F5C07395
:1029E00000EB8110D0F800014FF47A7280B2B2FB94
:1029F000F0F100FB1120002818BF01200D182D4F09
:102A0000002040F2FF1644EA001141EA8C1101F067
:102A10000F02C1F3011101EB420157F821104A08DE
:102A2000C90753F82280C90E03EB820228FA01F885
:102A3000D2F80CA0A8EB050906FA01F8C9F30809B9
:102A40002AEA080A09FA01F14AEA0109C2F80C90D7
:102A5000D2F8189029EA080848EA01019161401C5F
:102A60000228D0D3BDE8F0077047000000500040B6
:102A7000E0580040E4580040985800400080003082
:102A8000E4810030248300304C1800304C1D0030AD
:102A9000CC0E0030CC09003064810030248000303E
:102AA0000080013024800130000001308C0E0130A4
:102AB0007C6F0200846F0200FDF7C2BF10B5FDF706
:102AC000BFFF012818BF10BD0020FDF774FF2121B2
:102AD0000020FDF7BBFF2121BDE810400120FDF7DC
:102AE000B5BF10B5FDF760FFFDF7AAFF01280AD1B9
:102AF0000020FDF760FF21210020FDF7A7FF212125
:102B00000120FDF7A3FF0121052001F03CFE01217A
:102B1000052001F038FEFA490020487110BD10B5BB
:102B20004FF4066001F085FEBDE810404FF40660EA
:102B300001F070BEF24A0146D078002818BF01208B
:102B4000002918BF0121D170002111717047EC4A92
:102B5000516A506208467047E94900208870487001
:102B60007047E7490020887048700871704710B5B9
:102B7000044601468422E3481EF0EEFD04F1840180
:102B8000BDE810408422E0481EF0E6BD70B50007A5
:102B9000C00E0D46801E00EB400101EB0014DB4827
:102BA0004FF4987200EBC40029461EF0D5FDD848BA
:102BB00005F5987100EBC400BDE870404FF49872C1
:102BC0001EF0CABDDFF84CC348B14A424FF48063DF
:102BD00000EB810103EB820260461EF0BDBD4FF4A5
:102BE000806160461EF0BDBD2DE9F0410546002024
:102BF000FDF76AFFC84FDFF824830446EDB14C208F
:102C000004FB00F21646294638461EF0A5FD324662
:102C100005F5E46140461EF09FFD04EB440000EB27
:102C2000041407EB84004C211EF09BFD08EB84008C
:102C3000BDE8F0414C211EF094BD4C21401C4143A5
:102C40000C4638461EF08DFD21464046BDE8F04159
:102C50001EF087BD10B5AA4CE061FEF701FAFEF741
:102C6000BAF961696269C1F307216FF30F0262610A
:102C70006369C2B243EA02226261022803D1626937
:102C800042F00102626181421ABFA269002A10BDAE
:102C9000012918BF0021012818BF0020814208BF68
:102CA00010BDBDE8104010474FF04020816941F051
:102CB00002018161016941F00301016100F0F1BF8E
:102CC0002DE9F0414FF04022054690690C4640F056
:102CD00002019161106940F00300106100F0E1FF12
:102CE0000027002C7ED00020FDF765FE0020216823
:102CF000FEF756F840206168FEF752F82846FFF7C5
:102D0000A9FF0020FDF711FF0126002832D0A0689E
:102D1000FFF76AFF7F48636953B1E1694FF4806C44
:102D20004A420CEB820203EB81011EF015FD1AE012
:102D30007B4D4FF480611EF014FD002029560029C0
:102D40000EDB0A09120202EB800202F1405202F588
:102D500000320907C90E136806FA01F11943116020
:102D6000401C2628EAD36F48A16969B14FF400726C
:102D70001EF0F2FCE068A0B30120FDF7D6FEDFF8FC
:102D80008C81634E28B108E04FF400711EF0E9FC1D
:102D9000F0E71120FDF7C9FE68B1E56840464FF441
:102DA000987229461EF0D8FC30464FF4987205F50B
:102DB00098711EF0D1FC0220FDF7B7FE18B9122061
:102DC000FDF7B3FE68B1E56857484FF4987229469D
:102DD0001EF0C2FC55484FF4987205F598711EF02C
:102DE000BBFC00E014E04120FDF79FFE18B9512024
:102DF000FDF79BFE60B1246954B18422214641480D
:102E00001EF0AAFC842204F184013F481EF0A4FCB9
:102E10003B488770477007714762C1780021C170D5
:102E200007714FF4066001F004FDBDE8F0414FF476
:102E3000066001F0EFBC10B50020FDF7BCFD00F00E
:102E400020FF2F48006B002808BF10BD4FF0402026
:102E5000016921F003010161816921F002018161B1
:102E600010BD4FF4066001F0DABC10B54FF40660F7
:102E700001F0D5FCFDF7E4FD01280AD10020FDF7A3
:102E80009AFD21210020FDF7E1FD21210120FDF720
:102E9000DDFD2748D0F8401321F48031C0F84013FD
:102EA0000020FDF788FD00F0ECFE1548006B0028BF
:102EB00008BF10BD4FF04020016921F003010161FE
:102EC000816921F00201816110BD10B501F0ACFCF7
:102ED00010F0600018BF012010BD094A916990618F
:102EE000084670470648C069704705484069704702
:102EF00072B603494A6922EA0000486162B6704727
:102F0000308400100080013000C001308C0E013090
:102F10008C4E0130000002300000013000400130D2
:102F2000688B001000400230BC0F0130BC4F0130F4
:102F300000500040FE480078002818BF012070476C
:102F400070B5FDF77DFD002818BF70BD0024F84D59
:102F5000AC706C7021212046FDF778FD2121012005
:102F6000FDF774FD2C70BDE870400120FDF723BD16
:102F700070B50446FDF764FD002818BF70BD002140
:102F8000EB4DA970697021210020FDF75FFD212123
:102F90000120FDF75BFD022C3CBF0120FDF766FD23
:102FA000012028702C62BDE87040FDF704BD10B50B
:102FB000FDF746FD002818BF10BD0020DC4CA070B6
:102FC00060702121FDF742FD21210120FDF73EFD2A
:102FD0000120FDF74BFD012020702062BDE810406C
:102FE000FDF7E9BC0020FDF7E6BC10B5D04C002091
:102FF000A07060702121FDF729FD21210120FDF73E
:1030000025FD207800281CBF0120FDF72FFD0120A1
:10301000BDE81040FDF7CFBCC54988627047C44881
:10302000806A7047C249C8627047C148C06A704729
:10303000BF4A00F00F00D16A21F00F010843D062AF
:103040007047BB4890F82C0000F00F00704770B537
:10305000B74C0546A06A421CA262E16A11F0800FDB
:1030600014BFC1F3021101F00F0139B1B2FBF1F04D
:1030700001FB1020002808BFFEF7B7FE207850B1F2
:10308000206A10B1206A401E2062206A002804BF16
:103090000020FDF790FC20212846FDF7D7FC616A4F
:1030A00000291CBF28468847FDF795FF022815D147
:1030B000A048D0F8481311F0010F0FD0D0F84813F2
:1030C00041F00101C0F84813D0F8481321F0010184
:1030D000C0F84813606940F00200606196480168DA
:1030E00041F02001016070BD0020B0E70120AEE793
:1030F00010B5FFF751FB0446FFF755FB8F4804421C
:1031000008BF10BD8A48416941F0040141610E21A8
:1031100001EAD43104F001020A43416962F31F411C
:1031200041618548016841F02001016010BD00281F
:1031300018BF01207E490863704781487047814865
:1031400070477B48406B704779488179027A914299
:1031500014BF806BC06B70477548C06B70472DE91A
:10316000F04F0025DFF8D8918DB009F14C04AC4642
:103170006F1E09F8057004F805C06D1C262DF8DBDC
:103180000025002805DD565D09F805606D1CA84284
:10319000F9DC00220126CDF804C06D46CDF800C050
:1031A000002821DD19F902B0BBF1000F19DBBBF1DA
:1031B000140FA8BFABF1140B04DABBF10A0FA8BFC0
:1031C0000BF1120BBBF1260F0BD24FEA5B180BF081
:1031D0001F0B55F828A006FA0BFB4AEA0B0A45F824
:1031E00028A0521C8242DDDB002292460DF1080825
:1031F0004FEA521B02F01F0E55F82BB006FA0EFED6
:103200001BEA0E0F1ABF08F802A00AF1010A08F81B
:103210000270521C262AEBDB4FF0000A002816DD54
:1032200019F90A20002A0EDB142AA8BF143A02DA80
:103230000A2AA8BF1232262A3ABF18F8022004F838
:103240000A2004F80A700AF1010A8245E8DBDFF877
:10325000E09000220028C9F834C009DD14F902A06A
:10326000924502D0C9F8344002E0521C8242F5DB9C
:10327000354A0020A2F17204A2F1260A27540AF866
:1032800000C002F800C0401C2628F7DB00200029FF
:1032900006DD13F800B004F800B0401C8142F8DCF1
:1032A0000020CDF804C0CDF800C0002913DD23565E
:1032B000002B0DDB262B0BD24FEA531B03F01F0311
:1032C00055F82BE006FA03F34EEA030345F82B30DA
:1032D000401C8842EBDB002003464FEA501B00F005
:1032E0001F0E55F82BB006FA0EFE1BEA0E0F1ABF82
:1032F00008F800305B1C08F80070401C2628ECDB46
:10330000002000290ADD2356002B04DB262B3CBFBE
:1033100018F803301354401C8842F4DB0020C9F82D
:103320003CC0002918DD1356834212D00EE0000085
:10333000308400100050004080840010010007001D
:10334000688B00108E8B0010008C0010C9F83C2098
:1033500002E0401C8842E6DB11F0010F18BF252077
:1033600015D0420900F01F0355F8222006FA03F396
:103370001A420AD1420900F01F0055F8223006FA1D
:1033800000F0184345F8220001E0401EE9D5002076
:103390000246430900F01F0B55F8233006FA0BFBD9
:1033A00013EA0B0F1ABF08F80020521C08F800702F
:1033B000401C2628EDDB002000290BDD2256002AC8
:1033C00005DB262A3CBF18F802200AF80020401C22
:1033D0008842F3DB0020C9F838C00029DCBF0DB0FB
:1033E000BDE8F08F1AF90020824204D0C9F838A055
:1033F0000DB0BDE8F08F401C8842F3DB0DB0BDE896
:10340000F08FFE487047FE48006C70472DE9F001D0
:10341000FA4C002282B0551E04F1050CA5540CF89C
:103420000250521C052AF9DB00228B5CA354521C6B
:10343000052AFADB00230127194600280AD962561B
:10344000002A04DB052A3CBF07FA02F21343491C99
:103450008142F4D300210A466E4607FA01F818EAC1
:10346000030F1ABF7254521C7554491C0529F4DB12
:10347000002100280AD96256002A04DB052A3CBF35
:10348000B25C0CF80120491C8142F4D3DC4B0021D2
:10349000002819649EBF02B0BDE8F00170471CF916
:1034A00001208A4205D0C3F840C002B0BDE8F00157
:1034B0007047491C8142F2D302B0BDE8F001704769
:1034C00040F2DB114843CF4901EB80007047CE4901
:1034D000C0EB001001EBC0007047DFF824C3012BE4
:1034E0008CF806008CF8071003D9401C20F001006E
:1034F00011468CF808008CF8091000FB01F24FF619
:10350000FF7101EA4202ACF8102001EA4000ACF879
:1035100012007047BA48407A7047B948007A70473D
:10352000B74A9072D1727047B548C07A7047B448B4
:10353000807A7047B54A107051707047B349085C83
:1035400070472DE9F047DFF8B892044699F8030078
:10355000002804BF99F801001EF008F90AF0C3FE24
:1035600028B9002301227F2107200EF0F5FD99F8EC
:103570000400002808BFBDE8F0874FF00008D9F824
:103580001C0047464646454610F0070F1CBFDFF8B3
:10359000748210F0020F05D0B9F81010994A21F08A
:1035A00001018F1810F0F00F18BF974E10F4774FED
:1035B00018BF974DD9F828002060FDF70FFD10F0D7
:1035C000010F06D0FEF7CBF8022828BF99F80200B9
:1035D00000D20020E760C4E90108C4E904650120C5
:1035E000BDE8F087864900200871704770B5054630
:1035F0000020FDF769FA4C2100FB01F214468549D1
:1036000028461EF0A9F8224605F5E460BDE87040A2
:1036100081491EF0A1B8F0B583B00020FDF754FA3F
:10362000044669460020FEF734FA0022002C2AD90D
:103630006E464FF0010C4FF6F07502EB4200002190
:1036400000EB02104B0901F01F0756F823300CFA6B
:1036500007F73B4211D0CB075B0C03EB80034F080D
:1036600003EB870303F1405303F580331B889BB2C0
:10367000AB4202D903B00020F0BD491C2629E1D39A
:10368000521CA242D9D303B00120F0BD70B500078F
:10369000C00E0D46801E00EB400101EB00145F4898
:1036A0004FF4987200EBC40128461EF055F85C48B0
:1036B0004FF4987200EBC40105F59870BDE87040B6
:1036C0001EF04AB82DE9F04F07460007C00E83B040
:1036D000801E002527F03F0BE9464FF001084FF60A
:1036E000F0760290384665F31F1040EA0B0000F0B8
:1036F000FF0A5046FDF719FA00283DD05046FEF764
:103700006AFA08FA00F4022C88BF0224694650467F
:10371000FEF7BFF90022002C2ED9029898212844E8
:1037200000FB01FA02EB4200002100EB021C4809F9
:1037300001F01F0359F8200008FA03F3184215D0CE
:1037400001F001000AEB803000EB8C004B0800EB2D
:10375000830000F1405000F58030B0F88C0E80B24C
:10376000B04203D903B00020BDE8F08F491C2629E0
:10377000DDD3521CA242D5D36D1C022DB2D303B0AF
:103780000120BDE8F08F10B50446842225491DF0C4
:10379000E3FF04F18400BDE81040842222491DF0BB
:1037A000DBBF2DE9F04F83B0002002904020FDF7F1
:1037B000BCF9E9464FF001084FF6F077B0B340206E
:1037C000FDF782F9044669464020FEF762F90022BF
:1037D000002C3AD9002102EB420C480959F820305C
:1037E00001F01F0008FA00F0034228D0C807400C7F
:1037F00000EB8C004B0800EB830018E07484001091
:1038000030840010C81E0110342601103C840010C2
:103810002427011000000130004001308C0E0130DF
:103820008C4E01300080013000C001300DE000F10D
:10383000405000F5C030008880B2B84254D8491CCE
:103840000529CAD3521CA242C4D301267000A0F19C
:10385000020B002546EA0510C0B240F0400A50466F
:10386000FDF763F9B8B35046FEF7B5F908FA00F46E
:10387000022C88BF022469465046FEF70AF900214F
:10388000002C28D90BEB050000EB40004FEAC00AE2
:10389000002001EB410C420900F01F0359F82220DF
:1038A00008FA03F31A4210D000F001020AEB823248
:1038B00002EB8C02430802EB830202F1405202F554
:1038C000C032928C92B2BA420ED8401C0528E2D384
:1038D000491CA142DCD36D1C022DBBD3701CC6B2A7
:1038E000022EB3D901200290029803B0BDE8F08FF8
:1038F0002DE9F04100268E4D00280C4645D000F001
:103900000F01C0F3011001290EBF00210229BDE8FB
:10391000F081022828BFBDE8F0810F18FDF790F86C
:103920005FEA00081CBF0020FDF745F8002398203F
:10393000474303EB4300002200EB031C02F00100AD
:1039400007EB8030510800EB8C0000EB810000F1A8
:10395000405000F58030521CC0F88C4E262AEDD322
:103960005B1C022BE5D3B8F1000F08BFBDE8F08166
:10397000AE706E7021210020FDF768F82121012032
:10398000FDF764F82878A0B330E0FDF759F8070098
:103990001CBF0020FDF70FF8002303EB43000022BB
:1039A00000EB0310D107490C4FEA520C01EB8001E8
:1039B00001EB8C0C0CF1405C0CF5803C521CCCF8FB
:1039C0000040262AEED35B1C312BE6D3002F08BF24
:1039D000BDE8F081AE706E7021210020FDF736F851
:1039E00021210120FDF732F8287810B10120FDF7E0
:1039F0003DF8BDE8F0410120FCF7DDBF10B5FDF753
:103A0000E8FF4B49C88110BD494B10B4E02101EAE1
:103A1000102CDB89C1B2C0F30422994288BF194639
:103A200064246143B1FBF3F102EBC20303EB021226
:103A300001EB82014FF47A723E4B0CFB02F2A3FBC6
:103A400002329208521C520810F4803F08BF4942CB
:103A500010F4003F14BF8818881A00B210BC7047D9
:103A600010B5354C4FF4806134481DF07AFE0020CB
:103A700001232156002910DB0A09120202EB800201
:103A800002F1405202F500320907C90ED2F800C017
:103A900003FA01F14CEA01011160401C2628E8D329
:103AA00010BD10B5244C4FF4806124481DF059FE20
:103AB000002001232156002910DB0A09120202EB23
:103AC000800202F1405202F500320907C90ED2F815
:103AD00000C003FA01F14CEA01011160401C2628E4
:103AE000E8D341F2EC0116481DF03BFEBDE8104062
:103AF00041F2EC0113481DF034BE0D4810B5C06909
:103B000011490840FFF7A6F84FF480610B481DF0FB
:103B100028FE40F68C610A481DF023FE40F68C61B9
:103B200008481DF01EFEBDE810400020FDF729BD2D
:103B300030840010ABAAAAAA688B001000000230E3
:103B400000000130004001300100FF0082B04FF45E
:103B5000FA62009013E000BF00BF00BF00BF00BFCB
:103B600000BF00BF00BF00BF00BF00BF00BF00BF5D
:103B700000BF00BF00BF0198411E0191EBD2009829
:103B8000411E009128BF0192F5D202B070472DE985
:103B9000F0410027634D0126002808BF2E701FD07A
:103BA00001282F7018BF6F701AD04FF04028D8F836
:103BB000100040F00400C8F8100029785A4C002981
:103BC00014BF49F608305948E06014BF58484FF018
:103BD000BB70A0605748006830F0FF0206D101E0DA
:103BE0006E70E2E7E26860F30302E26089B1A06808
:103BF00040F01800A0600120FFF7A8FFA06840F483
:103C00008050A0600120FFF7A1FFA06840F4007081
:103C1000A0600120FFF79AFF687870B1E06840F07B
:103C20002000E060A06820F40070A0600120FFF791
:103C30008DFFE06840F01000E060D4F8B00040F084
:103C40000100C4F8B0000120FFF780FFE6674FF4E1
:103C5000E0602061C4F888702878002818BFC4F894
:103C60009460E06820F03000E060A06820F490509C
:103C7000A060D8F8100020F00400C8F81000BDE8DB
:103C8000F0812948C16821F03001C160816821F4C8
:103C9000905181604FF04020016921F004010161E1
:103CA00070474FF04020016941F0040101611D4956
:103CB0001D480A783AB1826842F018028260826830
:103CC00042F490528260497819B1C16841F03001E4
:103CD000C160D0F8B01041F00101C0F8B0107047D9
:103CE000B0F5007F28BF40F2FF10C0F30800124972
:103CF00041EA00200C49086470470B494FF020400E
:103D000008647047084A116C4FF020401064506CF2
:103D100011F0FF0FC0F308201CBF41F020411164D7
:103D2000704700007E8400100060004005F4010030
:103D300020009B00D0FE0400130000A04FF04020A4
:103D40000021016302224263826B02F03C0242F0D6
:103D500001028263026922F003020261026A22F018
:103D600001020262424A136843F0010313603C22DD
:103D700082612822C2613F4801603F4801603F489C
:103D800050F88C2F42F4805202603D4A481E106069
:103D90003C480160704710B501F0F9FA39480468F1
:103DA000002C08BF30BFFAD00021016001F0F3FA07
:103DB000204610BD10B501F0EAFA324B00204FF05A
:103DC000402101221C6824B1186001F0E4FA204669
:103DD00010BD72B6D1F838C00CF03C0CC1F838C038
:103DE0000A6320BF0863D1F838C00CF03C0C4CF0DB
:103DF000010CC1F838C062B6BFF36F8FBFF34F8FAD
:103E0000E0E710B504460F2000F0F8FC0F2000F0AA
:103E1000DDFC1D490A6842EA0400086010BD1A4929
:103E20000A6822EA000008607047164A516850602C
:103E30000846704770B51448006814490968114D68
:103E400000EA0104696800291CBF2046884714F075
:103E5000100F05D0094850F88C1F41F480510160C3
:103E600007480460286840F40040286070BD0000E6
:103E70000048004024480040104800400030004006
:103E800014480040808400101C480040184800403E
:103E9000704770470022B2EBD10F26D20368B3F10E
:103EA000FF3F04BF4368B3F1FF3F17D18368B3F10D
:103EB000FF3F04BFC368B3F1FF3F0FD10369B3F104
:103EC000FF3F04BF4369B3F1FF3F07D18369B3F1FB
:103ED000FF3F04BFC369B3F1FF3F01D0002070472B
:103EE0002030521CB2EBD10FD8D30120704710B450
:103EF0000023B3EBD20F30D2D0F800C00C68A44539
:103F000022D1D0F804C04C68A4451DD1D0F808C017
:103F10008C68A44518D1D0F80CC0CC68A44513D146
:103F2000D0F810C00C69A4450ED1D0F814C04C696B
:103F3000A44509D1D0F818C08C69A44504D1D0F8A3
:103F40001CC0CC69A44502D010BC002070472030B2
:103F500020315B1CB3EBD20FCED310BC01207047D5
:103F60002DE9F041054601F01AFA002021264FF410
:103F7000825784464FF4E0221660C5F800C01168ED
:103F800041F004011160116811F0040FFBD11760BA
:103F900080232C460021D4F80080B8F1FF3F04BFF5
:103FA000D4F80480B8F1FF3F1DD1D4F80880B8F1EF
:103FB000FF3F04BFD4F80C80B8F1FF3F13D1D4F811
:103FC0001080B8F1FF3F04BFD4F81480B8F1FF3F70
:103FD00009D1D4F81880B8F1FF3F04BFD4F81C8091
:103FE000B8F1FF3F08D0C2F800C0401CC0B208289A
:103FF000C2D30220BDE8F081491C2034B1EBD30FBD
:10400000C9D3C2F800C00120BDE8F0812DE9F0411C
:10401000054601F0C4F90020092684464FF4E02348
:104020001E60C5F800C0196841F0040119601968E4
:1040300011F0040FFBD12C464FF480620021276859
:10404000B7F1FF3F04BF6768B7F1FF3F17D1A7681B
:10405000B7F1FF3F04BFE768B7F1FF3F0FD1276912
:10406000B7F1FF3F04BF6769B7F1FF3F07D1A76909
:10407000B7F1FF3F04BFE769B7F1FF3F08D0C3F8CE
:1040800000C0401CC0B20328CAD30220BDE8F081A2
:10409000491C2034B1EBD20FD1D3C3F800C00120AA
:1040A000BDE8F0812DE9F05F8846814604274FF096
:1040B0007F0A4FF0020B4FF4E02601F070F94946F9
:1040C000424653464FF0060CC6F800B052F8040BB7
:1040D00041F8040BC6F800C0306810F0040FFBD1A3
:1040E0005B1EF1D2002030604C4645461F20D4E9CB
:1040F00000C3D4E90221D5F800E0E64504BFD5F8B5
:1041000004C09C4505D1AB68934204BFEA688A426B
:1041100008D07F1E03D34846FFF722FFCDE70220D9
:10412000BDE8F09F10341035401EE0D20120BDE8FC
:10413000F09F70B50D46044601F031F94FF400725E
:10414000214628461DF008FB012070BD2DE9F041F5
:104150000546C005ADF5007D14460E46C00D25D0C0
:10416000A8466FF308086F4601F019F94FF4007282
:10417000414638461DF0F0FAC5F30800C0F5007757
:10418000A74288BF274668443A4631461DF0F3FAF5
:104190004046FFF7E5FE022844D069464046FFF757
:1041A00081FF022843D03D443E44E41BB4F5007F28
:1041B00019D34FF40072314668461DF0DCFA2846E8
:1041C000FFF7CEFE02282DD069462846FFF76AFF8A
:1041D00002282CD0A4F5007405F5007506F50076CC
:1041E000B4F5007FE5D2C4B16F4601F0D8F84FF4C2
:1041F0000072294638461DF0AFFA2246314668461D
:104200001DF0B9FA2846FFF7ABFE02280AD069462E
:104210002846FFF747FF022809D00DF5007D012051
:10422000BDE8F0810DF5007D0A20BDE8F0810DF5B7
:10423000007D0B20BDE8F08130B4354D2A680021A7
:1042400001244FF0030C04FA01F3034204D04B00A5
:104250000CFA03F39A431A43491C0C29F3DB2A6036
:1042600030BC7047F0B42A4D2A68002101244FF079
:10427000030C022604FA01F3034206D04B000CFAA9
:1042800003F7BA4306FA03F31A43491C0C29F1DB7E
:104290002A60F0BC70472DE9F001002201251D4C79
:1042A0000F2605FA02F3034217D0D31702EB537C13
:1042B0004FEAEC0304EB83031F682CF0070CA2EB1E
:1042C0000C0C4FEA8C0C06FA0CF827EA080701FAE6
:1042D0000CFC47EA0C0CC3F800C0521C0C2AE0DBB3
:1042E0000B498A6A22EA00008862BDE8F001704743
:1042F00007498A6A1043886270470548416821F07F
:1043000080014160416821F4007141607047000004
:104310000010004020100040704772B64FF040205F
:10432000816941F040018161C16941F04001C16191
:1043300062B6016A41F00101016270474FF040200E
:10434000016A21F00101016272B6C16921F04001E8
:10435000C161816921F04001816162B6704710B589
:1043600072B64FF04024A06940F04000A061E069BF
:1043700040F04000E06162B6206A40F00100206237
:10438000D94843F63F71C160002181638164C0F860
:10439000D01003210A2000F0F6F90A2000F016FAE6
:1043A000206A20F00100206272B6E06920F040002F
:1043B000E061A06920F04000A06162B610BDCA4A69
:1043C00010605160484390607047C74A1060516068
:1043D000484310F0010F18BF401C90607047C2495D
:1043E000C1F8D0007047C049002818BF0120886478
:1043F0007047BD498863C86840F00200C8607047D4
:10440000DFF8E4C2CCF82000CCF82410CCF8282047
:10441000CCF82C300120CCF83000DCF8340010F05F
:10442000010F05D020BFDCF8340010F0010FF9D1E6
:1044300010F0020018BF4FF0FF307047AA48C16863
:1044400021F00201C1607047A748C16841F0010135
:10445000C1607047A44B186259629A6201201864C7
:10446000586C10F0010F04D020BF586C10F0010FF1
:10447000FAD110F0060018BF4FF0FF3070479A488D
:10448000C16821F00101C16070479748C16841F0DF
:104490000401C1607047944A8189116701685162C3
:1044A000416891628168D16201211165516D11F0FD
:1044B000010F04D020BF516D11F0010FFAD1536FDD
:1044C0000361936F1B148382936FC3F30523C3822D
:1044D000936F03F03F030383D36F1B144383D36FA6
:1044E000C3F305238383D36F03F03F03C383D2F861
:1044F0008030C3F309430384D2F88020C2F3090259
:10450000428411F0020018BF4FF0FF307047764828
:10451000C16821F00401C16070477348C16841F06F
:104520000401C1607047027C017B02F03F0241EA56
:1045300002416D4A916501685162416891628168EA
:10454000D16201211165516D11F0010F04D020BF1E
:10455000516D11F0010FFAD1D36D8382D36D1B0C15
:10456000C382136E0383136E1B0C4383536E8383CA
:10457000526EC2F30E42C28311F0020018BF4FF018
:10458000FF3070475848C16821F00401C16070478E
:104590005548C16841F00801C1607047DFF848C163
:1045A000CCF89820CCF82000CCF82430CCF8281097
:1045B0000120CCF89000DCF8940010F0010F05D039
:1045C00020BFDCF8940010F0010FF9D110F00600C4
:1045D00018BF4FF0FF3070474348C16821F0080111
:1045E000C160704701684FEA31423F49C1F8BC20C1
:1045F0004068C1F8C000C86840F02000C86070473B
:1046000001684FEA31423849C1F8BC204268C1F81C
:10461000C020027A407A02F0010262F35F00C1F822
:10462000C400C86840F02000C86070472E4B186274
:104630005A6299620120C3F8B400D3F8B80010F0B0
:10464000010F05D020BFD3F8B80010F0010FF9D149
:1046500010F0060018BF4FF0FF307047224A10627A
:1046600051620120C2F8B000D2F8B80010F0010F7A
:1046700005D020BFD2F8B80010F0010FF9D110F02A
:10468000060018BF4FF0FF3070471748C16821F08F
:104690002001C16070471448C16841F01001C16039
:1046A0007047A3F1050C104BC3F8A8C018625A62FA
:1046B00099620120C3F8A000D3F8A40010F0010F04
:1046C00005D020BFD3F8A40010F0010FF9D110F0ED
:1046D000060018BF4FF0FF3070470348C16821F053
:1046E0001001C1607047000000900040234810B5E1
:1046F000022140F8501F012101611021416241F265
:10470000060141610021816104218163902141639F
:10471000416B41F001014163C16B21F40021C16390
:10472000C16B41F40051C163C16B21F00101C16350
:10473000C16B41F00101C1634FF4817101610161FD
:10474000032000F043F80021032000F01CF80020B3
:1047500010BD10B5032000F045F808484FF48071F3
:104760000166002101661021816702214165002058
:1047700010BD034900200870704700000030004061
:1047800088840010704700F00303DA004FF0FF0C3C
:104790000CFA02F24FF0050C0CEBC30301FA03F321
:1047A00000F00C0101F1E021002807DAD1F8140D26
:1047B00090431A401043C1F8140D7047D1F800041B
:1047C00090431A401043C1F80004704700F01F01E5
:1047D000012202FA01F14009800000F1E020C0F856
:1047E0000011704700F01F01012202FA01F1400997
:1047F000800000F1E020C0F88011704700F01F0138
:10480000012202FA01F14009800000F1E020C0F825
:10481000801270474FF0E021C1F8000170474FF05F
:10482000E021C1F8800170474FF0E020D0F800018E
:1048300070474FF0E021C1F88002704708480068D7
:104840007047074A1168106008467047044A1268AA
:1048500000F1100352F8230042F8231070470000C3
:1048600008ED00E002210C20FFF78DBF72B64FF07B
:104870004020816941F480518161C16941F48051D6
:10488000C16162B6704772B64FF04020816921F471
:1048900080518161C16921F48051C16162B6704764
:1048A000AA4881B0016F11F4007FFBD1816E11F035
:1048B000010F1CBFD0F88410009104D0D0F88410F0
:1048C000009A9142FAD0016F11F4007F04BF4CF2BC
:1048D0007101016642F24131816601B070479B4926
:1048E00081B04FF40D528A660A6FCA66012898BFDC
:1048F000012005D9401EB0F5803F28BF4FF6FF705C
:1049000082B24FF05C5040EA022048664FF01140FE
:10491000C1F88000086F10F4007FFBD1886E10F0A2
:10492000010F1CBFD1F88400009004D0D1F884009E
:10493000009A9042FAD0086F10F4007F04BF4CF246
:104940007100086642F24130886601B070477F48C6
:1049500081B0016F11F4007FFBD1816E11F0010F66
:104960001CBFD0F88410009104D0D0F88410009AB5
:104970009142FAD04FF40D51816601B070474FF06B
:104980004020806910F4805008BF70476F48806EE7
:1049900000F0010070476D48406EC0F30F20704773
:1049A0006A48D0F88400704710B50C20FFF726FF46
:1049B0000C20FFF70BFF65490220486710BD6349D3
:1049C00010B5032088670C20FFF70CFFBDE81040EE
:1049D0000C20FFF713BF5E4A11681060084670474D
:1049E0005A4810B5016FC16659480068002818BFC1
:1049F00080475848016841F48051016010BD544817
:104A00004068704710B572B64FF04020816941F49C
:104A100080518161C16941F48051C16162B6032056
:104A20004A4988670C20FFF7DDFE0C20FFF7E6FE01
:104A300000F03CF9484B0420C3F888004FF6FF70A3
:104A4000C3F88C0072B66033FFF749FF4FF4007073
:104A5000186062B610BDF8B572B63C48016F11F42B
:104A6000007FFBD1816E11F0010F1CBFD0F88410C4
:104A7000009104D0D0F88410009A9142FAD04FF4FB
:104A80000D51816634494FF400320A6662B6D1F89E
:104A900004124FF04025002946D02D4C4FF6FF73ED
:104AA000591AA1602A6BD5F834C002F00F020CF03D
:104AB0000F0C6244121D01FA02F2A2F54341DFF825
:104AC0009CC0513961452FD2D0F88400191AE16099
:104AD000B1F5803F28D2224B4FF0000CA1FB030719
:104AE0000CFB037301FB0C3163461CF049FE401CB8
:104AF00040082061B0F57A7F38BF4FF47A70194BC7
:104B00009968002908BF98605A681A609968C3E9D3
:104B100001108A4215D9824205D9814201D96160CA
:104B200002E0606000E0626000F0D0F872B6A86950
:104B300020F48050A861E86920F48050E86162B6F2
:104B4000F8BD8242EFD88142EBD8E8E700C00040D0
:104B50008C8400108084001000A000404F6225006B
:104B600000E1F505288C00104FF04020816941F0EC
:104B7000040181610C48016841F404710160001F67
:104B8000016821F004010160016841F01001016039
:104B90007047064908607047BFF34F8F05490448C6
:104BA0000860BFF34F8FFEE714ED00E008ED00E072
:104BB0000400FA050CED00E04FF04020816941F05F
:104BC000040181610B48016841F0010101600B495A
:104BD0000948C1F8C40070470948006842F27001F2
:104BE0000840704708480749016008498160002172
:104BF000C1607047144C004001005FA0006000409D
:104C000000440040A0C00E0000100040508A59002F
:104C1000022824BF00207047DC4B53F8202043F8C3
:104C200020101046704770B5D94C206FD74D10F04A
:104C3000010F05D00120E0662868002818BF8047D2
:104C4000206F10F0020F08BF70BD0220E066686898
:104C5000002808BF70BDBDE87040004710B572B6AF
:104C60004FF04020816941F080018161C16941F0CC
:104C70008001C16162B60222C5490A6501230B6643
:104C80000323CB664A6572B6816921F08001816198
:104C9000C16921F08001C16162B60920FFF796FD6C
:104CA0000221BDE810400920FFF76DBD72B64FF03C
:104CB0004020816941F080018161C16941F080013A
:104CC000C16162B60220B24908657047B04902204E
:104CD000486572B64FF04020816921F08001816102
:104CE000C16921F08001C16162B670474FF0402078
:104CF0008069C0F3C0107047A548016F11F4007FB0
:104D000014BF4FF440714FF480710166704710B5C5
:104D10009F4CE06F10F0020F4FF0010018BF03200E
:104D2000606700F06DF94FF040210A6B496B02F0AB
:104D30000F02D04001F00F01C8400521B0FBF1F097
:104D40004FF405710009C4F880109249A1FB0010CE
:104D50004009C4F88400206F10F4007F14BF4FF4A2
:104D600040704FF48070206610BD8948016F11F4C7
:104D7000807F14BF4FF440714FF40071016670479B
:104D8000834B30B4DA6F12F0010F14BF03220222FA
:104D90005A6700EB4005C5EBC010C1EBC0004FF4F3
:104DA000FA744C43C0EB001000EB40007A4904EB6E
:104DB000C000A1FB00104FF0402100220C6B4FF00F
:104DC000020CC008496B04F00F0401F00F012144EC
:104DD000C8400521B0FBF1F0B0F5803F05D3511C70
:104DE0004008CAB2B0F5803FF9D242EA0C2141F046
:104DF0001001C3F88810C3F88C00186F10F4807F7E
:104E000014BF4FF440704FF40070186630BC704708
:104E10005F48016F11F4003F14BF4FF440314FF46D
:104E20008031016670475A48016F11F4803F14BF0A
:104E30004FF440314FF40031016670475448006F21
:104E4000C0F3002070475248006FC0F34020704705
:104E50004FF040218969C1F3C011002904BF00202F
:104E600070474B4900280CBFD1F80002D1F804026A
:104E700070474FF040239A69C2F3C012002A04BF62
:104E800000207047424A00280CBFD2F88000D2F8B8
:104E90008800C0F30A200CBFD2F88020D2F8882006
:104EA00002F00F02D3F830C05B6B0CF00F0C03F074
:104EB0000F0363441A449140012202EB400048432F
:104EC0003449A1FB001000097047344901200870E3
:104ED000704770B432224FF0402351431A6BD3F81D
:104EE00034C002F00F020CF00F0C6244121DD140CE
:104EF00008BF012104D0B1F5803F28BF4FF6FF71F4
:104F00009A69C2F3C012002A1CBF70BC704772B607
:104F10009A6942F080029A61DA6942F08002DA61AD
:104F200062B602241A4A1465250415664FF0040C73
:104F3000C2F888C0C2F88C10DFF864C0C2F86CC038
:104F40005467184902283CBF104E46F82010002133
:104F5000124801704FF400711166017819B920BF31
:104F600001780029FBD01566C2F878C0C2F86CC081
:104F7000546572B6986920F080009861D86920F075
:104F80008000D86162B670BC70470000A484001035
:104F900000A000401F85EB51CDCCCCCCA0840010EC
:104FA000020002027B6E00004FF0E02100208861C9
:104FB000086127494860704710B54FF0E0246061F0
:104FC0000020A0610221401EFFF7DDFB07202061C9
:104FD000BDE8104009F0A2B810B509F0A3F84FF0F1
:104FE000E0210020086110BD10B509F09BF84FF0DA
:104FF000E0210020086116480188491C018010BD8D
:105000001348806870472DE9F041114C0027054690
:105010002780A0684FF47A71B0FBF1F04FF0E026E2
:10502000401E7061B7610221C81EFFF7ACFB07206C
:10503000306109F073F82188A942FCD309F072F8B5
:105040003761BDE8F08103494843014988607047F2
:10505000AC84001040420F004FF04020816921F4E1
:1050600000518161C16921F40051C1617047A849B3
:105070000A78824218BF062828BF7047A54AA64B67
:1050800052F830C0C3F808C002EBC0025268DA60C0
:10509000087070474FF04020816941F400518161F0
:1050A000C16941F40051C161704710B50121072069
:1050B000FFF769FB4FF04020816941F400518161A5
:1050C000C16941F40051C161934A002111609349C3
:1050D0005160DFF83CC200219CF800303BB10CF17C
:1050E00010031C6894605B68D3608CF800108C49D6
:1050F0001161816921F400518161C16921F400517C
:10510000C16110BD8248406870478348806970471C
:105110004FF04020806910F4005008BF70477E486F
:10512000006900F0010070474FF04020806910F4E2
:10513000005F04D0784B186910F0010F01D10020F6
:10514000704710B472494FF6FE7000248A684AB165
:105150009A69D1F808C0624504D08C604C6010BCDC
:105160000120704700BF00BF00BF00BF00BF00BFED
:1051700000BF00BF00BF00BF00BF00BF00BF00BF37
:1051800000BF00BF00BF00BF00BF00BF00BF00BF27
:1051900000BF00BF401E0028D8DC8C604C6010BCF3
:1051A000002070475A4988607047594880687047A6
:1051B0005948016941F001010161554901204860E8
:1051C00070475548016921F00101016150490020F3
:1051D000486070470021002808BF4FF0006103D0ED
:1051E000022808BF4FF080614B48026922F04062FC
:1051F00011430161704748490120096901F040618C
:10520000B1F1806F04BF02207047B1F1006F08BF99
:10521000002070474048406970473D48007870471B
:105220004FF04020806910F4005F38D03A4A10698E
:1052300010F0010F33D03648406801282FD0906914
:105240006FF07F43984238BF00EB400C27D2516982
:10525000B1EB9C0F01D30120704700BF00BF00BF1E
:1052600000BF00BF00BF00BF00BF00BF00BF00BF46
:1052700000BF00BF00BF00BF00BF00BF00BF00BF36
:1052800000BF00BF00BF00BF00BF00BF00BF00BF26
:1052900000BF00BF00BF00BF00BF9842D7D30020AF
:1052A000704710B50720FFF7A9FA0720FFF78EFA1D
:1052B0001948016941F01001016110BD164810B58F
:1052C000016921F0100101610720FFF78BFABDE8A9
:1052D00010400720FFF792BA0D4AD168D060084607
:1052E000704738B50C4CE069E061094910F0020FD5
:1052F0001CBFA2698A60C96800291CBF00018847D9
:10530000E06900900748016841F08001016038BD04
:10531000B8840010C884001000D00040D0121300E0
:10532000660F001580840010704770B505464FF475
:105330000D500406A0660320E066264860664CF225
:10534000710020662448C4F8800042F24630A0660E
:1053500002210020FFF717FA0020FFF737FA002D8F
:1053600008BF70BDA06E42F241310843A06670BD17
:10537000012110B5880781674FF40D518166002027
:10538000FFF730FABDE810400020FFF737BA0120E0
:1053900081074867704701208107886770474CF292
:1053A00071008107086670470C4A11681060084652
:1053B00070470A4808B5006818B18047002818BF30
:1053C00008BD4CF2710188070166016FC166006F6C
:1053D000009008BD075E5F3700AF2F91F884001082
:1053E000FE49002088717047FC488079704770B58D
:1053F000FA4C00254FF4E4612570E570F8481CF084
:10540000B0F94FF4E461F7481CF0ABF9A5602571E1
:105410004C21F5481CF0A5F94C21F4481CF0A1F9E9
:1054200065717421F2481CF09CF97421F1481CF05C
:1054300098F9E56070BDE9480079002818BF01209F
:105440007047E6484079002818BF01207047E348BC
:10545000C078002818BF01207047E548704770B534
:10546000E54DE64E044601462A783078E04B10447C
:10547000420018461CF07FF92A783078DD4B104442
:105480004200214618461CF076F9D44801214171AA
:10549000817941F00401817170BDD048C0687047C6
:1054A000CF4870472DE9F041CC4F8046387800282E
:1054B00014BFD348D348057814BFD348D3480478E1
:1054C00005FB04F6FEF729FF21462846FEF777FF85
:1054D000C3494346C34A0846FEF792FFFEF72EFF34
:1054E00072004146BF481CF046F90120F870B879B7
:1054F00040F00100B8710120BDE8F0812DE9F047CE
:10550000B64D044601462878DFF8D4C2DFF8F082B1
:10551000DFF8F092BC4EBD4F002815BF98F8002070
:1055200099F8002033783B7802FB03F04FEA400201
:1055300060461CF020F92878DFF8A8C22146002830
:1055400015BF98F8002099F8002033783B7802FBCB
:1055500003F04FEA400260461CF00DF90120E870AC
:10556000A87940F00100A871BDE8F0879B488068E9
:10557000704770B5A64C0546014622789A485200FD
:105580001CF0F9F822782946520098481CF0F3F8EC
:10559000924801210171817941F00201817170BD50
:1055A0002DE9F04FADF25C7DDFF830820120CDF8BF
:1055B000400798F80300CDF83C0798F80400CDF8B0
:1055C000380798F805B002F063F90446FDF774FA5D
:1055D000CDF85407FDF7AEFCCDF85007FBF7CCFF34
:1055E000CDF84C07FBF7FAFC8246FBF7F4FC0746C4
:1055F000FDF764FAFCF766F80830060998F8010030
:105600000025002804BF0420C8F814002AD002F0A6
:1056100057F98146022C06D009F01EF802280CBF6B
:105620000920072014E016F0A2F948F202110842FE
:105630001CBF3C20C8F814000CD102F05BFA30B15A
:105640000DF0E7FEC0B116F006FA082814D01E20AF
:10565000C8F81400B9F1060F04BF0220C8F81400FE
:1056600088F80150FBF7BAFC10F0010F0CD002F0E3
:10567000ACFA3C2802D007E00F20E9E7FFF748FD2D
:10568000002818BFFFF7CCFD4FF00109022F14D1FD
:1056900002F030FA88B9022C04D0052C08BF05208E
:1056A00007D00AE04FF47A7070434FF47A7190FBA0
:1056B000F1F0C8F8140088F80190D8F81400042814
:1056C000BCBF0420C8F81400D8F8180040B1D8F8BE
:1056D0001C10D8F81400884298BF0846C8E9050590
:1056E00098F80100B8F81410000240EA014040F0B8
:1056F00001020023912107200CF02EFD1AF0010F6A
:1057000025D1022C23D00020FBF73BFFFDF74FFCF7
:105710000025AA4607F007FE01281ED00DF5E4601B
:10572000FDF70FFF002800F0EA810DF5E46008F0B6
:1057300022FBD8F81400C01EA842ACBF01260026E8
:10574000DDF82C0748B3DDF8380750B144E0FDF729
:10575000F7FB0020CDF84007DAE74FF0010A00F030
:10576000B8B96846DDF82C171CF00FF80746AEB143
:10577000274C3946207842001B481BF0FCFF20785C
:105780003946420019481BF0F6FF88F8049098F853
:10579000060040F0020088F806001DE0FEF7BDFD9F
:1057A0001B4C01212078FEF70AFE104A3B46A2F16D
:1057B0004C010846FEF724FEFEF7C0FD207839466E
:1057C00042000A481BF0D7FF88F8049098F80600BA
:1057D00040F0020088F806001CE00000FC84001085
:1057E0005C270110348C001094A10010E0A100107F
:1057F0007C2E01102CA20010698500106A85001013
:1058000067850010648500106885001065850010AC
:105810006B850010DDF82807002800F0D880DDF83F
:105820003C07002840F0D38098F80000DDF82847B6
:10583000002863D1D8F8087027B3FB480078CDF86A
:105840004807FA480078CDF84407FEF766FDDDF812
:105850004417DDF84807FEF7B8FD21463A460846EA
:10586000FEF7F8FDFEF76AFDF1480078022804BF54
:10587000384607F084FFEE480078092804BF204628
:1058800007F07DFFEB480078012811D9E84F387800
:10589000042804BF204607F072FF214668461BF02B
:1058A00079FF04463878052804BF204607F067FFD3
:1058B00002F020F910B301F0EBFF02281ED10DF029
:1058C000A8FD18B116F0C7F8082817D1DA48002249
:1058D0000378DA480778002F10D90020002B0AD966
:1058E00002FB0301401C34F911C083424FEAEC0C67
:1058F00024F811C0F4D8521CBA42EED37EB398F803
:105900000020CF482146002A0CBFCB4AC64A127855
:1059100014BFC64BC94B1B7802FB03F24FEA42028D
:105920001BF029FF98F80000C64B2146002814BF41
:10593000BD48C148007814BFBC4AC04A127800FB79
:1059400002F04FEA400218461BF015FF88F803905A
:1059500098F8060040F0010088F8060030E0FFE704
:10596000CDF8444798F80000002814BFAE48B2486C
:10597000077814BFAD48B148047807FB04F0CDF8B0
:105980004807FEF7CAFC21463846FEF718FDAC4929
:10599000AC4A0846DDF84437FEF732FDFEF7CEFC90
:1059A000DDF84807DDF844174200A6481BF0E3FE87
:1059B00088F8039098F8060040F0010088F8060087
:1059C0009B480078032804BF9D4807F0D8FEDDF807
:1059D0003007002873D0BBF1000F70D1044698F84F
:1059E000000038BBD8F80C7027B397480178974867
:1059F00000780844401C4008019002200090FEF707
:105A00008CFCDDE90010FEF7E0FC21463A46084632
:105A1000FEF720FDFEF792FC8D480078022804BFB7
:105A2000384608F06CF88A480078092804BF2046F8
:105A300008F065F8D6B18748834E844F2146337805
:105A40003A781A4452001BF096FE32783B7882482E
:105A50001A44214652001BF08EFE88F8059098F8F3
:105A6000060040F0040088F8060021E0764826464B
:105A70000178764800780C18FEF74FFC601C40084F
:105A80000221FEF79CFC73493346734A0846FEF731
:105A9000B7FCFEF753FC620031466F481BF06BFE0B
:105AA00088F8059098F8060040F0040088F8060091
:105AB00067480078032804BF664808F020F8FDF71F
:105AC00091FDD8F814006D1CA84211DCD8F8100024
:105AD00070B1FCF7F3FFDDF84C07FBF752FDDDF882
:105AE000540788B1DDF8500760B1FDF760FA0BE0AC
:105AF000DDF84007002818BFFDF759FA0AE601F063
:105B00002DFF07E6FDF71CFABAF1000F04BF0420D1
:105B1000C8F8140010D0DDF83C0788F80300DDF861
:105B2000380788F8040088F805B0C8F81890D8F845
:105B30001400401BC8F81C00B8F814104FEA0A20E3
:105B400040EA01420023912107200CF005FB0DF2F1
:105B50005C7D5046BDE8F08F10B50024FDF7C2F91A
:105B60003E4910F0070F0AD0CA78002A08BF012466
:105B700010F0020F03D00A79002A08BF012410F0A8
:105B8000F00F03D04879002808BF01240020002C22
:105B900008BF10BD00200870BDE8104000E508B542
:105BA00040F20F3102F03EF8012804D1FFF7D4FF94
:105BB000009002F0CEF92948C17800291CBF417934
:105BC000002904D0007900281CBF012008BD002056
:105BD00008BD08B540F20F3102F024F8012804D1C5
:105BE000FFF7BAFF009002F0B4F91C48C178002911
:105BF0001CBF4179002904D0007900281CBF012076
:105C000008BD002008BD7047144910B50022CA70B5
:105C10000A714A7100281CBF012048700DF0E9FA92
:105C2000BDE81040FAF7DFBB6785001068850010FB
:105C3000F9850010668500106485001065850010E8
:105C40005C270110348C0010698500106A850010F3
:105C5000FF8500107C2E01102CA20010FC84001087
:105C6000002818BF0120FE49C8717047FC48C07960
:105C7000704710B54FF4E461FA481BF072FDBDE8BF
:105C800010404FF4E461F8481BF06BBDF7487047D3
:105C9000F7480178F748007848434100F3481BF083
:105CA00060BD70B50646F2480478F2480578FEF704
:105CB00034FB29462046FEF788FBEA4A3146EB488A
:105CC000FEF7C8FBFEF73AFBEB480078152818BF33
:105CD00070BDE648BDE8704007F051BD2DE9F047C2
:105CE0000746E34815460C460678E24890F80080DF
:105CF000FEF713FB41463046FEF767FB3A46D949AB
:105D00001046FEF7A7FBFEF719FB00200221A8F1C1
:105D100002092060B9F1020F84BFDFF84883A6F1C1
:105D2000020C20D90220BCF1020F19D901FB060395
:105D300038F9132002F10A0ABAF1140F06D9D4F87F
:105D400000A0002AB8BF524252442260B5F900A018
:105D500038F913209245B8BF2A80401C6045E5D32E
:105D6000491C4945DED3C4480078162804BF38468C
:105D700007F005FD3846BDE8F087002818BF012070
:105D8000B749C870704710B5B54C002804BFA06073
:105D900010BDDFF8E8C2BA490B78BA490A78014663
:105DA0005A43520060461BF0E6FCB448A06010BDA8
:105DB00010B54C21B4481BF0D4FCBDE810404C2178
:105DC000B2481BF0CEBCB0487047002818BF012075
:105DD000A3490871704710B57421AD481BF0C1FC90
:105DE000BDE810407421AB481BF0BBBC002818BFB5
:105DF00001209B494871704710B5994C002804BF99
:105E0000E06010BD74220146A3481BF0B4FCA24818
:105E1000E06010BD924900208861704770B5904DD8
:105E200000260446EE702E716E710DF0E2F9FAF75D
:105E3000DAFA002C14BF012000202870AE61BDE802
:105E40007040FFF7ADBB2DE9F04F89B04FF4E4612E
:105E50008A481BF086FC74218F481BF082FCFDF7FA
:105E600041F80446FCF728FE0890FDF763F8079018
:105E7000FBF782FB0690FCF721FEFBF7AFF810F072
:105E8000010F0BD001F0A1FE3C2807D1FFF740F92C
:105E900020B10420FFF7EBF8FFF7C2F90020FBF771
:105EA00070FBFDF784F800252E4607F03CFA012828
:105EB00053D06846FDF745FB00285ED0684607F0E2
:105EC0005AFF14F0070F1CD06D48DFF8B0B1DDF8B1
:105ED000089090F800806B48DA460778FEF71DFAC4
:105EE0000120FEF780FA39464046FEF76EFA524628
:105EF00049465846FEF7AEFA0020FEF774FAFEF760
:105F00001DFA14F0F00F20D06448DFF88CB102279E
:105F100001786348DA46DDF8109000780844401CA8
:105F20004FEA5008FEF7F9F90120FEF75CFA39460E
:105F30004046FEF74AFA524649465846FEF78AFA64
:105F40000020FEF750FAFEF7F9F9FDF74BFB6D1C48
:105F5000102D03D2FDF72BF8A7E701260520FFF748
:105F600086F8FCF7ABFD0698FBF70BFB089848B1E9
:105F7000079828B1FDF71BF804E001F0EFFC94E767
:105F8000FCF7DEFFDEBB364F14F0070F1BD03C489A
:105F9000DFF8E8C001783B48E046007801FB00F2FA
:105FA00010200021002A88BF03460AD938F9115071
:105FB00005EB5005B5FBF3F52CF81150491C8A424E
:105FC000F4D82E48B86014F0F00F18D03348324B94
:105FD000017833481C4600780A184FF010014FF042
:105FE00000000AD034F9105005EB5105B5FBF1FC67
:105FF00023F810C0401C8242F4D82748F86009B04A
:106000003046BDE8F08F012070474FF47B30704779
:106010004FF47B3000687047034600209A682C2AB2
:1060200088BF2C220021B1EB920F28BF704753F894
:1060300021C0491C6044B1EB920FF8D37047194A54
:106040000168914239D14168B1F5807F35D98368C3
:1060500000222C2B88BF2C230021B1EB930F23E0CF
:10606000FC8400105C270110348C00105493001045
:106070006485001065850010F9850010749A001081
:10608000678500106885001094A10010E0A1001041
:106090007C2E01102CA20010A0A200106985001017
:1060A0006A8500104353494D09D250F821C0491C5C
:1060B0006244B1EB930FF8D30AB10020704701207E
:1060C00070474FF47B31FE4B0A689A423ED191F8FB
:1060D00027300022012B08BF0122052804BF91F8B8
:1060E0002300704713DC012804BF087F7047022893
:1060F00004BF91F820007047032804BF91F82100E5
:106100007047042804BF91F82200704731E014283A
:1061100008D015280CD0162811D0172804BF18460F
:10612000704726E0002A1CBF91F82400704704E065
:10613000002A1CBF91F8250070472D207047002AC7
:106140001CBF91F82600704728207047052812D000
:1061500007DC01280DD002281CBF032804280AD020
:1061600007E0142818BF1528E7D01628ECD0172808
:1061700001D0FF207047002070472DE9F047ADF5B2
:10618000007D00244FF4007168461BF0EAFAFF20FE
:10619000A04660F307082D20254660F3070560F34D
:1061A0000F25282060F317454FF47B37C44E64F366
:1061B0001F654FF481794FF02C0AFF224FF40071D4
:1061C00068461BF0ECFACDE902A4CDE90648059437
:1061D0000A94CDE900690494CDE908453846FDF7F5
:1061E000BFFE69463846FDF75DFF012818BF002055
:1061F0000DF5007DBDE8F0872DE9F047ADF50C7D8C
:10620000894605461F4690464FF0000A4FF400713C
:106210006846949E1BF0A5FA4FF0000CCDF800C222
:106220004FF47B34CDF804C2CDF808C2CDF80CC2CF
:10623000CDF810C2CDF814C2CDF818C2CDF81CC2EA
:10624000CDF820C2CDF824C2CDF828C29C492068E0
:10625000884206D0FFF791FF0DF50C7D5046BDE852
:10626000F087D4E901120DF5007AE3688AE80F009F
:1062700004F110010DF5047A0FC98AE80F00D4E982
:106280000801A26A8A92CDE9880184988DF820924B
:106290008DF82182401C8DF822728DF81C528DF8E9
:1062A00023628490002D14BF8698859800F1010028
:1062B00014BF8690859080AB82980021CDF80CC2E7
:1062C0002C2894BF02462C220020B0EB920F06D25D
:1062D00053F820C0401C6144B0EB920FF8D3484201
:1062E0008390FF224FF4007168461BF058FA80AC8F
:1062F00094E80F008DE80F0084AC94E80F0004AC24
:1063000084E80F00DDE988018A9A4FF47B34CDE9F7
:1063100008010A922046FDF723FE69462046FDF754
:10632000C1FE012818BF00200DF50C7DBDE8F087E7
:106330002DE9F041ADF50C7D0F46804616464FF431
:10634000007168461BF00DFA002580954FF47B34F0
:106350008195829583958495859586958795889571
:1063600089958A9556492068884218D16068B0F5A9
:10637000807F14D9A06821464FF0000C2C2888BFDC
:106380002C200023B3EB900F11D251F823205B1C7B
:106390009444B3EB900FF8D3BCF1000F07D0FFF794
:1063A000ECFE002804BF0DF50C7DBDE8F0810FCC9C
:1063B0000DF5007C8CE80F000FCC0DF5047C8CE80B
:1063C0000F00D4E90001A2688A92CDE988018DF816
:1063D00024828DF825728DF8266201208DF827021F
:1063E0008298002180AB83952C2894BF02462C22F2
:1063F0000020B0EB920F06D253F820C0401C61443D
:10640000B0EB920FF8D348428390FF224FF4007113
:1064100068461BF0C4F980AC94E80F008DE80F00CB
:1064200084AC94E80F0004AC84E80F00DDE9880137
:106430008A9A4FF47B34CDE908010A922046FDF791
:106440008FFD69462046FDF72DFE012818BF00206C
:106450000DF50C7DBDE8F0812DE9F04F194D4FF0A1
:10646000000885B06C42474646461720FFF729FED4
:106470004FF47B32844612491068884217D1506825
:10648000B0F5807F13D9936800212C2B88BF2C2373
:106490000020B0EB930F80F0F98052F82090401C60
:1064A0004944B0EB930FF8D3002900F0EF80FFF7D9
:1064B00064FE002804BF05B0BDE8F08F142003E09F
:1064C0004353494DF1D8FFFFFFF7FBFD0290152024
:1064D000FFF7F7FD00901620FFF7F3FD40B20190A3
:1064E0001620FFF7EEFD404240B20390FCF7FAFCA5
:1064F000DFF8A8914FF0000B824689F803B089F8C5
:1065000004B089F805B00CF074FEF9F76CFF0020B8
:1065100089F80000C9F818B0FFF742F81AF0F00F38
:1065200005D01BF041F9012808BF48F001081AF016
:10653000070F7DD05A485C4A002690F800E0594881
:10654000037899F80200A3EB000984468145C4BF93
:10655000AEEB0C01A1F1010B1CDD61468B4516DD94
:1065600001F1010A01FB03070AFB030A32F8177065
:1065700032F81AA0A7EB0A073FB2002FB8BF7F423C
:106580003FB2B742C8BFBEB2491C8B45E8DC401CD5
:106590008145E2DC0098002818BF864288BF48F099
:1065A00002080027E246AEEB0A0000905045C8BF43
:1065B000A9F1010B1BDD6046834513DD0AFB0301D6
:1065C00032F811E002EB41014988AEEB010109B25A
:1065D0000029B8BF494209B2B942C8BF8FB2401CB6
:1065E0008345EBDC00980AF1010A5045E3DC029890
:1065F000002818BF874288BF48F00408E246009888
:10660000504514DD614689450CDD0AFB031032F963
:106610001000A842C8BF0546A042B8BF0446491CA6
:106620008945F2DC00980AF1010A5045EADC00E0F5
:1066300009E00198002806DD854202DC03988442C7
:1066400001DA48F00808FF2F88BFFF27FF2E88BF18
:10665000FF267F2DC8BF7F2504DC15F1800FB8BF52
:106660006FF07F057F2CC8BF7F2404DC14F1800FFE
:10667000B8BF6FF07F04E0B20090EBB2F2B2F9B2B3
:106680004046FFF7B9FD05B0BDE8F08FBCF1000F43
:1066900018BFBCF1010F3FF411AF08E7FC840010F4
:1066A00065850010648500105C270110FE490020FC
:1066B0008862704740B2FC4910F1050FBCBF002250
:1066C0008A6288707047F84890F902007047F6486F
:1066D00000787047F44840787047F3480021C17152
:1066E00041718172C172017341727047EE4920F0AD
:1066F0007E4008627047EC48006A7047EA48408A6A
:106700007047E948808A7047E748B0F9160070473B
:10671000E548B0F918007047E348B0F91A0070472F
:10672000E148407B7047E048C078002818BF01204E
:10673000704710B54FF4E461DC481BF012F8DA49F9
:106740000020C87010BD30F911C000EB4100B0F955
:106750000210BCEB010048BFA1EB0C0000B2142AF0
:1067600005D0B3F900108142B8BF18807047A0F17E
:1067700014010029CCBF1438002000B2F1E72DE944
:10678000F74F90B00025CA480095019502950395F2
:1067900004950595069507950895006817460C46DB
:1067A000052A08BFB0F97A600AD0062F08BFB0F9F1
:1067B000786005D00A2F0CBF1E26B0F9766010D085
:1067C000B0F97400DFF8E882B0420ADA15F0CFF8C9
:1067D00048F2021108421CBFD8F80000B0F87460FB
:1067E00036B23246694610981AF0E3FF049800B2B8
:1067F0002080BDF822106182BDF81A106181BDF8B9
:106800001C10A181BDF81E10E181BDF8201021826D
:10681000BDF81410A180BDF81610E180BDF8181065
:1068200021810028B8BF25800021A2488DF82410BE
:10683000A14A00788DF826008DF8251012788DF881
:1068400027207242DDF82480ADF82A20ADF82860B8
:10685000ADF82C00C8F307261098DDF82CB04FEAED
:1068600018690D90ADF83010B246B1452FD908F037
:10687000FF051FFA8BF00F9006FB005081B20E90BF
:106880000CAB2A460D98FFF75EFF0E986A1C401C61
:1068900081B20CAB0D98FFF756FF0F98C8F3074570
:1068A00006FB00500E90C01E81B2E81E82B20CABF7
:1068B0000D98FFF748FF0E980CAB801E81B2A81E02
:1068C00082B20D98FFF73FFF761CB145CFD808F094
:1068D000FF05C8F30740A0F10108A8452AD91FFA0F
:1068E0008BF60AFB065081B2AAB20CAB0D98FFF7EB
:1068F0002AFF0AF1010000FB065081B2AAB20CABDC
:106900000D98FFF720FFA9F1020000FB065081B2AD
:10691000AAB20CAB0D98FFF716FFA9F1010000FB1E
:10692000065081B2AAB20CAB0D98FFF70CFF6D1C9C
:10693000A845D4D8BDF830106180052F09D04FF09C
:106940000000E082A082012F208300F0718100F01E
:10695000D9B9FEF7A5FD00211AF030FF002800F09C
:106960000781DDE909300022ADF83020ADF8342090
:10697000C3F30722DDF82CA010991E0E9146964213
:1069800071D91FFA8AFCDDB202FB0C5E1FFA8EF889
:10699000CDF838C031F91880BDF83050BDF834C09A
:1069A0000FFA80FBD845C4BF6D1CADB24FEA204B37
:1069B000D845BCBF0CF1010C1FFA8CFCADF830506F
:1069C0000EF101081FFA88F8ADF834C031F91880CB
:1069D0000FFA80FBD845C4BF6D1CADB24FEA204B07
:1069E000D845BCBF0CF1010C1FFA8CFCADF830503F
:1069F000DDF83880C3F3074B02FB08BEAEF1020896
:106A00001FFA88F8ADF834C031F918800FFA80FB0E
:106A1000D845C4BF6D1CADB24FEA204BD845BCBFB2
:106A20000CF1010C1FFA8CFCADF83050AEF10108EE
:106A30001FFA88F8ADF834C031F918800FFA80FBDE
:106A4000D845C4BF6D1CADB24FEA204BD845BCBF82
:106A50000CF1010C1FFA8CFCADF83050521CADF853
:106A600034C096428DD8DAB2C3F3074E964579D931
:106A70001FFA8AF509FB05231FFA83F8BDF83030A9
:106A800031F91880BDF834C00FFA80FBD845C4BF77
:106A90005B1C9BB24FEA204BD845BCBF0CF1010CEC
:106AA0001FFA8CFC0AE000001C85001014A30010E3
:106AB00074870010648500106585001009F10108D5
:106AC00008FB05281FFA88F8ADF83030ADF834C05F
:106AD00031F918800FFA80FBD845C4BF5B1C9BB20C
:106AE0004FEA204BD845BCBF0CF1010C1FFA8CFCBF
:106AF000ADF83030A6F1020808FB05281FFA88F827
:106B0000ADF834C031F918800FFA80FBD845C4BF06
:106B10005B1C9BB24FEA204BD845BCBF0CF1010C6B
:106B20001FFA8CFCADF83030A6F1010808FB0525F2
:106B3000ADB2ADF834C031F915500FFA80F84545C3
:106B4000C4BF5B1C9BB24FEA20484545BCBF0CF15B
:106B5000010C1FFA8CFCADF83030521CADF834C07B
:106B6000964585D8BDF83400E082BDF83010A1828A
:106B70000025DDF82CA0DDF82480109E052F44D0E0
:106B8000FE48062F006803BFB0F8781002221046B6
:106B9000B0F876101CBF01220020B4F902C0B4F98D
:106BA00000309C4541D18B423FDDC8F307210144B1
:106BB000C0EB186E8E4526D9C8F3074308F0FF00D6
:106BC0009B1A1044A3F10109814519D91FFA8AF3D0
:106BD00001FB03039BB236F913C006EB4303B3F981
:106BE0000230BCEB030B48BFA3EB0C0B0FFA8BF38B
:106BF000142811D0AB42C8BF1D46401C8145E5D8C2
:106C0000491C8E45D8D8258310E0DC480222006854
:106C1000B0F87A101046C0E7A3F1140CBCF1000FD5
:106C2000CCBF143B00231BB2E4E72383012F69D1BF
:106C3000D3484FF0000AB4F900900778D148109D6E
:106C400090F8008014F093FE10F4807F04D0222688
:106C50004FF0010C002307E010F4004F4FF0000C40
:106C600004D02426002305270A2005E0C348464611
:106C700000230068B0F98000814543DB1846002FEF
:106C800088BFB4F900903DD900FB08F1153135F902
:106C9000112005EB410131F9021CB2EB010B48BF99
:106CA000A1EB020B0FFA8BF1894505D0401CB842CD
:106CB000EAD3BAF1000F25D000202080BB4238BFB4
:106CC000721E1FD26046B44519D203FB08019042E0
:106CD00012D235F9119005EB4101B1F902A0B9EBDF
:106CE0000A0148BFAAEB090109B2142819D0B4F966
:106CF00000908945B8BF2180401CB042E5D35B1CA1
:106D0000BB42DFD3A088002804BF4FF40040A0801E
:106D10006089002804BF47F6FF70608113B0BDE8AA
:106D2000F08FA1F11409B9F1000FCCBF1439002183
:106D300009B2DCE7084318BF70479348016A11F0B5
:106D4000807F08BF70478D490968096F11F4003FC3
:106D500008BF7047002111701821018270478A48CE
:106D6000006B70472DE9FF5F86480027DDF83CA0E7
:106D700005780E98119E8B46B9463C4650452CD05E
:106D800006FB050E10983BF91EC006FB05093BF9F2
:106D90001900BCEB000148BFA0EB0C0106FB05A8E5
:106DA0003BF91840B4EB000C48BFA0EB040C01EB1E
:106DB0000C0004B232F91EC032F91900BCEB00011C
:106DC00048BFA0EB0C0132F918C0BCEB000248BF71
:106DD000A0EB0C0288180FFA80F96B48006B0128B1
:106DE00018BF012B37D04FF001081AF0ECFC6749AF
:106DF000002C0A7807DD109906FB05113BF91110EC
:106E00001431282909D80099B1F914103C2904DC5F
:106E10000099B1F916103C2926DD0E9902EB0A0CF7
:106E200011448C4520D9129B139D13442A448B4254
:106E30001CBF8D1A15F1020F30F9115000EB4106FD
:106E4000B6F90260A5EB060508D01E353C2D08D921
:106E50004FF0000808E0A1450CDD0AE00A35142DCA
:106E6000F6D8491C8C45E2D8A14503DDB8F1000FE6
:106E700000D0012704B03846BDE8F09F7047424873
:106E8000B0F90E00704740490020C88170470021CA
:106E9000018041804FF400428280C1800181521EF6
:106EA00042818181C181018241828182C1820183CB
:106EB00070473548C06A7047002818BF0120324922
:106EC000C862704700223049022802D080208A62BE
:106ED00088708A62704770B52B4E04460D46306B41
:106EE000844206D044EA052200236B2107200BF0E0
:106EF00033F934B90020022D02D08021B062B17084
:106F0000B062346370BD2DE9F0418846054614F047
:106F100016FD044614F00FFD04FB00F11A4E221872
:106F2000002496F9020009B210F1800F274618BF1D
:106F300010F1050F1BDAB6F91A006439814211DA33
:106F40000124B8F1000F12D10021002A0FD935F920
:106F50001100B0F5487F01DA002403E0491C91429A
:106F6000F5D324B911F0E1FC012808BF0124306BEE
:106F7000012808BF002C22D10AE00000748700100D
:106F800065850010648500101C8500106A8500105E
:106F9000B06A4EF6C42188420BD200F07FFC00217B
:106FA000022819D0042808BF4FF4FA71B06A0844C7
:106FB000B0624EF66021814228BF012400D2B76240
:106FC000306B844206D044F4807200236B2107208A
:106FD0000BF0C2F854B906E00CF008F9002814BF11
:106FE00011210821E2E78020B762B0703463BDE868
:106FF000F081002818BF0120FE4948637047FD4812
:10700000406B7047FB4988837047FA48808B704714
:10701000F848406A7047F7494862F9F704BAF549F9
:10702000886370472DE9F04FF34987B002240A784E
:10703000F249A2F1020C521E91F800800021009149
:10704000A8F10101CDE9011C00212546A8F10209A2
:107050000B46BCF1020F84BFA9F1010CCDF80CC0A6
:107060005FD94FF0000CCDF814C0CDF810C0AC467D
:107070004D4551D2039F04FB08C6BC450FD230F9E1
:10708000167000EB4606B6F90260B7EB060E48BF75
:10709000A6EB070EBEF1320F01D9E34608E00CF172
:1070A000010CE145E6D8DDF814C0BCF1000F1BD09F
:1070B000A9F1010CAC4517D304FB08C665450FD2F6
:1070C00030F9167000EB460636F9026CB7EB060E87
:1070D00048BFA6EB070EBEF1320F01D9E24608E029
:1070E000ACF1010CAC45E7D2DDF810C0BCF1000FEB
:1070F00012D04FF0010CCDF800C0DDF804C0DC4523
:1071000088BFCDF804B0514538BF5146A24288BF70
:107110002246A34238BF2346641CDDF808C06445FC
:107120009FD3B448DDF800C0846B644518BFC0F835
:1071300038C0019807B0BDE8F04F15F081BB2DE9CC
:10714000FF4F8BB0AB4DDDE918A704460020287037
:1071500068700CF05FF8002840F03A8100F098FB6E
:10716000052871D0687B0190A649A548DDF83090CC
:1071700091F800B00068A44990F886600978009101
:10718000B0F98480B5F918003228688A05DA002839
:1071900004BF7006060E04D100E010B9287901285A
:1071A0002BD10CF079F840BB012F26D0BAF1010F9A
:1071B00002D1A88AC82820D8A88A002804BF688AD3
:1071C00000281AD00CF012F8012819D0B9F80000E4
:1071D000E881009900201BEB01030AD039F9101057
:1071E000B5F90E209142C8BFE981401C80B28342AC
:1071F000F4D8B5F90E0040450EDD0020E87223E01A
:107200007F48006890F887600198012814BF4FF00C
:107210003C084FF04108D9E7286A10F4803F13D0AA
:1072200077480068006F10F4803F0DD0E87A401C6A
:10723000C0B2E872B04207D910202882012028721B
:1072400000204FF0FF34E87211F06FFBA8B100F09E
:1072500025FB042811D195F8200010F0800F0CD0E8
:107260006748006890F8700010F0800F05D0072084
:10727000288201204FF0FF3428720BF0B7FF01285D
:1072800071D15F48BAF1000F00680A9090F8881039
:107290006BDC012F69D0286A10F4003F12D00A98E5
:1072A000006F10F4003F0DD0A87A401CC0B2A87245
:1072B000884207D9112028820120287200204FF02F
:1072C000FF34A8720C9800904E484FF0000B012F2D
:1072D000007803904C48007801900A9890F8870055
:1072E000069045D0019840080790039840080990FF
:1072F0000020049082460590DDE9001001EB40007B
:10730000029000231A461946BAF1000F0CBFDDE9BE
:107310000076DDE902760020002E88BFA6F1010E7E
:1073200029D937F91080B8F1640FD8BF002214DDD5
:1073300070450DD207EB400CBCF902C0B8EB0C094C
:1073400048BFACEB08090FFA89FCDC45A8BFE3464F
:10735000491C002A04BF01225B1C401C8642E0D865
:10736000012B05D807E033E0FFE70020A872A9E76A
:10737000002028732CE0BAF1000F0CBF0491059196
:107380000AF1010ABAF1020FBBD3079904988842A7
:10739000EED9099905988842EAD9BBF1320FE7DCAA
:1073A000287B401CC0B22873296A11F4801F0FD0BB
:1073B0000A99096F11F4801F1CBF0699884207D9EA
:1073C000142028820120287200204FF0FF342873F7
:1073D00014F0CDFA10F4014F35D000F059FA02281C
:1073E00031D14FF001081AF0F3F9074614F0A7FA6B
:1073F00006460BE01C8500106585001064850010B2
:1074000074870010698500106A85001014F093FAE3
:10741000024600210020002E08D900FB021337F994
:1074200013300F2B0FDB401CB042F6D3B8F1000F26
:1074300009D0491C0129EDD9B8F1000F03D0012072
:107440004FF0FF3428720FF026FA032823D10020D2
:1074500000900190287C8DF80000BDF80000022209
:1074600064F30F20ADF80000E979BDF8020061F384
:107470000300697961F30710297A61F30820A9797B
:1074800061F34920ADF80200E889ADF80400062157
:1074900068460FF003FAB4F1FF3F26D0002C07BF77
:1074A000A87901280FB0BDE8F08FFEF7F1FB0024AA
:1074B000AC71012028704FF4E461E3481AF051F9EF
:1074C000EC7000F0EBF904280D982CD0002818BFC0
:1074D000FEF714F80E98002804BF0FB0BDE8F08F37
:1074E0000FB0BDE8F04FFDF7BABF287A01281CBFE6
:1074F0000FB0BDE8F08F0D98FEF7D3FB00242C727F
:10750000012068704FF4E461CF481AF02AF9EC705A
:107510000D98002818BFFDF7F1FF0E980028DFD165
:107520000FB0BDE8F08F002818BFFDF7BBFF0E9825
:10753000002804BF0FB0BDE8F08F0FB0BDE8F04FDA
:107540001AF04BB92DE9FF4FDFF800A3044689B0CC
:10755000DAF800001D461646B0F878B013F0F9FCD2
:10756000012804BF4FF6FF7000EA4B0B14F0FFF93F
:1075700048F20217384207D0B5F91410012320460B
:10758000169A1AF02FF904E0012220461699FFF707
:10759000F6F8DFF8BC820024254688F80440DDF8C0
:1075A0002890FDF77DFF00940194029403940494C5
:1075B0000594069407940894A44C69462068B0F892
:1075C000762048461AF0F5F82168BDF91A00B1F99D
:1075D000761049428842B8BF0125BDF82000B0F5B9
:1075E000E17F88BF01259A48057114F0C0F948F27F
:1075F000021108420DD11698B0F91200002808DCDB
:107600000BF0F4FD012804D091480079012840F0E6
:10761000E38014F0ACF948F2021810EA080F00F009
:10762000D38047F6FF7001908A484FF000094D461D
:1076300090F800A08848179C077814F098F9414604
:1076400008420FBF584681480068B0F874000FFA2E
:1076500080F814F08CF948F2021108421FBF7B48F1
:107660000068B0F87400404208BFCBF1000000B2DF
:10767000029014F07CF910F4807F06D000204FF0C7
:10768000010B4FF0220C00900EE010F4004F4FF071
:10769000000B06D000204FF0240C4FF0050A00909C
:1076A00002E00020BC4600900198804571DA009A03
:1076B000BAF1000F63D9ACF101000590AAF1010005
:1076C0000490ACF1020003905846E3453CBF11B270
:1076D000019151D202FB070399B236F9111000292A
:1076E000B4BFC1F1000E8E46C6451CDD41450CDD20
:1076F000B4F904E0714503DDA180E08001992181A6
:1077000009F101010FFA81F90DE0DDF808E08E457D
:1077100009DDB4F90AE08E4503DD6181A08101999C
:10772000E181691C0DB20599884222D236F913E035
:1077300006EB4303B3F90230BEEB030148BFA3EBF2
:107740000E0109B214281BD0009B9A421CBF049B57
:107750009A4204D058451CBF039B984204D1B4F907
:1077600002308B42B8BF6180B4F900308B42B8BFA1
:107770002180401C6045ADD3521C5245A4D31FE06C
:10778000A1F11403002BCCBF1439002109B2DBE7AF
:10779000FFE70098BAF1000F12D95B46E3450CD21F
:1077A00000FB073189B236F9112002998A42BCBF29
:1077B000691C0DB25B1C6345F2D3401C5045ECD3F1
:1077C000A4F81090658204E0062230461799FEF76F
:1077D000D6FF1999012008701798B0F910000028F9
:1077E00008DC1798B0F91200002803DC184800796B
:1077F000012815D114F0BBF848F20211084207D055
:10780000052347F6FF71189A0A9819F0EBFF04E078
:10781000052218990A98FEF7B2FF1A9901200870FC
:107820001698418A0A4841821699098A81821699D6
:107830004989C1821699898801831899098A4183E7
:107840000DB0BDE8F08F000014A300107487001085
:107850001C850010658500106485001010B50BF0C4
:10786000C1FA0BF0A3FB002010BD0000FE49C87058
:107870007047FD48C0787047FB4908717047FA4867
:1078800000797047401E022894BF012000207047F5
:10789000F54800787047F44880787047F2480078DF
:1078A000022805D005281CBF0020704706F0BBBD8C
:1078B0000BF07FBCEC4908707047EB49487070478B
:1078C000E9484078704770B5E74E044682B030789A
:1078D0000D46A0421ED00022612100928DF80010BA
:1078E0008DF801408DF8025001928DF803000228B6
:1078F0001FD0052814BF002006F095FD8DF8040068
:1079000014F0B5F88DF805000722002369461046EB
:107910000AF0AFFC3078844218BF7070B570072C45
:1079200024BF02B070BDDFE804F016070B13160F7A
:1079300016000BF03EFCE1E7284600F01DFB0AE0D4
:1079400028460BF0E1FC06E0284606F05DFD02E06B
:1079500028460AF0F3FC347002B070BDC349002021
:107960000968B1F8B01011F4807F08BF7047FCF7C8
:1079700012BABE4900200968B1F8B01011F4807F36
:1079800008BF7047FCF716BAB84900200968B1F87B
:10799000B01011F4007F08BF704719F028BFB2493A
:1079A000487900281CBF401E4871704770B5B04828
:1079B0000068AD4C10F0130F0FD010F0100F05D071
:1079C000AC4951F88C2F42F480520A60AA490860F1
:1079D0006079002804BF012060714FF04020806969
:1079E000A24D10F0020F296806D1A448006810F0DB
:1079F000010F01D0607940B1B1F8B010002011F44E
:107A0000807F18BFFCF7D6F907E0B1F8B01000206E
:107A100011F4806F18BF19F0EFFE9949084208BFB2
:107A200070BD2968D1F8B010090C617170BD10B536
:107A300072B6FDF79DFCBDE81040FDF7ADB810B57E
:107A4000012802D0022805D007E04FF47F30FCF770
:107A500087FA02E08C498B48086072B6FDF788FC13
:107A6000BDE81040FDF798B87F4900288A7918BF13
:107A700001208871C0B2824208BF704700220028EE
:107A800018BF01220023012102200AF065BB7648BD
:107A90008079002818BF01207047734AD17981424C
:107AA00008BF704710720120507270476E48007A0C
:107AB00070476D49487270476B48407A704770B59F
:107AC000694C0028E57918BF0120E071C0B2F8F7D1
:107AD00069FCE079854214BF002870BD247819F054
:107AE00090FE022C1CBF052C70BD02212046BDE873
:107AF0007040E8E610B513F03AFF48F20211084270
:107B00001CBF002010BD5848C079002818BF0120B4
:107B100010BD0028544918BF01208872704710B565
:107B200013F025FF48F2021108421CBF002010BDCF
:107B30004D48807A002818BF012010BD4A48C07AFD
:107B400070472DE9F041484D00281CBF0020E87225
:107B500004D1E87A002818BFBDE8F0814B4E3768A1
:107B60003020FCF77FFB06213020FCF794FBF06A05
:107B700040F03000F062464C4FF07F0811E0FDF716
:107B80000EFCF06A10F0100F03D0E87A40F07E008F
:107B9000E872F06A10F0200F03D0E87A40F001009C
:107BA000E872201EA4F1010403DDE87A38EA00003F
:107BB000E5D13020FCF79CFB3760BDE8F0812A4816
:107BC000C069704728488069704727488069002845
:107BD00018BFC07A70472449086270472248006A7B
:107BE00070472149486270471F48406A70471F48E4
:107BF000026802F5C873118A508A02F5A872FBF771
:107C0000AEBA10B507F001FA002818BFC07A10BD4F
:107C100010B507F0FAF900280CBF4FF0FF3090F9CB
:107C2000240010BD2DE9F04FDFF83CA099B00E46BE
:107C3000CAF81C0007F0E9F9CAF81800002800F09B
:107C4000DD8090F800C08AF80CC041788AF80D10E9
:107C5000837804460CF101008AF80E3000F0FE0033
:107C60008AF80F00E27815E058850010748700103C
:107C7000184800400030004014480040144C0040B8
:107C800008001300AD2007B0304C00400010004049
:107C9000803801008AF8102020798AF81100607974
:107CA0008AF812000AF114004FF0000B80F800B0BF
:107CB00080F801B020788AF813006046FBF70DFCCD
:107CC0009AF812109AF81100FBF72AFC6946204630
:107CD00007F0B9F9E089DAF8205000281CBF6843A2
:107CE000050BB4F81280DAF82490B8F1000F08BF41
:107CF0004FF48058E78A002F08BF4FF480574FF4A5
:107D000080501890002016F0040F18BF052016F0C0
:107D1000080F18BF40F0020016F0020F18BF40F025
:107D2000F00016F0010F18BF40F4774016F4807F82
:107D300018BF40F4803016F4007F18BF40F47E0076
:107D4000E16901EA000600981090059812900798E2
:107D5000CDF844B0CDE9130B01981590A07A179097
:107D60000398169010A93046FAF7AAFF16F0070FED
:107D700074D00020F8F7A8FE9AF8101088421AD0A4
:107D80000020F8F796FE9AF8100000EB400101EB96
:107D90000010754901EB80004C2119F0E2FC9AF8C3
:107DA000100000EB400101EB0010704901EB800076
:107DB0004C2119F0D6FC06F006FE18B10146002051
:107DC000F9F7E7FC06F016FE6843050B06F032FEF5
:107DD00009FB00F0000B4030C1090A20012202FA21
:107DE00000F30B4201D1401EF9D5A0F10509207B1B
:107DF000002818BFA0F1010B11D10CE05C4800680D
:107E0000B0F8B00010F4807F18BFFBF7D3FF00205C
:107E100019B0BDE8F08F0020F9F7DDFE8346607BE6
:107E2000002814BF401EF9F70EFF0BEB09010529CE
:107E300005DDA9EB010101F10509052104E0002997
:107E4000BCBFA9EB010900218144B9F1050F06DD92
:107E5000A9F10500C5404FF0050908E00EE0B9F1B1
:107E6000000F04DAC9F1000085404FF0000900203E
:107E7000F9F7CBFE49460020F9F7FFFE16F0F00FA8
:107E800043D0207C70B116F0100F03D0411E0120AA
:107E9000F9F7BBFE16F0400F04D0207C411E0220F3
:107EA000F9F7B3FE207D70B116F0200F03D0411E0C
:107EB0001120F9F7AAFE16F0800F04D0207D411E94
:107EC0001220F9F7A2FE607C70B116F0100F03D0FB
:107ED000411E0120F9F7D1FE16F0400F04D0607C5E
:107EE000411E0220F9F7C9FE607D70B116F0200F27
:107EF00003D0411E1120F9F7C0FE16F0800F04D008
:107F0000607D411E1220F9F7B8FEE07A00281CBF00
:107F10000001F9F776FB029806F031FD049830B1C4
:107F20002B469AF80D209AF80C1019F06FFC3A467F
:107F300041462846189B19F06EFC0698FDF723FF72
:107F40000898FDF759FF0BF0BDFA19B00120BDE804
:107F5000F08F10B5FAF789FF06F019FD05490020EA
:107F60008861012010BD0000000001300040013098
:107F70007487001058850010FE4908707047FD484E
:107F800000787047FC4810B4FC4A016891421CD14B
:107F90004168B1F5987F18D8D0F808C00146BCF503
:107FA000007F12D800220B461146B2EB9C0F24BF73
:107FB00010BC704753F82140491C2244B1EB9C0F80
:107FC000F8D3002A04BF10BC7047002010BC7047D3
:107FD000E948FBF7C5BFE7490120087070472DE964
:107FE000F04117460E4605461024FFF7EBFD15F04D
:107FF000070F18BF062403D115F0F00F18BF08248F
:108000003246102C28BFBDE8F081002A08BFBDE829
:10801000F08120443B4690F920102046BDE8F04115
:1080200007F039B82DE9F04FADF6446D0C46074620
:10803000FFF7C8FD064617F0070F00F00381E94679
:108040004FF005084846FBF7D1FA751D96F9251043
:108050004FF464634A46404607F01DF895F8200047
:1080600000286ED1FFF70BFCFFF70CFC012868D14C
:10807000C34890F800B0C34890F800A0512005F024
:108080008BFA0021CDF8400E084605F013FA05469C
:108090000121002005F00EFA8146BB4800785128E6
:1080A00004BF002005F06BFB4FF000435A1E002078
:1080B0000BFB0AFABAF1000F0AD935F810109942F1
:1080C000C8BF0B469142B8BF0A46401C8245F4D84F
:1080D000981800EBD070421001234046AB4963F37F
:1080E000070063F30F20C9F8001062F31F4000215E
:1080F000C9F8040009F10803BAF1000F12D935F8E4
:108100001100801A00EBD07040107F28C8BF7F207C
:1081100004DC10F1800FB8BF6FF07F005854491C89
:108120008A45ECD8FFF7ABFB4FF4443101EB8020DC
:108130000AF108024946FCF709F8DDF8400E05F09F
:108140002BFA06EB080090F8200003287AD18C481F
:1081500005788C4890F80080512005F01DFA824681
:108160000021084605F0A6F9814687480078512885
:1081700004BF002005F003FB0020854A530C04EBEC
:108180008001401CCA87A1F840300428F7D300239F
:10819000B8F1000F25D90020002D88BF03F0070C8F
:1081A0001CD9BCF1040F28BF022204D2002816BF3C
:1081B00023280322012203FB050104EB820239F983
:1081C0001110B2F93AB08B45B8BF5187B2F93CB043
:1081D0008B45C8BF9187401CA842E2D35B1C434536
:1081E000D9D36C4A002084F83C0002F1080B4FF010
:1081F000010C04EB800132F910E0B1F93E30734517
:1082000007DB94F83C300CFA00FE43EA0E0384F8D6
:108210003C30B1F940103BF91030994206DC94F83B
:108220003C100CFA00F3194384F83C10401C04285D
:10823000DFD305FB08F04100484619F0F1FA50463B
:1082400005F0AAF917F0F00F04BF0DF6446DBDE874
:10825000F08F07246D46FAF745FE10F0300F0CBF83
:10826000022001206946FBF711FA96F927104FF416
:1082700018732A46204606F00EFF0DF6446DBDE841
:10828000F08F2DE9F34F89B0002006900878039015
:1082900048680490886805900D7B487B0190887B36
:1082A0008A8AD1E9088BC0F5807602EA000709982E
:1082B000B1F91090B1F912A0896910F0010F07917E
:1082C0004FF0000044D000900198002840F2EB806D
:1082D0000098012101FA00F20798104018BF012010
:1082E00000240290610904A804F01F0250F8211034
:1082F00001209040014200F0CB803BF9020B029933
:10830000A0EB0A0000290CBFA9EB000509EB000552
:1083100038F9020BA0EB0A0014BF4844A9EB000097
:10832000002DB4BF694229460028B8BF40428842A8
:1083300070D9224600990398FAF743FA0246C0F32F
:108340000420D1B212F4803F7ED0002D7DDB84E08A
:10835000F9F79DFD009001980321684301EB40006F
:1083600020F003024146584619F005FA0098F9F743
:108370008EFD11E08085001000EE0300544352464C
:108380006485001065850010F985001046544F463D
:108390000080FFFF9885001001984FF0000B002827
:1083A00056D90121079801FA0BF2104018BF01209D
:1083B00000250290690904A805F01F0250F8211059
:1083C00001209040014238D038F9020B0299A0EB0D
:1083D0000A0000290CBFA9EB000409EB00042A469F
:1083E00059460398FAF7EDF9C0F30421C2B210F42C
:1083F000803F02D0002C02DB03E0002C01DD941B47
:1084000000E09419BC4206DD1F293ABF0024491C34
:108410003C4607E03CE0002C04DA0029C6BF3C469D
:10842000491E002400F4783040EA012040EA0403A9
:108430002A4659460398FAF717FA6D1C262DB9D328
:108440000BF1010B019801E003E004E08345A8D3A0
:1084500029E0002D01DD8D1900E08D1BBD4205DDF9
:108460001F283ABF0025401C3D4606E0002D04DAD7
:108470000028C6BF3D46401E002502F4783141EA7F
:10848000002040EA0503224600990398FAF7ECF928
:10849000641C262CFFF426AF00980199401C009024
:1084A0008842FFF415AF0998032826BF01200690E3
:1084B00006980BB0BDE8F08F2DE9F04F8BB000228D
:1084C00005920A7800924A6802928A6803924D7B6C
:1084D0008A7B0492B1F91080B1F9122007920C6ADC
:1084E0008A690892898A049AC0F1080A01EA020698
:1084F00000283BD0BAF1000F7ADB4FF0000B002DC3
:1085000077D9012000FA0AF00690AAF101000121B2
:1085100001FA00F009900121089801FA0BF21040CD
:1085200018BF012000270190790902A807F01F0257
:1085300050F821100120904001427DD034F9021BF7
:108540000798081A019900290CBFA8EB000908EB4D
:1085500000093A4659460098FAF733F9034610F4F1
:10856000803F72D0B9F1000F74DA71E04FF0000B68
:10857000002D3ED90121089801FA0BF2104018BFD6
:10858000012000270190790902A807F01F0250F886
:1085900021100120904001424BD034F9021B079872
:1085A000081A019900290CBFA8EB000908EB000983
:1085B0003A4659460098FAF704F9FE49014011F489
:1085C000803F17D0B9F1000F29DA11F4F8511CBF20
:1085D000A1F5807141F4803121D110F4604F1ED09B
:1085E000A0F500504FF4D05110F4003F17D014E024
:1085F0004AE042E0B9F1000F11DD11F4F85118BF63
:10860000A1F580710BD110F4604F08D0A0F5005097
:108610004FF4D05110F4003F01D04FF48D3100F4ED
:108620003830084340F080033A4659460098FAF73C
:108630001BF97F1C262F02E016E006E00AE0A2D319
:108640000BF1010BAB4595D317E0B9F1000F01DD3C
:1086500006988343BAF1000FC4BF099803433A4612
:1086600059460098FAF700F97F1C262FFFF45CAFFB
:108670000BF1010BAB45FFF44EAFBAF1000FC2BFD7
:1086800005980BB0BDE8F08F0027002D2ED9049877
:108690000DF1080A4FF0010BC0F5807940F48078A5
:1086A0000024600904F01F015AF820000BFA01F1C0
:1086B000084215D0224639460098FAF782F8C1B22E
:1086C00001EB590101EA0801B14288BF314620F0AF
:1086D000FF0040EA0103224639460098FAF7C4F841
:1086E000641C262CDDD37F1CAF42D9D3012005901A
:1086F0000BB0BDE8F08F2DE9F04F89B00022049255
:108700000A7800924A6802928A6803924A7B019230
:10871000B1F91060B1F912B00C6A8969C0F10508AD
:108720000591002837D0B8F1000F70DB4FF0000939
:10873000002A6BD908F10800012101FA00FA401E55
:1087400001FA00F006900121059801FA09F21040A3
:1087500018BF012000250790690902A805F01F0233
:1087600050F821100120904001425FD034F9020BF3
:108770000799A0EB0B0000290CBF371A37182A46BF
:1087800049460098FAF71DF8034610F4803F3FD0A1
:10879000002F41DA3EE00027002A4FD90120059939
:1087A00000FA07F20A4214BF4FF0010A4FF0000A24
:1087B0000025690902A805F01F0250F821100120C8
:1087C000904001421BD034F9020BBAF1000FA0EB2C
:1087D0000B000CBFA6EB000906EB00092A46394640
:1087E0000098F9F7EEFFB9F1000FC8BF40F48030F0
:1087F00040F480532A4639460098FAF735F86D1C44
:10880000262DD6D301987F1C8742C7D316E01AE0E5
:10881000002F01DD23EA0A03B8F1000FC4BF069858
:1088200003432A4649460098FAF71EF86D1C262D88
:1088300092D3019809F10109814584D3B8F1000F61
:1088400004BF01200490049809B0BDE8F08F2DE921
:10885000F04F89B0002204920A7800924A6802928E
:108860008A6803924A7B0192B1F91060B1F912B0A3
:108870000C6A8969059150490969421AC2F10308D5
:10888000814277D83DD101984FF00007002871D977
:108890000120059900FA07F20A4214BF4FF0010ABD
:1088A0004FF0000A0025690902A805F01F0250F8E0
:1088B00021100120904001421BD034F9020BBAF183
:1088C000000FA0EB0B000CBFA6EB000906EB0009A4
:1088D0002A4639460098F9F774FFB9F1000FC8BF6E
:1088E00040F4003040F400432A4639460098F9F736
:1088F000BBFF6D1C262DD6D301987F1C8742C7D3A2
:108900004FE0B8F1000F51DB01984FF0000900284B
:1089100047D908F10D00012101FA00FA401E01FAC1
:1089200000F006900121059801FA09F2104018BFE5
:10893000012000250790690902A805F01F0250F8E0
:10894000211001209040014223D034F9020B0799F5
:10895000A0EB0B0000290CBF371A37182A464946EE
:108960000098F9F72EFF034610F4003F03D0002FC4
:1089700005DA02E015E0002F01DD23EA0A03B8F171
:10898000000FC4BF069803432A4649460098F9F7EA
:108990006BFF6D1C262DCED3019809F1010981458D
:1089A000C0D3B8F1000F04BF01200490049809B0AF
:1089B000BDE8F08F001F0100808500102DE9F14F08
:1089C000ADF54E7D0020C090BF9072B6FAF78AFADE
:1089D0000746FCF78BF948B1FCF730FAC090FCF77A
:1089E00017FAFCF730FABF90FCF71DFAFAF75CF9BA
:1089F000FAF762F8C590FAF79DFAC490FAF75EF8B4
:108A0000FAF71FFBBC900020FAF712FB0120F9F7E0
:108A1000DAF9C8901120F9F7D6F9C9900220F9F7D0
:108A2000D2F9CA901220F9F7CEF9CB90FBF7A7FF45
:108A3000C390FBF78CFF4FF49350FBF7FAFE62B63E
:108A40000020F9F791F9C29001210020F9F77FF990
:108A50000020F9F79EF90021C1900846F9F78CF93A
:108A60000120F9F714FACC900020FAF770F8C790BB
:108A70000020FAF75FF8C690F8F77EFDCD90002051
:108A8000F8F77FFD002006469EAD45F82060401CAB
:108A90000C28FAD317F0070F4FF001040AD040F664
:108AA0008C61FE489E9418F05CFE40F68C61FC4898
:108AB00018F057FE17F0F00F47D00120F8F735F8FF
:108AC00038B19821F74818F04CFE9821F64818F074
:108AD00048FE1120F8F729F838B19821F34818F02A
:108AE00040FE9821F24818F03CFE0220F8F71DF8ED
:108AF00038B19821EF4818F034FE9821EE4818F06C
:108B000030FE1220F8F711F838B19821EB4818F030
:108B100028FE9821EA4818F024FE0120F8F705F80D
:108B2000002818BFA0941120F7F7FFFF002818BFF6
:108B3000A1940220F7F7F9FF002818BFA294122091
:108B4000F7F7F3FF002818BFA3944FF0405ADFF85F
:108B500074B3DFF874939E984FF0FF0858B3304613
:108B60008DF8006001A9F8F794FF9DF80000F8F770
:108B7000B0FF8DF80C009DF80000F7F7A5FF8DF809
:108B80000D009DF80000F9F768F900280CBF4FF0C0
:108B9000FF31002106918DF80E80B9F80200ADF882
:108BA0001000ADF812609DF80000F8F712FFADF864
:108BB0001400CDE908AB9F986F4640B38DF828604C
:108BC00007F12C013046F8F764FF9DF82800F8F70C
:108BD00080FF8DF834008DF8354010968DF8368082
:108BE000B9F80200ADF83800ADF83A609DF82800F9
:108BF000F8F7EFFEADF83C009DF80C009DF80D1065
:108C000048430AEB40010BEB4000CDE91210A0985D
:108C10004FF4806A02264FF0AA3BE0B38DF8504033
:108C200007F154012046F8F734FF9DF85000F8F79B
:108C300050FF8DF85C009DF85000F8F7CCFF04FA67
:108C400000F08DF85D009DF85000F9F7BCF81A901F
:108C50008DF85E80B9F80400ADF86000ADF862A050
:108C60009DF85000F8F7B5FEADF8640097481C90E9
:108C700097481D909DF85D00022809D99DF85C1069
:108C8000801E48431C9901EB40001C908DF85D60EC
:108C90001A9800B100E007E09DF850004FF0AA31AB
:108CA000F9F77FF8CDF868B0A198E0B3112007F18B
:108CB0007C018DF87800F8F7ECFE9DF87800F8F765
:108CC00008FF8DF884009DF87800F8F784FF04FA17
:108CD00000F08DF885009DF87800F9F774F824907D
:108CE0008DF88680B9F80600ADF88800ADF88AA046
:108CF0009DF87800F8F76DFEADF88C007548269069
:108D0000754827909DF88500022809D99DF88410A0
:108D1000801E4843269901EB400026908DF885601F
:108D2000249800B100E007E09DF878004FF0AA31E8
:108D3000F9F737F8CDF890B0A298E0B307F1A401A5
:108D400030468DF8A060F8F7A4FE9DF8A000F8F773
:108D5000C0FE8DF8AC009DF8A000F8F73CFF04FAC7
:108D600000F08DF8AD009DF8A000F9F72CF82E90DA
:108D70008DF8AE80B9F80800ADF8B000ADF8B2A03B
:108D80009DF8A000F8F725FEADF8B40053483090E8
:108D9000534831909DF8AD00022809D99DF8AC10D8
:108DA000801E4843309901EB400030908DF8AD6053
:108DB0002E9800B100E007E09DF8A0004FF0AA3126
:108DC000F8F7EFFFCDF8B8B0A398E0B3122007F1A1
:108DD000CC018DF8C800F8F75CFE9DF8C800F8F7E4
:108DE00078FE8DF8D4009DF8C800F8F7F4FE04FA78
:108DF00000F08DF8D5009DF8C800F8F7E4FF389032
:108E00008DF8D680B9F80A00ADF8D800ADF8DAA030
:108E10009DF8C800F8F7DDFDADF8DC0031483A9068
:108E200031483B909DF8D500022809D99DF8D4100F
:108E3000801E48433A9901EB40003A908DF8D56086
:108E4000389800B100E007E09DF8C8004FF0AA3163
:108E5000F8F7A7FFCDF8E0B0F8F7C0F810F0010F71
:108E60000BD0FEF7B2FE3C2807D1FCF751F920B138
:108E70000420FCF7FCF8FCF7D3F9FAF798F84FF068
:108E80000008C346C2464646C14604F04CFA0128D3
:108E90007DD0BBF1800F7AD8AAA827E0000001306E
:108EA000004001308C0E01308C4E0130240F013017
:108EB000244F0130BC0F0130BC4F01305410013041
:108EC000545001300040003080850010CC09003043
:108ED000CC490030CC0E0030CC4E00304C18003065
:108EE0004C5800304C1D00304C5D0030FAF729FB27
:108EF00000286ED0AAA804F03EFFBC98002818BF36
:108F000000273BD09EA850F82700A0B307EB8701AD
:108F1000684600EBC104207810F00F0F2BD0F8F753
:108F200052FF10F0010F26D0216A257B01F00300CB
:108F300000EB8502D21C22F0030221F00301CDE9EF
:108F4000BD1278A90C1878A8BD9918F014FC00205F
:108F5000002D0BD9411934F8102034F8113024F8C1
:108F60001030401C24F811208542F3D878A9BE9A0D
:108F7000BD9818F000FC7F1C0C2FC3D31AF1010A16
:108F80007DD04FF0000A5046B0AD012700E077E0F9
:108F90000BF1010B45F82070401C0C28FAD3052E6C
:108FA0006ED2DFE806F003172A3D500000249EA889
:108FB00050F8240048B104EB8401684600EBC1017D
:108FC0004846FFF744FC45F82400641C0C2CEED303
:108FD0003BE068E000249EA850F8240048B104EB70
:108FE0008401684600EBC1014846FFF784FB45F861
:108FF0002400641C0C2CEED327E000249EA850F81B
:10900000240048B104EB8401684600EBC1014846E6
:10901000FFF752FA45F82400641C0C2CEED314E040
:1090200000249EA850F8240048B104EB840168464F
:1090300000EBC1014846FFF724F945F82400641C01
:109040000C2CEED301E04FF001080121002055F86F
:109050002020CAB1401C0C28F9D3A9B11F2E0DD273
:10906000761CCE9807FA06F1014207D1761C042E31
:1090700004D8CE9807FA06F10142F7D001E005E0E6
:1090800017E04FF0000901E009F10109FAF7AAFA27
:10909000B8F1000F0DD1BC98002818BFF8F7A5FE55
:1090A000F9F785FFF1E6FEF764FCB8F1000F3FF435
:1090B000ECAEFAF797FAF9F701FD0520FBF7D7FFB9
:1090C0000120C899F8F76DFE1120C999F8F769FEDB
:1090D0000220CA99F8F765FE1220CB99F8F761FED5
:1090E000BC98F9F7A5FF0020C199F8F745FE0020CC
:1090F000C299F8F72CFECC98F8F7C9FEC798F9F793
:1091000026FDC698F9F716FDCD98F8F73AFAC598F6
:1091100030B1C49810B1F9F74AFF01E0F9F710FF38
:10912000FBF7E4FD48B1C098002818BFFBF7E4FD49
:10913000BF98002818BFFBF718FEC398002818BF77
:10914000FBF7AEFBB8F1000F0CBF012000200DF5BE
:109150004F7DBDE8F08F70B5FE4D1646D5F844231F
:109160001205120D1DD000281CBFC1F30800FAF72C
:10917000B7FDD5F8480340F00100C5F84803D5F81D
:10918000480320F00100C5F848030022341E23DD07
:10919000D5F8481340F2D32011F0010F08D1401E3A
:1091A00001D2002070BDD5F8481311F0010FF6D0A0
:1091B000D5F84403C0F30B000244D5F8480340F04F
:1091C0000100C5F84803D5F8480320F00100C5F8B0
:1091D0004803641E002CDBDC1001B0FBF6F080B20B
:1091E00070BD2DE9F84F040016D0DB48006CC0F3C9
:1091F0000829FAF787FD49EA004200237621072073
:1092000008F0AAFFD348D0F8401341F48031C0F8E9
:109210004013322000900AE0FAF76FFD0120BDE80C
:10922000F88F00BF00BF00BF00BF00BF0846411E4F
:109230000091F6D24FF0000840F2FF17C2464646B2
:1092400008EB070000EBD0704510A9B264220120A2
:10925000FFF781FFF0B1A04288BF6F1E38BF05F154
:1092600001081ED1AA461FFA8AF14FF064024FF09E
:109270000100FFF770FF04460023524677210720C4
:1092800008F06AFFA4F5B0504B38A0289CBF01201D
:10929000BDE8F88FB9F1000F10D04846FAF720FD6D
:1092A0000EE0011B48BF211A321B48BFA21B91428E
:1092B000BCBFAA460646B845C2DDD4E7FAF71DFD95
:1092C00049F4803200237721072008F045FF002071
:1092D000BDE8F88F2DE9F04FA04CADF5157D0126C6
:1092E0002778FEF7D5FA012840F06B8104F029FFBA
:1092F0009B480068B0F91E10B0F91C0018F095FAF0
:1093000017F0020F00F0548180ADFEF73BFE4FF0E6
:10931000000828B101465022284618F01DFA21E025
:10932000FF225021284618F03AFA8E4880904FF4D8
:10933000987081905020CDE98208CDE984084FF0E3
:10934000FF308B908A90CDF818828990CDE9878084
:10935000ADF838828DF83A82CDF83082CDF834827B
:109360008DF83B828048FAF7FBFD8598401C85907C
:10937000F9F79AFC41F29B60FFF733FF7749C86029
:10938000F9F759FD80A8CDE9008040F23339002576
:1093900077E0284605F039FE002871D0008900EA00
:1093A000090434F0CC006BD040F20F312846FEF7B0
:1093B00039FC002864D0F9F795FD009900295DD1AA
:1093C000F9F748FC24F0EE0030F47E4017D01F205F
:1093D000FFF7F4FA0090F9F771FB009800284DD1DF
:1093E0007EB114F0010F03D007200199FEF71AFE99
:1093F00014F0100F03D0F0200199FEF713FE00982F
:10940000E0BB14F0220F06D0FCF71DFD0090F9F729
:1094100055FB009890BB8EB314F0020F16D0FCF7EA
:10942000A5F88346514801785148007848434FEAEF
:10943000400AFEF7C7FB4FF0060C5FEA0B0205D0AF
:1094400090F926105346604605F025FE14F0200FD3
:1094500014D0FCF722F804464648017846480078C4
:1094600008444FEA400AFEF7ADFB014608202200FF
:1094700004D091F92810534605F00DFEFEF769FD62
:109480006D1C05F0BEFDA842009802D9002880D0CE
:1094900003E0002808BF012000D0002018B1FCF72D
:1094A000B2FD01281FD087980023401C87905020D0
:1094B00084901A462121072008F04EFE00231A4608
:1094C0001946FE20CDF80080FCF796FE80AD05F031
:1094D00070FD50B381698891C169899141698A9110
:1094E000C0688B9027E017F0080F14BFA220A120BE
:1094F00084901A48C16859B11749096CC1F3082111
:10950000ADF838129DF83A12491C8DF83A1206E06F
:10951000ADF838829DF83B12491C8DF83B12C0F81B
:109520000C808698401C8690D0E74FF0FF308B90DF
:109530008A90899088900B4880904FF49870819021
:109540005020CDE982080021AA682C46084654F82C
:10955000203013E000500040006000408085001083
:10956000748700105443524600EE030067850010D4
:1095700068850010698500106A850010401C194438
:10958000B0EB920FE3D34842E860FF224FF4007142
:10959000684618F004F950222946684618F0DCF8AD
:1095A0009C4C2046FAF7DCFC69462046FAF77AFD27
:1095B0000020FCF729FB00233A464021072008F051
:1095C000CBFD0DF5157DBDE8F04F03F069BB924A68
:1095D000022804BF1181704707DC002804BF5180B6
:1095E0007047012808BF91807047112804BFD180BF
:1095F0007047122808BF5181704701460020022998
:10960000854A04BFB2F90800704709DC002904BF8D
:10961000B2F902007047012908BFB2F9040070478F
:10962000112904BFB2F906007047122908BFB2F928
:109630000A00704770B50126FEF7A4FC20B100694E
:10964000A12818BFA22801D0002070BD002405F079
:10965000D8FC002834D9204605F0D7FC00281EBFCE
:10966000058925F0CC0030F47C4024D040F20F3145
:109670002046FEF7D7FAF0B115F0010F0AD0F9F73E
:10968000CAFF38B944F4807200232021072008F073
:1096900063FD002615F0100F0BD00120FAF712F829
:1096A00038B944F4805200232021072008F054FDEB
:1096B0000026FEF74EFC641C05F0A3FCA042CAD8AD
:1096C000304670BD002070470020704752484078F7
:1096D0007047514900204870704770B5002105223D
:1096E0000846FFF738FD00234B4A002833D0517855
:1096F000002908BF5361A0F5A05CACF5257CBCF146
:109700000E0F28D9491CC9B25170D2F814C00A29C9
:109710006044506129D941495370096CC1F3082450
:10972000DCB14FF23951884224BF4FF619418142D2
:1097300013D34FF6A90181422CBF651C651E284634
:10974000FAF7CEFA44EA054200237521072008F013
:1097500003FD012070BD537007E041F29B60FFF7ED
:1097600040FD00281CBF012070BD002070BD10B559
:10977000FEF708FC38B32A4A0168914223D14168B8
:10978000B1F5987F1FD8D0F808C00146BCF5007F1E
:1097900019D800220B461146B2EB9C0F07D253F8A2
:1097A0002140491C2244B1EB9C0FF8D35AB9188FC1
:1097B00000281CBFA0F57F41B1F1FF0103D0FAF7EB
:1097C0008FFA012010BD002010BD10B5FEF7DAFBA6
:1097D000D8B1134A0168914217D14168B1F5987F19
:1097E00013D8D0F808C00146BCF5007F0DD8002280
:1097F0000B461146B2EB9C0F09D253F82140491C8D
:109800002244B1EB9C0FF8D30AB1002010BD188F91
:1098100010BD000000EE03008085001000600040D5
:109820005443524670470020704710B503F00700BC
:10983000042808BFFEF7FBF8002010BD10B403F0A9
:1098400007020024FE4BDFF8FCC3012A02D0022AE3
:1098500017D013E005208CF80000FB48CCF80C4032
:1098600000681A68532111701A68452151701A68EE
:10987000010A91701968C8701868047110BC002042
:1098800070479CF80020052A14D1DCF80C20052A2A
:1098900028BF104605D21B689B5C0370501CCCF897
:1098A0000C00052806D10120CCF80C4008700320DC
:1098B0008CF8000010BC0120704770B503F007025F
:1098C0000125DF4CDF4B4FF0000C012A02D0022AA9
:1098D00025D022E005201870DB48C3F80CC00068D2
:1098E0002268AC2111702268010A517021688870C9
:1098F0002068C570206880F804C005F0FBFA48B104
:10990000D24D286805F0FFFB20B128682168007E51
:10991000487102E02168FF204871002070BD1A786C
:10992000052A10D1DA68062A28BF104604D2246816
:10993000A45C0470501CD860062804D1C3F80CC085
:109940000D7003201870012070BD03F00702022A79
:109950001CBF002070472022027001200870704751
:109960002DE9F041B74F0D46064613F0070F04D01E
:1099700003F00700022808D004E012F0040F1CBF17
:109980000020B8700020BDE8F08103F083F90028C2
:1099900014BF0124002403F080F9002814BF022220
:1099A000002242EA0403B878002814BF04220022EF
:1099B00042EA0300307001202870BDE8F08170B5E4
:1099C00003F0070C00269F4C9D4DBCF1010F0AD0FF
:1099D000204613F0070F00780DD0BCF1040F08BF2C
:1099E000062818D029E0E6602868067028684670C6
:1099F0000520207021E005281FD1E068022803D24D
:109A00002B681A54401CE060022816D10120E66041
:109A10000870062010E02868007855280BD12868C7
:109A20004078AC2818BFBC2805D128680122411C09
:109A3000062003F015F903202070002070BD70B5DA
:109A400003F0070200257E4C7E4B012A02D0022A39
:109A500024D021E005201870DD6003F0CDF841F638
:109A6000E8710144B0F5783F10D8CA78086862F30D
:109A70001F60774A904208BF002007D10A18236868
:109A800012791A54401C1428F8D305E000202168EC
:109A90000D54401C1428FAD3002070BD1A78052AF2
:109AA00013D1DA68142A28BF104607D2D4F800C0B0
:109AB0001CF802C080F800C0501CD860142804D1E3
:109AC0000120DD60087003201870012070BD70B5A2
:109AD00003F0070200255A4C5A4B012A02D0022AF1
:109AE0003FD03CE005201870DD6003F085F841F6BA
:109AF000E8710144B0F5783F2BD8CA78086862F362
:109B00001F60534A904224D12268087C107022685A
:109B1000487C50702268887C90702068CA7CC27033
:109B200020680A7A02712268487A50712268887A1D
:109B300090712268C87AD0712268087D10722268FC
:109B4000487D50722268887D9072C87D2168C872F5
:109B500005E0002021680D54401C0C28FAD3002099
:109B600070BD1A78052A13D1DA680C2A28BF10466E
:109B700007D2D4F800C01CF802C080F800C0501C06
:109B8000D8600C2804D10120DD6008700320187013
:109B9000012070BD70B503F007020025284C294E46
:109BA000012A02D0022A36D033E005F002FA40B38F
:109BB000D0E906212368C0681A70D4F800C0130ADF
:109BC0008CF80130D4F800C0130C120E8CF802305F
:109BD0002368DA702268117123680A0A5A712368AF
:109BE0000A0C090E9A712268D171216808722268E4
:109BF000010A51722268010C9172010E2068C17233
:109C000004E021680D54401C0C28FAD30520307064
:109C1000F560002070BD3278052A10D1F2680C2A58
:109C200028BF104604D223689B5C0370501CF06070
:109C30000C2804D10120F56008700320307009E081
:109C4000CC6F0200B0850010044C004074870010F7
:109C500034CD12AB012070BD70B503F007020024B3
:109C6000F54DF64B012A02D0022A3ED03BE00520FA
:109C700018700026DC6002F0BFFF00F50051B0F55F
:109C8000783F98BF11F0030F27D1ED4A0868904242
:109C900004BF0022104620D151F82030401C1A4445
:109CA0000728F9D302B1C6B128680A7C02702A6875
:109CB000487C50702A68887C90702A68C87CD07074
:109CC0002A68087D10712A68487D50712A68887D4D
:109CD0009071C87D2968C87105E0002029680C547E
:109CE000401C0828FAD3002070BD1A78052A13D129
:109CF000DA68082A28BF104607D2D5F800C01CF839
:109D000002C080F800C0501CD860082804D101208F
:109D1000DC60087003201870012070BD2DE9F0414F
:109D200003F0070C0027C54E4FF00508BCF1010FEA
:109D30000DD013F0070F0FD03246BCF1020F12788E
:109D400010D0BCF1040F08BF062A26D058E086F8D0
:109D500000807770F76053E07270BA48F0620620B6
:109D600030704DE0052A15D1F268042A28BF10464C
:109D700009D2C2F10303D6F82CC0DB002CFA03F39E
:109D80000370501CF060042804D10120F7600870B3
:109D9000032030700120BDE8F08170780125002497
:109DA00010F0010F11D002F027FFB0F5783F23D853
:109DB0006A030021B1EB900F07D252F8043B491C13
:109DC0001C44B1EB900FF8D3B5B1707810F0020FCE
:109DD0000ED005F0EEF878B182680021B1EB920F59
:109DE00006D250F8043B491C1C44B1EB920FF8D347
:109DF000002D18BFF46200D1F762777086F80080FA
:109E00000020BDE8F081F0B503F0070C00268A4D74
:109E10008A4C83B0BCF1010F0ED013F0070F1DD098
:109E2000224603271278BCF1020F26D0BCF1040FA2
:109E300008BF062A36D03CE002AA01A9684603F012
:109E40007EFB052020702968019808702968009819
:109E50004870296802988870E6602AE0E068032864
:109E600003D229680A54401CE060022821D306214D
:109E70002170032808BFE6601BE0052A0FD1E268C5
:109E8000032A28BF104604D22B689B5C0370501C29
:109E9000E060032803D10120E6600870277003B05A
:109EA0000120F0BD286882780178407803F03AFB01
:109EB000277003B00020F0BD08B503F007000128AB
:109EC0000AD105F017F838B101208DF800000246DC
:109ED00069460D2002F0C4FE002008BD08B503F05D
:109EE000070001280AD105F005F838B100208DF8E7
:109EF0000000012269460D2002F0B2FE002008BDDC
:109F000008B503F00700012809D104F0F3FF30B1D0
:109F100003208DF800000122694602F0A1FE002016
:109F200008BD0020704708B503F0070001280AD1DA
:109F300004F0E0FF38B10B208DF8000001226946E3
:109F4000032002F08DFE002008BD1FB513F0070F9F
:109F50000ED104F0CFFF58B19DF80800F0280AD0C8
:109F600004F0C8FF20B1012202A9092002F078FE06
:109F700004B0002010BDFEF72BF8F9E70020704771
:109F800070B503F007002C4C2C4D012808D013F0BD
:109F9000070F12D0042804BF2878062816D01FE027
:109FA0000020E86021680870216848702168887086
:109FB0002168C8700520287012E0E86804280FD2D4
:109FC00021680A54401CE860062008E004F092FF73
:109FD00030B104221046216802F042FE03202870AE
:109FE000002070BD10B503F00700012804D104F073
:109FF000A8F8124900200871002010BD7FB51C464A
:10A000000E46054613F0070F08D104F073FF28B180
:10A01000012202A91C2002F023FE03E004F0070045
:10A02000022802D004B0002070BD0AF0A4FA287003
:10A030000120307004B070BDCC6F0200B0850010FC
:10A0400054464953EFBEADDE10B503F0070CFE4C8D
:10A05000BCF1010F06D013F0070F09D0BCF1020FBD
:10A0600018D015E00020E06008F06DF8E0610FE026
:10A07000E068002804BF1002E06106D0012804D186
:10A08000E0691043E06108F05DF8E068401CE060C2
:10A09000002010BDE26812B1012A04D007E0A18BB4
:10A0A000090A017003E0237F037001200870501C2F
:10A0B000E060012010BD10B503F0070CE24CBCF1CC
:10A0C000010F06D013F0070F09D0BCF1020F18D012
:10A0D00015E00020E06008F039F8E0610FE0E0688A
:10A0E000002804BF1002E06106D0012804D1E06915
:10A0F0001043E06108F02DF8E068401CE0600020AB
:10A1000010BDE26812B1012A04D007E0A18B090A50
:10A11000017003E0237F037001200870501CE06091
:10A12000012010BD70B503F0070CC74D0E46044664
:10A13000BCF1010F06D013F0070F07D0BCF1020FDE
:10A1400018D015E00020E860286111E0E8680028D8
:10A1500004BF1002E86108D0012806D1E869104365
:10A1600081B2E861E88811F01AFCE868401CE860F8
:10A17000002070BD286902280ED2E88811F015FC75
:10A180002B6982B2002B04BF100A207004D0012B6F
:10A1900002D12270012030702869401C2861012002
:10A1A00070BD10B403F0070CA74CBCF1010F08BF41
:10A1B00000200BD013F0070F03D0BCF1020F09D021
:10A1C00005E0E068002808BFE280401CE06010BCA9
:10A1D00000207047E2681AB9A37903700120087063
:10A1E000501CE06010BC012070472DE9F047064686
:10A1F00003F00700944F8946012808BF002037D09C
:10A20000DFF84882924D13F0070F02D0022833D0B6
:10A210002FE0F868002808BF7A7027D0012804BF13
:10A220001002F86122D0022820D1F8691043F861A9
:10A230007E7884B204F05EFEC0B1062E16D2DFE84E
:10A2400006F00306090C1013A8F80E400EE0A8F85B
:10A250000C400BE02868848308E02868A0F81441CB
:10A2600004E02868048601E028684486F868401CF9
:10A27000F8600020BDE8F087386902282AD297F8F4
:10A2800001A0002404F036FEC8B1BAF1060F16D2C0
:10A29000DFE80AF00306090C1013B8F80E400EE0D0
:10A2A000B8F80C400BE02868848B08E02868B0F808
:10A2B000144104E02868048E01E02868448E38695F
:10A2C000002804BF200A307004D0012802D1347065
:10A2D00089F800003869401C38610120BDE8F0872A
:10A2E0002DE9F0411C4615460E46074604F002FED5
:10A2F00088B1564814F0070F04D004F00701022972
:10A300000CD008E0002D1ABF90F80801C0084FF0EB
:10A31000FF300CF02FFE0020BDE8F08190F808011E
:10A32000C008387001203070BDE8F0812DE9F0419F
:10A330001C4615460F46064613F0070F08D104F0D9
:10A34000D9FD28B1022D3CBF28460AF024F903E0CC
:10A3500004F00700022802D00020BDE8F0810AF0D6
:10A3600013F9307001203870BDE8F08170B503F04A
:10A3700007020026374C344D012A02D0022A15D09C
:10A3800012E008F0E1FF21680870FDF781FA21680A
:10A39000487004F015FB21688870FDF77FFA21688A
:10A3A000C87005202870EE60002070BD2A78052A4C
:10A3B00010D1EA68042A28BF104604D223689B5CA7
:10A3C0000370501CE860042804D10120EE6008707E
:10A3D00003202870012070BD2DE9F04103F0070C27
:10A3E0001C4E0025184CBCF1010F08D013F0070FCC
:10A3F00008BF627178D0BCF1020F76D095E0FDF70E
:10A40000C1FD6179012943D00A216161002875D01D
:10A410004169FF292CBFFF21C9B2326811708169DF
:10A42000FF2934BFC9B2FF2132685170C169FF29C9
:10A4300034BFC9B2FF21326891703268017CD1709B
:10A4400090F82010326807E0B0850010D036011077
:10A4500074870010CC6F02001171018C3268090AF8
:10A460005171016A3268090C9171016A3268090EF2
:10A47000D171016BFF2934BFC9B2FF21326811725B
:10A48000406BFF2834BFC0B2FF20316848724BE0F8
:10A490001121616158B3326890F83C1001231170AA
:10A4A000002100EB81023768B2F83EC0491C4FEA38
:10A4B0001C2C07F803C037685B1C92F83EC007F8F5
:10A4C00003C0B2F840C037685B1C4FEA1C2C07F889
:10A4D00003C0D6F800C05B1C92F840200CF80320A3
:10A4E0005B1C0429DDD31FE01FE021E006E0FFE74D
:10A4F000FF221121306817F052F915E0306805701D
:10A50000306845703068857031685020C870316897
:10A51000FF20087131684871316888713168C871ED
:10A520003068057230684572E5600020BDE8F08152
:10A530006369E2689A4228BF104607D2D6F800C085
:10A540001CF802C080F800C0501CE060984206D1A0
:10A550000120E56008706079002818BF657101204E
:10A56000BDE8F08103F00702FB4B4FF0000C012A1D
:10A5700008BFC3F80CC001D0022A01D000207047E8
:10A58000DA68022A3DBF80F800C0501CD86010462F
:10A59000022803D10120C3F80CC0087001207047C5
:10A5A0002DE9F047064603F00700EB4F8A464FF0CF
:10A5B0000008012808BFC7F80C8001D0022802D08B
:10A5C0000020BDE8F087F868A0BB0024254602F013
:10A5D00013FB014600F5005018384FF400524FF0BD
:10A5E0004009B1F5783F20D890F803C003686CF3B8
:10A5F0001F63DFF868C3634517D1091FB4EB910FE0
:10A6000006D252F8043B641C5D40B4EB910FF8D3C2
:10A61000C17D406961F31F60A84206D104F06AFC65
:10A62000012804BF8020307001D086F80090F868BF
:10A63000401CF860012803D1C7F80C808AF800009C
:10A640000120BDE8F0872DE9F04103F00702002664
:10A65000C34CC14D012A02D0022A56D052E0C14853
:10A6600000680520287004F045FC002849D0BE4F42
:10A67000386804F048FD002843D011F070F9804696
:10A6800011F071F939680A7E12F0040F11D0C98AED
:10A690002268090A117039682268897D5170396809
:10A6A0002268898A090A917039682268097DD17007
:10A6B00010E0898A2268090A117039682268097DC8
:10A6C000517039682268C98A090A9170396822680C
:10A6D000897DD17022684FEA18211171216881F8B3
:10A6E00005802268010A91712168C8713868226862
:10A6F000817C11722268017C5172008B2168000AF2
:10A700008872EE600020BDE8F0812A78052A10D119
:10A71000EA680B2A28BF104604D223689B5C0370AA
:10A72000501CE8600B2804D10120EE600870032063
:10A7300028700120BDE8F0812DE9F04703F0070201
:10A740000025874C844B012A02D0022A5CD058E0B5
:10A75000052018700026DD6002F04EFA00F5005367
:10A76000B0F5783F98BF13F0030F44D17F4A1968C2
:10A77000914204BF0022114608D153F821C0491C60
:10A7800062440729F9D3002A08BF01269F7C93F869
:10A7900013807EB3002241F6E8710144B0F5783FA2
:10A7A00007D8CB78086863F31F606C4B984208BFEA
:10A7B00001228E7C91F81390002A08BF002013D04C
:10A7C00004F0F7FB216880690E70216881F8019020
:10A7D0002268010C000E91702168C8702068077112
:10A7E000206880F805800CE021680D54401C062884
:10A7F000FAD306E0FFE7002021680D54401C06282C
:10A80000FAD30020BDE8F0871A78052A13D1DA6858
:10A81000072A28BF104607D2D4F800C01CF802C08F
:10A8200080F800C0501CD860072804D10120DD60EA
:10A830000870032018700120BDE8F08770B5054648
:10A8400003F007000C46022829D104F053FB30B373
:10A85000454800220068037EC3F380008000C3F3F4
:10A86000400100EB410003F001010844082812D226
:10A87000DFE800F00406080A0C0E111004220AE0BA
:10A88000052208E0062206E0072204E0022202E098
:10A89000032200E001222A700120207070BD0020F8
:10A8A00070BD10B503F0070C2B4CBCF1010F06D0A6
:10A8B00013F0070F0AD0BCF1020F1AD017E00020E6
:10A8C000E060206111F0CDF8E06110E0E068002860
:10A8D00004BF1002E06107D0012805D1E0691043F0
:10A8E000E06180B211F0BAF8E068401CE06000203E
:10A8F00010BD2269022A0BD212B1012A04D007E04E
:10A90000A18B090A017003E0237F03700120087006
:10A91000501C2061012010BD70B503F00701002616
:10A920000D4D0446012908BF2E6301D0022901D034
:10A93000002070BD286B002804BF0D4816F07AFF78
:10A94000296B102928BF267002D20948405C20706C
:10A95000481C2863012070BDB085001034CD12ABB7
:10A96000CC6F0200044C00407487001054464953D9
:10A9700034AA00102DE9F04103F007010026FD4D37
:10A980000746012908BF2E6301D0022902D000200A
:10A99000BDE8F08195F8300000F00F0428792043DD
:10A9A00004D1F54816F046FF01202871052C28BF78
:10A9B0002E71F148005D3870286B401C286301201F
:10A9C000BDE8F08170B5044603F007000D4602288B
:10A9D0001CBF002070BD16F032FF207001202870CF
:10A9E00070BD2DE9F04103F007020026E34DE14C74
:10A9F000012A02D0022A1AD016E005202070002277
:10AA000011461046E66002F09AFD4FF6FF7101EA2A
:10AA100040006061FCF73CFF032803BF2878202832
:10AA2000D74802F09FFDA0620020BDE8F0812278A7
:10AA3000052A1DD1D4F814C0E268624528BF10462B
:10AA400007D212F0010F1CBF6378037013D0501CA3
:10AA5000E06060450CD10120E660087003202070A2
:10AA6000FCF716FF032806BF2878202802F087FD90
:10AA70000120BDE8F081A76A22F00103FB5A1F0AFA
:10AA800007706370E3E770B503F007020025B94C67
:10AA9000012A02D0022A11D00EE0BA48052200682D
:10AAA000B0F91210B0F91000227008444000E560BF
:10AAB000606102F0EFFFA062002070BD2278052ADD
:10AAC00017D1D4F814C0E268624528BF104607D2F7
:10AAD00012F0010F1CBF637803700CD0501CE060B3
:10AAE000604506D10120E56008700320207002F067
:10AAF000DFFF012070BDA66A22F00103F35A1E0A8F
:10AB000006706370EAE70020704770B50D46044692
:10AB100013F0070F04D003F00700022805D002E06D
:10AB20001046FCF7A9FE002070BDFCF7A8FE2070BF
:10AB30000120287070BD70B503F0070203258D4C0D
:10AB4000012A02D0022A17D014E004F007FB0646BF
:10AB5000FCF795FE0146304604F07DFD206200289A
:10AB60001ABF052020702570304604F058FD606241
:10AB70000020E060002070BD2278052A0BD1236AF6
:10AB8000E2689B5C0370501CE060626A904202D3F2
:10AB9000012008702570012070BD00207047002042
:10ABA00070477FB51C460E46054613F0070F08D1C7
:10ABB00004F0A0F928B1012202A9282002F050F8DF
:10ABC00003E004F00700022802D004B0002070BDAA
:10ABD00002F093FD28700120307004B070BD2DE9A3
:10ABE000F04103F007020027624E88460546012A1D
:10ABF00002D0022A0BD007E0052030701220F76047
:10AC0000706102F0AFFCB0620020BDE8F0813078E6
:10AC1000052819D1F2687069824228BF104608D20F
:10AC200012F0010F1CBF7078287010D0F068401C23
:10AC3000F0607169884207D10120F76088F8000050
:10AC40000320307002F09BFC0120BDE8F08100245D
:10AC500002F053FD012804D1F068B16A20F0010030
:10AC60000C5A200A28707470E0E770B50D4604464F
:10AC700013F0070F04D003F00700022805D002E00C
:10AC8000104604F068FA002070BD04F067FA2070E6
:10AC90000120287070BD7FB51C460E46054613F096
:10ACA000070F08D104F026F928B1012202A92220B9
:10ACB00001F0D6FF03E004F00700022802D004B040
:10ACC000002070BD08F0DAFC28700120307004B05C
:10ACD00070BD7FB51C460E46054613F0070F08D120
:10ACE00004F008F928B1012202A9232001F0B8FFDD
:10ACF00003E004F00700022802D004B0002070BD79
:10AD000008F0C2FC28700120307004B070BD7FB51F
:10AD10001C460D46064613F0070F08D104F0EAF86A
:10AD200028B1012202A91E2001F09AFF03E004F0DD
:10AD30000700022802D004B0002070BDFCF7EFFE2F
:10AD40000446FCF7D7FE44EA40003070012028702A
:10AD500004B070BD7FB51C460E46054613F0070FC4
:10AD600012D104F0C7F878B1012202A90C2001F039
:10AD700077FF0DE0B085001034AA0010F9850010AF
:10AD8000F02E01107487001004F00700022802D092
:10AD900004B0002070BD08F0D7FA28700120307090
:10ADA00004B070BD7FB51C460E46054613F0070F74
:10ADB00008D104F09FF828B1012202A90F2001F068
:10ADC0004FFF03E004F00700022802D004B0002087
:10ADD00070BD10F0BEF800F00F0040F010002870B9
:10ADE0000120307004B070BD2DE9F04103F0070C74
:10ADF000FD4D0E460746BCF1010F07D0FB4C13F08A
:10AE0000070F07D0BCF1020F1BD017E00020E8604D
:10AE1000286113E0E86804283CBF21680A5403282D
:10AE200009D1206821680068C97800BA20F0FF00C5
:10AE30000843FBF75BFCE868401CE8600020BDE8C5
:10AE4000F081286970B9FBF756FC216820F07E423A
:10AE5000100E08702168100C48702168100A887064
:10AE60002068C2702A69042A06D22068032A805CFE
:10AE7000387004BF01203070501C28610120BDE8EB
:10AE8000F0817FB51C460D46064613F0070F08D12A
:10AE900004F030F828B1012202A9102001F0E0FEF0
:10AEA00003E004F00700022802D004B0002070BDC7
:10AEB00010F053F800F00F0410F04BF864F31F107B
:10AEC00030700120287004B070BD70B5C64D1446B6
:10AED00013F0070F04D003F00702022A06D003E0A4
:10AEE0001046F5F769FA6C63002070BD95F83420C0
:10AEF00002700120087070BD70B514460E460546FC
:10AF000013F0070F04D003F00700022808D005E073
:10AF10001046FBF7CFFB60B216F096FC002070BD28
:10AF2000FBF7D1FB28700120307070BD2DE9F04196
:10AF300003F0070CAD4DAC4C4FF00008BCF1010F15
:10AF40000DD013F0070F1AD02246A94E032712780E
:10AF5000BCF1040F1DD0BCF1020F3DD02FE0C4F8AE
:10AF60000C80286880F80080286880F801802868B4
:10AF700080F80280286880F80380052007E0E068F8
:10AF800004281CD229680A54401CE0600620207066
:10AF900015E0062A13D103F0ADFF80B128680078D0
:10AFA00010B101280ED009E02868407800287068A8
:10AFB00014BF40F0800020F08000706027700020F7
:10AFC000BDE8F081286840780028706814BF40F41C
:10AFD000007020F40070F0E7052A0FD172687368E2
:10AFE000C2F3C01203F4007342EA53122B681A70C2
:10AFF00002700120C4F80C80087027700120BDE8A1
:10B00000F08110B503F00702774C012A02D0022A22
:10B010000DD00AE004F07AFB0021206200281ABF5C
:10B020004FF4056060626162E160002010BD636AF8
:10B03000E2689A4228BF104607D2D4F820C01CF814
:10B0400002C080F800C0501CE060984204BF01209C
:10B050000870012010BD10B4DFF898C113F0070F7D
:10B0600004D003F00702022A13D00FE0012A04BF24
:10B07000DCF8000040F0010006D0002A04BFDCF834
:10B08000000020F0010001D1CCF8000010BC00202D
:10B090007047DCF80030002213F0010F18BF0122C6
:10B0A000534BD3F804C0544B1B68B3F8F030C3F3D0
:10B0B0000334012303FA04F41CEA040F18BF42F01E
:10B0C000020202700B7010BC0120704770B514466C
:10B0D0000E46054613F0070F04D003F007000228C0
:10B0E0000ED00BE0002C14BF0120002003F008F864
:10B0F00024B13F48016821F440510160002070BD37
:10B1000003F005F8002814BF012200222A70012054
:10B11000307070BD2DE9F04103F0070C324C0F4642
:10B120008046BCF1010F12D0314E13F0070F4FF0E3
:10B13000030510D02046BCF1020F027826D0BCF1E6
:10B14000040F02BFE0680128062A33D036E005204C
:10B150002070002018E0E06810B1012804D011E050
:10B160006270062020700DE07168607800EA0203CA
:10B1700019437160716820EA020291437160F9F726
:10B180005BF82570E068401CE06017E0E06801288B
:10B1900008BF062A03D16078F9F764F82570706853
:10B1A00088F8000001203870E068401CE060012051
:10B1B000BDE8F0816078F9F755F825700020BDE80A
:10B1C000F08170B5044603F007000D4602281CBF4D
:10B1D000002070BDFCF75BFC002814BF0122002298
:10B1E00022700120287070BDB0850010CC6F020065
:10B1F00000100040144C00407487001070B50D46DC
:10B20000044613F0070F04D003F00700022805D00E
:10B2100002E0104607F0BFFF002070BD07F0BEFF40
:10B2200020700120287070BD70B50D46044613F0E3
:10B23000070F04D003F00700022805D002E01046F3
:10B24000F5F7CFFE002070BDF5F7CEFE207001208F
:10B25000287070BD70B503F00702DFF830C40C46EB
:10B260000546012A08BF05200DD013F0070F08BFBF
:10B27000062008D0022A09D0042A04BF9CF8000046
:10B28000062809D00EE08CF800000BE0FCF756FC15
:10B2900028700120207070BD03208CF80000012070
:10B2A000FCF74FFC002070BD70B503F00702F74DAE
:10B2B0000E460446012A04BF0020E86001D0022A9D
:10B2C00001D0002070BD11F00FFBEA68002A04BF16
:10B2D000000A207004D0012A02D1207001203070B1
:10B2E000501CE860012070BD03F0070210B4E74B6A
:10B2F000012A04BF0020D86001D0022A02D010BC6D
:10B3000000207047DA68022A0CD24FF0010C002AA4
:10B3100008BF80F800C005D0012A03D1682404705A
:10B3200081F800C0501CD86010BC0120704770B577
:10B33000044603F007000D46022807D013F0070F5C
:10B3400004BF1046FCF792FA002070BDFCF791FA9A
:10B3500020700120287070BD2DE9F04103F0070234
:10B360000027CA4E0C460546012A08BFF76001D0E7
:10B37000022A02D00020BDE8F08116F06AFAF268D5
:10B38000002A04BF000A28700BD00121012A04BF43
:10B390002870217005D0022A03D1F76021700320A4
:10B3A0003070F068401CF0600120BDE8F08170B59D
:10B3B00003F0070C0026B64DB44C82B0BCF1010F6F
:10B3C00006D013F0070F1FD0BCF1020F2DD029E0DB
:10B3D00068460EF0BDF9BDF8000029680009087044
:10B3E000BDF80200C0F30321BDF8000041EA0010DF
:10B3F000296848702968BDF80200887028689DF89F
:10B400000410C170E6600DE0E06804283CBF2968C4
:10B410000A54401CE060042804D104221420296846
:10B4200001F01EFC02B0002070BDE268042A02D2C6
:10B430002B689B5C0370501CE060042804D1012041
:10B44000E66008700320207002B0012070BD70B566
:10B4500003F0070C00268E4D8C4CBCF1010F06D07A
:10B4600013F0070F0CD0BCF1020F19D016E00EF04C
:10B4700062F92A68010A117029684870E6600DE0D7
:10B48000E06802283CBF29680A54401CE06002289A
:10B4900004D102221520296801F0E2FB002070BDD2
:10B4A000E268022A02D22B689B5C0370501CE060A9
:10B4B000022804D10120E6600870032020700120DA
:10B4C00070BD70B503F0070C0026714D6F4CBCF1D8
:10B4D000010F06D013F0070F12D0BCF1020F1FD0DE
:10B4E0001CE00EF010F92A68010E11702A68010C98
:10B4F00051702A68010A91702968C870E6600DE0F1
:10B50000E06804283CBF29680A54401CE060042815
:10B5100004D104221620296801F0A2FB002070BD8E
:10B52000E268042A02D22B689B5C0370501CE06026
:10B53000042804D10120E660087003202070012057
:10B5400070BD2DE9F04703F0070C514C00274F4E1A
:10B55000BCF1010F0FD013F0070F4FF0010833D0EB
:10B560000325BCF1020F56D0BCF1040F04BF3078A4
:10B57000062861D087E00EF016F905460EF024F992
:10B5800080460EF00AF981460EF018F9014620684F
:10B5900080F80090226808095070C5F3032040EA43
:10B5A0000110216888702168280CCD70216808710D
:10B5B0002168280E487121684FEA182081F806801A
:10B5C0002168C871F7605EE0F068002804BF236856
:10B5D0001A7023681B78012B01D03BB110E00028C2
:10B5E00018BF08283CBF23681A5409E02068077177
:10B5F00020684771206887712068C7710720F06054
:10B60000F068401CF06008283DD1F76081F80080A8
:10B610000620307037E0F268082A02D223689B5C6B
:10B620000370501CF060082803D1F76081F8008097
:10B6300035700120BDE8F087206800780EF0B0F882
:10B640002068216840788978000140EA11100EF0E6
:10B65000B8F82168206822688978407901F00F01E4
:10B6600040EA016021681279C978090441EA02219F
:10B6700008430EF09CF82068C08840BA0EF0A7F886
:10B680000EF0AAF835700020BDE8F087B0850010F4
:10B69000CC6F020070B503F0070C0026F84DF94C92
:10B6A000BCF1010F06D013F0070F0CD0BCF1020F54
:10B6B00019D016E00EF022F82A68010A11702968E4
:10B6C0004870E6600DE0E06802283CBF29680A5433
:10B6D000401CE060022804D12868008840BA0EF0BF
:10B6E00009F8002070BDE268022A02D22B689B5C38
:10B6F0000370501CE060022804D10120E66008704D
:10B7000003202070012070BD10B503F00702DD4C4E
:10B71000012A02D0022A27D024E003F0F7FF0023F9
:10B72000002804BF236263621BD000F15001216234
:10B730004168B1F5887F90F820100CD390F8212053
:10B7400001EB020C01FB02C190F8222090F82300CB
:10B750001044084404E090F822000A1801FB00207D
:10B760006062E360002010BD636AE2689A4228BF0D
:10B77000104607D2D4F820C01CF802C080F800C0E0
:10B78000501CE060984204BF01200870012010BDE9
:10B7900003F00702012A02D0022A05D002E0B949CB
:10B7A0000020C86000207047012202700A70104615
:10B7B000704710B513F0070F04D003F00702022AF8
:10B7C00005D002E0104601F0E7FE002010BDAE4AB1
:10B7D000127802700120087010BD10B513F0070F29
:10B7E00004D003F00702022A05D002E0104602F05E
:10B7F0006CF9002010BDA54A127802700120087073
:10B8000010BD0020704703F007029E4B012A04BFC1
:10B810000020D86001D0022A01D000207047DA68E9
:10B820004FF0010C002A08BF80F800C0501CD860FF
:10B83000012808BF81F800C0012070471FB513F030
:10B84000070F07D103F056FB20B1012202A90B20FC
:10B8500001F006FA04B0002010BD70B503F0070037
:10B86000884C1546012804BF0020E06024D013F066
:10B87000070F21D103F03EFBF0B1E068804E0328B2
:10B880003CBF31680D54401CE060032814D1F7F729
:10B890000BFA3068B0F8010045BAF7F70DF904006B
:10B8A00018BFF7F79FFB306829460078F5F771FF5E
:10B8B000002C18BFF7F799FB002070BD70B503F09E
:10B8C0000700704D1446012804BF0020E86020D016
:10B8D00013F0070F1DD103F00DFBD0B1E868684EDF
:10B8E00002283CBF31680C54401CE860022810D18B
:10B8F000F7F7DAF9F7F7E0F8040018BFF7F772FB8B
:10B90000306841780078F6F727F8002C18BFF7F771
:10B910006CFB002070BD70B50D46044613F0070F98
:10B9200004D003F00700022805D002E01046F7F724
:10B9300079FB002070BDF7F778FB2070012028709C
:10B9400070BD7FB51C460E46054613F0070F08D1A3
:10B9500003F0D0FA28B1012202A9182001F080F9E1
:10B9600003E004F00700022802D004B0002070BDFC
:10B9700007F0C5FC002814BF012200222A70012014
:10B98000307004B070BD7FB51C460E46054613F0FE
:10B99000070F08D103F0AEFA28B1012202A919203D
:10B9A00001F05EF903E004F00700022802D004B0C1
:10B9B000002070BD07F090FC28700120307004B0AA
:10B9C00070BD2DE9F04103F0070C2E4C0E460746E2
:10B9D000BCF1010F07D02A4D13F0070F07D0BCF1BF
:10B9E000020F19D015E00020E060206111E0E0684E
:10B9F00003283CBF29680A54401CE060032808D192
:10BA00002868B0F8010040BA01B228680078FDF754
:10BA1000DEFD0020BDE8F0812269022A12D242B97F
:10BA200028680078FDF7E9FD2A68010A5170296845
:10BA30008870286822691044012A4078387004BF51
:10BA4000012030702069401C20610120BDE8F08198
:10BA500010B503F007000B49012808BF00200CD0E7
:10BA600013F0070F064B02D0042811D021E0C8685C
:10BA700004283CBF1B681A54401CC86019E0000031
:10BA8000CC6F0200B0850010F9850010FF85001012
:10BA9000C86804280DD318681968407889780004AC
:10BAA00040EA01201968C978014318680078F7F75F
:10BAB0001FFF002010BD7FB51C460E46054613F043
:10BAC000070F08D103F016FA28B1012202A92B2092
:10BAD00001F0C6F803E004F00700022802D004B029
:10BAE000002070BD02F0B8FD28700120307004B055
:10BAF00070BD7FB50D46044613F0070F04D003F068
:10BB00000700022808D004E0012202A9122001F057
:10BB1000A7F804B0002070BD02F0B9FC207001202D
:10BB2000287004B070BD10B503F00702FE4C012A66
:10BB300002D0022A07D004E00020E060F8F75FFF9F
:10BB4000E061002010BDE268042A07D2C2F10303BD
:10BB5000D4F81CC0DB002CFA03F30370501CE06027
:10BB6000042804BF01200870012010BD10B503F0A7
:10BB70000700012807D103F0BDF920B100221146CA
:10BB80001F2001F06DF8002010BD2DE9F04103F0F9
:10BB90000705E54E174688460446012D04BF0020E0
:10BBA000F0601BD013F0070F16D103F0A3F998B182
:10BBB000F068DE4B03283CBF19680F54401CF0604E
:10BBC00003280BD1186890F9022090F9011090F920
:10BBD0000000FAF7ADFB01E0022D02D00020BDE825
:10BBE000F081F06830B1012809D002280CD0032878
:10BBF0000FD015E01420FAF764FA207010E0152039
:10BC0000FAF75FFA20700BE01620FAF75AFA207064
:10BC100006E01720FAF755FA2070012088F8000096
:10BC2000F068401CF0600120BDE8F08170B50D4661
:10BC3000044603F007000021BB4E012814BF13F097
:10BC4000070FF16001D0022801D0002070BDF0681C
:10BC500040B101280BD002280ED0032811D00428AF
:10BC600014D019E00120FAF72CFA207014E0022019
:10BC7000FAF727FA20700FE00320FAF722FA207073
:10BC80000AE00420FAF71DFA207005E00520FAF713
:10BC900018FA207001202870F068401CF060012024
:10BCA00070BD70B503F0070C0026A04C9E4DBCF192
:10BCB000010F06D013F0070F0CD0BCF1020F1FD0FC
:10BCC0001CE007F0B0FCEE60216808702168000AF3
:10BCD000487013E0E868022803D221680A54401C27
:10BCE000E86002280AD1EE602068007810F0010FA9
:10BCF00004D002221A20216800F0B2FF002070BD9B
:10BD0000EA68022A28BF104604D223689B5C0370AD
:10BD1000501CE860022804D10120EE600870032066
:10BD20002870012070BD7FB51C460E46054613F0F5
:10BD3000070F08D103F0DEF828B1012202A926205E
:10BD400000F08EFF03E004F00700022802D004B0E8
:10BD5000002070BD0FF074FE28700120307004B018
:10BD600070BD7FB51C460E46054613F0070F08D17F
:10BD700003F0C0F828B1012202A9212000F070FFD1
:10BD800003E004F00700022802D004B0002070BDD8
:10BD90000FF061FE28700120307004B070BD7FB5D7
:10BDA0001C460E46054613F0070F08D103F0A2F813
:10BDB00028B1012202A9252000F052FF03E004F07F
:10BDC0000700022802D004B0002070BD13F03CF838
:10BDD00028700120307004B070BD7FB51C460E463F
:10BDE000054613F0070F11D103F084F870B10FF07E
:10BDF0003EFE01469DF8080081420BD00FF034FE54
:10BE0000012202A9202000F02BFF03E004F007002C
:10BE1000022802D004B0002070BD0FF028FE287068
:10BE20000120307004B070BD2DE9FF413E4E1C462C
:10BE30000F46054613F0070F1CD103F05BF8C8B19D
:10BE40009DF80800002818BF012802D0022807D05A
:10BE500014E0F070012202A9082000F001FF0DE0BB
:10BE6000F07004208DF80800012202A9082000F0DB
:10BE7000F7FE03E004F00700022803D004B000201E
:10BE8000BDE8F081F07828700120387004B0BDE87A
:10BE9000F0817FB51C460D46064613F0070F08D10A
:10BEA00003F028F828B1012202A9082000F0D8FEEA
:10BEB00003E004F00700022802D004B0002070BDA7
:10BEC000FBF7E6FC801E052813D2DFE800F003072D
:10BED0000E05100000240DE001240BE0022406F002
:10BEE00030FA042808BF052404E0032402E00424F7
:10BEF00000E0FF2434700120287004B070BD2DE9EB
:10BF0000F0411C4617460E46054613F0070F0FD1A9
:10BF100002F0F0FF60B1384607F037F90022114611
:10BF2000012000F09DFE07E0B0850010CC6F0200FC
:10BF300004F00700022802D00020BDE8F08107F0DD
:10BF400027F9287001203070BDE8F08110B5104647
:10BF500013F0070F08BF07F0E5F9002010BD10B57A
:10BF6000104613F0070F08BF07F0E3F9002010BDDB
:10BF700070B5044603F007000D4602281CBF0020E0
:10BF800070BD07F0DEF920700120287070BD03F04D
:10BF9000070230B4FC4B4FF0000C012A05D0022AF6
:10BFA00004BF1A78022A0BD01EE002201870F7484E
:10BFB000C3F80CC06FF07F410068081AD86113E025
:10BFC000DA68042A28BF104606D2DD69D40025FAB3
:10BFD00004F40470501CD860042805D10120C3F873
:10BFE0000CC008700320187030BC0120704713F09B
:10BFF000070F04BFE64802700020704710B503F039
:10C000000700E149012804BF0020C86013D013F0E5
:10C01000070F10D1C868DF4B04283CBFD3F800C01D
:10C020000CF80020401CC860042804D1042213200E
:10C03000196800F015FE002010BD2DE9F0471646E6
:10C0400003F007020024D04F012A04BFFC603C61CA
:10C0500064D0DFF8448313F0070F07D0022A33D0EF
:10C06000042A04BF387806284FD058E0FD68002D18
:10C0700008BF3E6225D0012D06D0D7F81490AC1E23
:10C080004C4516D284B908E0701C7861396A0844BE
:10C09000B0F5007F88BF7C6113E04FF400724FF46D
:10C0A0007A31BE4815F058FBBA49386A096820440D
:10C0B0000E54601C484504D1B848C0F8FC810620E5
:10C0C0003870681CF8602AE0FF2202707B69CBB1EF
:10C0D000D7F820C03A699444BCF5007F10D2B04D27
:10C0E0002D68454518BF047005D10CF5783C9CF8C7
:10C0F00000C880F800C0501C984204BF012008709E
:10C10000501C38610120BDE8F0874FF47A30F7F712
:10C1100027FFA2494FF47A30F7F7C4FF3C700020A4
:10C12000BDE8F0872DE9F0478C4603F007010024B5
:10C13000954F1646012904BFFC603C6162D013F0A4
:10C14000070F984BDFF8608207D0022932D004290C
:10C1500004BF387806284DD055E0FD68002D08BF93
:10C160003E6224D0012D06D0D7F81490AC1E4C4569
:10C1700015D27CB908E0701C7861396A0844B0F5C2
:10C18000007F88BF7C6112E04FF40072194683483B
:10C1900015F0E2FA7F49386A096820440E54601CA1
:10C1A000484504D17D48C0F8FC8106203870681CE1
:10C1B000F86028E0FF2101707B69C3B13A6A3969F0
:10C1C0000A44B2F5007F10D2784D2D68454518BF5E
:10C1D000047004D102F5783292F800260270481CEF
:10C1E000984204BF01208CF80000481C38610120EF
:10C1F000BDE8F0871D461846F7F7B2FE67492846A6
:10C20000F7F750FF3C700020BDE8F08770B503F0F1
:10C2100007005D4C1546012804BF0020E06014D0E3
:10C2200013F0070F11D102F065FE70B1E0685949B3
:10C2300002283CBF0A681554401CE060022804D163
:10C2400002220968052000F00BFD002070BD2DE9D9
:10C25000F041054603F007004E4C4B4E0F460128B7
:10C260000AD013F0070F14D002281BD0042804BFF3
:10C270003078062834D03FE00020F0602168087054
:10C2800021684870216888702168C8700520307066
:10C2900032E0F06804282FD221680A54401CF06074
:10C2A000062028E0F06860B906F06CFD216808708F
:10C2B0002268010A51702268010C000E91702168F9
:10C2C000C870F06804283ABF2168095CFF21297012
:10C2D00024BF01213970401CF0600120BDE8F081CD
:10C2E00002F008FE40B12068C178006861F31F6069
:10C2F00006F043FD032030700020BDE8F0810020EF
:10C3000070477FB51C460E46054613F0070F08D14F
:10C3100002F0F0FD28B1012202A9292000F0A0FCC2
:10C3200003E004F00700022802D004B0002070BD32
:10C3300007F033F828700120307004B070BD03F0AE
:10C3400007001149012808BF002009D013F0070F8A
:10C3500007D1C86818B9164B1B681A448A61401C7B
:10C36000C860002070472DE9F04103F00701064C3A
:10C370001646054601291DD00D4F13F0070F3868EA
:10C380001CD002292FD02BE0B0850010B084001003
:10C3900035840010CC6F0200554E564D44AA001053
:10C3A000FCE9030000E60300324E564DFCE70300B3
:10C3B000948700100020E060206111E0A56905F07D
:10C3C000CFFF01280CD1A0693968884224BFE03131
:10C3D000814205D9E068042838BF2E54401CE06033
:10C3E0000020BDE8F081A66905F0BAFF50B1A2694E
:10C3F00039688A4224BF01F1E000904284BF20697D
:10C40000305C00D8FF2028702069401C206101208A
:10C41000BDE8F0817FB51C460E46054613F0070FB8
:10C4200008D102F067FD28B1012202A91D2000F009
:10C4300017FC03E004F00700022802D004B000203B
:10C4400070BD06F098FE28700120307004B070BDF9
:10C450007FB51C460E46054613F0070F08D102F0C3
:10C4600049FD28B1012202A9112000F0F9FB03E0E7
:10C4700004F00700022802D004B0002070BD12F0C2
:10C4800048FB28700120307004B070BD0020704758
:10C490000020704770B50D46044613F0070F04D016
:10C4A00003F00700022805D002E010460AF0E7F981
:10C4B000002070BD0AF0EFF920700120287070BDD7
:10C4C00010B503F00702F84CF84B4FF0000C012AAE
:10C4D00002D0022A34D031E0C3F80CC002F00AFDC9
:10C4E00000282BD0F24802F01DFE38B3F148006856
:10C4F000007E10F0040FEE4810D0C18C2268090AAB
:10C500001170226890F826105170818C2268090AF7
:10C510009170216890F82400C8700FE0818C226827
:10C52000090A1170226890F824105170C18C226899
:10C53000090A9170216890F82600C870002010BD8B
:10C54000DA68042A28BF104604D22468A45C047068
:10C55000501CD860042803D10120C3F80CC0087017
:10C56000012010BD70B503F00701CF4DCF4C01295C
:10C5700002D0022914D011E0012001F0D3FC0020E8
:10C58000E06001F0E4FC2081296808702A68010A53
:10C590000028517004BF002001F0C4FC002070BDD1
:10C5A000E168022902D22A68525C0270481CE060ED
:10C5B000012070BD2DE9F04103F007020026BB4DBC
:10C5C0000F460446012A02D0022A09D005E00520C0
:10C5D0002870EE602889400068610020BDE8F08185
:10C5E0002878052817D1EA686869824205D212F0D6
:10C5F000010F1CBF6878207010D0E868401CE8600C
:10C600006969884207D10120EE60387003202870E4
:10C61000002001F087FC0120BDE8F08101F0B0FCB2
:10C62000010A21706870E8E71FB513F0070F04D105
:10C63000012202A91B2000F013FB04B0002010BD52
:10C64000002070470020704703F007009749012839
:10C6500006D013F0070F04BF0878012806D014E0B5
:10C66000012008700020C86088610DE0C8680428B7
:10C6700005D28B69401C42EA03228A61C860042803
:10C6800003D103200870886908620020704703F016
:10C690000700DFF818C2012807D013F0070F04BF06
:10C6A0009CF80000022809D01EE002208CF800004F
:10C6B0000020CCF80C00CCF81C0015E0DCF80C00D5
:10C6C000022808D2DCF81C10401C42EA0121CCF8F8
:10C6D0001C10CCF80C00022806D1DCF81C00CCF8A9
:10C6E000240003208CF800000020704770B403F091
:10C6F000070200256D4C012A02D0022A06D002E072
:10C7000002202070E56070BC002070472278022A69
:10C710001CD1D4F824C0E268624528BF10460ED26E
:10C7200012F0030F04D1236A53F8046BC4E90763C2
:10C73000237F0370E069000AE061501CE0606045FF
:10C7400004D10120E56008700320207070BC012036
:10C75000704770B503F007000025544C0E460128C1
:10C7600006D013F0070F04BF2078022805D02BE075
:10C7700002202070E560E56126E0616AE068884299
:10C7800019D2E169090A41EA0262401CE26110F033
:10C79000030FE0600FD1206AB0F5802F28BF026040
:10C7A00006D2B0F5005F03D304224349F7F7CEFC6D
:10C7B000206A001D2062616AE068884204D101207D
:10C7C000E560307003202070002070BD70B503F06C
:10C7D000070C0025354CBCF1010F08BFE5603AD0CD
:10C7E00013F0070F03D0BCF1020F36D033E0052A57
:10C7F00008BF4FF47A302DD005DC16D2DFE802F006
:10C80000171A1D2022002B48202A006808BFF83084
:10C8100020D006DC102A1DD0112A08BF244819D0C8
:10C8200003E0302A11D0312A12D0A56113E04FF471
:10C8300000500FE04FF47F300CE04FF4483009E037
:10C840001E4807E04FF47C3004E001F0F1FC01E009
:10C8500011F0BBFCA061002070BDE268042A07D281
:10C86000C2F10303D4F818C0DB002CFA03F3037001
:10C87000501CE060042824BF01200870012070BD16
:10C8800070B403F0070C094DBCF1010F07D0064C42
:10C8900013F0070F14D0BCF1020F2ED02AE00020B5
:10C8A000E860286126E00000CC6F0200B08500102F
:10C8B000D036011074870010CC85001000EE030004
:10C8C000E86805283CBF21680A54042810D1236871
:10C8D0002268D4F800C0D3F80130A96912781BBAD5
:10C8E0009CF804C023F0FF0343EA0C0341F8223014
:10C8F000401CE86070BC002070472B6973B1042BAA
:10C9000007D22268032B1A445278027004BF012018
:10C910000870581C286170BC012070472268D5F847
:10C9200018C012785CF8222026684FEA126C86F84C
:10C9300001C026684FEA124C86F802C026684FEA0A
:10C94000122C86F803C0D4F800C08CF80420D8E775
:10C9500010B503F00700012804D1002211460E2073
:10C9600000F07EF9002010BD2DE9F04103F007042E
:10C97000A94E174688460546012C04BF0020F060EA
:10C9800017D013F0070F12D102F0B4FA78B1F068A3
:10C99000A24902283CBF0A681754401CF0600228D4
:10C9A00007D102220968072000F05AF901E0022CA1
:10C9B00002D00020BDE8F081F26812B1012A04D053
:10C9C00009E0FAF765FF287005E0FAF767FF2870BD
:10C9D000012088F80000F068401CF0600120BDE8EC
:10C9E000F08170B503F0070000258B4C012808D0BA
:10C9F00013F0070F0BD0042804BF2078062825D099
:10CA00002DE0A561E5616570E560257027E0E068CF
:10CA1000022807D2A16942EA0121A161617811448B
:10CA2000617010E0042807D2E16942EA0121E16166
:10CA300061781144617006E0052804D261788A4269
:10CA400004BF06212170401CE06008E0D4E9060123
:10CA500001F088FC002804BF0120A0702570002090
:10CA600070BD10B56C4C13F0070F07D003F0070032
:10CA7000042804BF2078062822D02BE0E068022892
:10CA800007D2A16942EA0121A16161781144617074
:10CA900013E06349091808D260490968014401F8A4
:10CAA000022C61781144617007E05E49091804D2D4
:10CAB00061788A4204BF06212170401CE06009E0D1
:10CAC0005949A06901F070FC002804BF0120A07042
:10CAD00000202070002010BD03F0070CBCF1010FF6
:10CAE00000D0BEE74C49002088614870C8600870DB
:10CAF000704730B403F007050024DFF81CC1012D96
:10CB000007D013F0070F0DD0022D3CD0042D54D0C8
:10CB10006FE0CCF81840CCF81C40CCF80C408CF8F6
:10CB2000004066E0DCF80C0002280BD2DCF818109C
:10CB300042EA0121CCF818109CF8011011448CF83D
:10CB4000011019E0042817D2DCF81C10032842EA6F
:10CB50000121CCF81C109CF801301A448CF80120FB
:10CB60000AD106228CF80020DCF81820114304BFFB
:10CB70004FF40071CCF81C102C49401CCCF82C1040
:10CB8000CCF80C0035E0DCF80C20042A28BF104655
:10CB90000AD2C2F10303DCF82C50DB0025FA03F3C0
:10CBA0000370501CCCF80C00042803D10120CCF8F1
:10CBB0000C40087030BC012070479CF8000006282B
:10CBC00015D1DCF8180000224102DCF81C004302F9
:10CBD0001046B2EB930F06D251F8045B401C2A4476
:10CBE000B0EB930FF8D3CCF82C208CF80040CCF8A5
:10CBF0000C4030BC002070474FF47F300168880A39
:10CC0000424211EB822218BF401C404201EB8000DF
:10CC1000C01C20F003007047B0850010CC6F0200EC
:10CC2000FEFDFFFFFDFDFFFF44AA0010EFBEADDEDD
:10CC3000F848002202704270827002714271C27024
:10CC4000DFF8D4C3114601EB410300200CEB430392
:10CC50001A54401C0628FBD3491C2029F3D37047E3
:10CC600014F0FCBD2DE9F04115460E460746F7F7D6
:10CC7000DBFD00F008040820F7F7D1FD2A46314615
:10CC8000384614F0EBFD05462046F7F7C3FD28466D
:10CC9000BDE8F081DF4880787047DE484078704713
:10CCA000DC490020487070472DE9F04100250C4612
:10CCB0002C2880F02082DFE800F0F4F316242D3CCD
:10CCC0001B49F24CF4848ACCF18F98A7C3F0EFEEA5
:10CCD000EDF4FBEBEAE9E8A2E7E6E5E4E3E2F4E100
:10CCE000E0F4DF9DF4DE0020F8F78EFF00F002BADA
:10CCF0002078AC280CBF01200220FAF7A0FE00F03B
:10CD0000F9B921780120FAF7DEFDC2490120487007
:10CD100000F0F0B9E178206861F31F6002F015FAC5
:10CD200001210320FAF7CFFDBA490120487000F035
:10CD3000E1B9208840BA06F028F802210320FAF76A
:10CD4000C2FDB4490120487000F0D4B96178207860
:10CD5000DFE0B04E01277770307870BBF6F7B5F89A
:10CD600058B324783770FAF793FD012808BF0024E0
:10CD700014F0040F18BFFCF7A5FC14F0020F06D046
:10CD80001F20FBF71BFEF9F75EF844F0010414F0D6
:10CD9000010F10D0FAF77CFD022802D106F009FA43
:10CDA00048B1FAF775FD052802D101F03CFB10B13E
:10CDB0000020F9F733F8002030700020707000F088
:10CDC0009AB92078401E01F085FE00F093B92078D2
:10CDD00006F0BDFA00F08EB9207810F00F0018BFF1
:10CDE00001200EF0CAF800F086B920780EF0BBF8EA
:10CDF00000F081B9207806F0C4FA00F07CB9207800
:10CE000006F0B0F900F077B9207818B101280CD0FD
:10CE100000F071B9002011F079FE022011F087F9BD
:10CE2000032011F0A3F900F066B9012011F06EFEA5
:10CE3000022011F06DF9032011F089F900F05BB9BF
:10CE4000207801F021FB207800284FF00100E8D085
:10CE5000F2E7207830B3FAF71BFD052800F04B818C
:10CE6000022818BF012506F057FA01460220FAF7FA
:10CE70002AFD00F040B92EE035E12EE129E1CDE0B8
:10CE8000C4E0F1E09CE07FE0CCE030E131E02CE078
:10CE90001CE00DE08BE085E079E06BE03CE050E0E9
:10CEA00002E170E000210620FAF70DFD00F022B942
:10CEB0002078002818BF012006F017FA20780028F3
:10CEC00018BF012001F096FA00F015B9207806F09D
:10CED000F8F900F010B901F0BFFB0146207881425B
:10CEE00018BF01F0B4FB00F006B9208806F004FB7F
:10CEF00000E1207820B1012845D0022805D0FAE0D1
:10CF00004FF47F30F7F72CF8F5E002F04BF80021F2
:10CF10000420FAF7D8FCEDE0F7F786FC00F00804EF
:10CF20000820F7F77CFC3B49CA78002A04BF00229E
:10CF30008A702046F7F76EFC01210620FAF7C3FC41
:10CF4000D8E02078062804D2DFE800F00306090BB9
:10CF50000E1102210846DCE702210520D9E7002155
:10CF600006E000210420D4E700210620D1E70421B7
:10CF70000320CEE7E0782268002360F31F6262217D
:10CF8000072005F0E9F8B6E0F9F766FAB2E02068A4
:10CF9000E17800BA20F0FF0008430CF0E0FB0CF051
:10CFA0001BFCA8E0208840BA0CF0C8FBA3E0206876
:10CFB000E17800BA20F0FF0008430CF0A8FB9AE0EB
:10CFC000FAF766FC02281CBF0628052871D12078D4
:10CFD000012811D0FAF774FC0546FAF759FC064609
:10CFE0002078002804BF0020F8F70EFE022D14BFA1
:10CFF000052D062E7ED104E00CF025FD0021062033
:10D0000087E706F089F90146284682E7207806F08E
:10D0100030FB6FE0E885001044AC0010207806F08B
:10D0200030FB67E0207800F00100FAF772FD0EF0A7
:10D0300051FC18B1FAF72CFC02280CD02078C0F370
:10D040004000FAF73CFD207800284FF0000008D09F
:10D0500011F07DF84EE02078C0F34000FAF71DFD96
:10D06000F1E711F083F845E00EF0F5FC247806F0C6
:10D07000DAFA054606F0CDF9012808D1042C06D0CD
:10D080000EF028FC18B1FAF703FC02280DD0012C91
:10D0900008BF28460ED0022C08BF45F0805009D0AA
:10D0A000042C18BF082C08D024E0204606F078F99C
:10D0B00020E020E006F0BCF907E045F0005006F063
:10D0C000B7F9042C18BF082C14D120460EF0BEFC72
:10D0D00010E0207811F0BBFE0DE020780EF0ADFCE2
:10D0E00006F09DF807E0207800F0F8FA03E02078D9
:10D0F00007F03EFA01252846BDE8F081E849CA68F4
:10D100001043C860704710B5E0B1FAF7C1FB0446A0
:10D11000F7F7C0FF0220F8F75DF8052C0DD0782056
:10D12000F3F773FF0520F7F7A2FFDE48F8F7D4F80E
:10D13000F8F7B7F8F8F73CF80DE03C20F3F765FF97
:10D140000320F0E7F8F73DF8F8F7B8F80020F8F713
:10D15000C3F8F7F781FFBDE81040F8F75BBE10B5E4
:10D16000F3F73CFF10F0010F08BF10BDFAF790FB7A
:10D17000052818BF10BDF3F754FF3C2804D0BDE8C4
:10D1800010400220F8F726B8FAF788FB022804D0EE
:10D19000BDE810400020F8F71DB8BDE810400120A0
:10D1A000F8F718B8BE4910B508208871FAF770FB77
:10D1B000022818BF012813D0032818BF05280FD054
:10D1C0000020F5F78AFEF7F7FCFFF8F777F8002064
:10D1D000F8F782F8F7F740FFBDE81040F8F71ABEFD
:10D1E000AFF2DD00BDE81040F5F777BE2DE9F0475E
:10D1F0004FF00008F5F779FEDFF8A4A20446DAF84C
:10D200000C00C14640B1DAF80C0010F0400F18BF16
:10D2100044F00404CAF80C9014F00F067DD00127E6
:10D22000FAF736FB05463046F5F762FE012E1DD0B3
:10D23000FAF734FB44EA0064002322460321072066
:10D2400004F08AFF14F0050F14BF00200120F3F74B
:10D2500093F814F0060F60D04FF00108FAF71EFBA8
:10D260000646022D45D0052D0AD056E09AF8060054
:10D27000854208BF00278AF80650002FD8D1E8E77A
:10D2800014F0020F1AD0F8F7F1FC00281CBF0020A0
:10D29000F8F7E6FCF3F7F0FA50B3F3F7FCFA040AF8
:10D2A000F3F7F9FAC0B244EA002200236C2102200D
:10D2B00004F052FF0020F3F7D9FA20E07A484069E1
:10D2C0008047044601F0C8F901281CBF207810F0FF
:10D2D000040F02D010F0080F02D00120F8F7C0FCB4
:10D2E000724C206820B10120F8F78EFCC4F8009041
:10D2F00005E014F0020F1CBF0120F8F785FC01F0D7
:10D30000A7F8002818BF01F0AAF8022E05D0022DB8
:10D310004FF0020004D001F077F84046BDE8F087F6
:10D3200005F0F2FFF9E72DE9F84F0026F8F737F896
:10D33000FAF7AEFA022804D101F098FD002818BFD0
:10D340000126FFF753FF002818BF0126DFF85081A0
:10D3500098F8020000287DD0D8F808006D464FF0FC
:10D36000FF344FF0000940B1D8F808200023012114
:10D37000084604F0F1FEC8F80890F7F755FA00F0F7
:10D38000080A0820F7F74BFA98F80300DFF820B1F5
:10D3900008B398F8050000EB4001401CC0B20BEB4D
:10D3A000410188F80500202828BF88F8059098F8E2
:10D3B0000300401E88F803004C780F780020002CF2
:10D3C00005DD0A1892782A54401C8442F9DC81F861
:10D3D000009081F801905046F7F71CFA002C49DBC9
:10D3E00022466946F8B2FFF75FFC08B1012641E02A
:10D3F000D8F808006D464FF0FF3440B1D8F8082047
:10D4000000230121084604F0A7FEC8F80890F7F7AA
:10D410000BFA00F0080A0820F7F701FA98F8030061
:10D4200018B398F8050000EB4001401CC0B20BEBAC
:10D43000410188F80500202828BF88F8059098F851
:10D440000300401E88F803004C780F780020002C61
:10D4500007DD00E01EE00A1892782A54401C84423E
:10D46000F7DC81F8009081F801905046F7F7D2F987
:10D47000002CB5DAF7F7D8F900F008040820F7F720
:10D48000CEF998F80310002908BF88F802902046CA
:10D49000F7F7C0F9002E14BF01200020BDE8F88F77
:10D4A000E8850010ADF0000090740200588600106E
:10D4B00044AC001002460020022928BF704752B138
:10D4C000012A18BF704701EB4100C0EB4110FE4933
:10D4D00001EB8000704740F2DB104843FB49F7E75F
:10D4E00070B5F7F7A1F900F008060820F7F797F9EB
:10D4F000F74C00256078FF2806D240F6D861F34843
:10D5000014F02FF9E5702571E079FF2805D2E821A4
:10D51000ED4814F026F9257265723046BDE870407A
:10D52000F7F778B9DFF8ACC300FB01F31CEB030C91
:10D5300088BF7047E64B1A62C3E906017047DFF8FF
:10D5400090C30028DCF8183018BF0360E0480029B9
:10D55000C06918BF0860002A1CBFDCF820101160E9
:10D5600058437047DA4801214171007840F2DB11DD
:10D5700080F001004843D54901EB80007047D44852
:10D58000C278002132B1027922B9027882F0010218
:10D590000270C17041717047CD4900231E284A783E
:10D5A000487006D01F2804BF0120087002D05128FF
:10D5B00000D10B7010467047C548007840F2DB116F
:10D5C00080F001004843C14901EB800070472DE91C
:10D5D000F007BF4F97F800C040F2DB140CFB04FCCF
:10D5E000BA4CBE6904EB8C0C03FB06F40CEB440C48
:10D5F0008E4234BF35460D46FC69E31A934238BF6C
:10D600001A46BB78012B16BF052B6C0800244FF07F
:10D610000008002A9CBFBDE8F00770472346AC42D3
:10D620000FD297F80290B9F1050F30F8139006BFAA
:10D63000A3EB040A2CF81A902CF813905B1CAB4255
:10D64000EFD308F101080CEB460C00EB41009045CC
:10D65000E4D3BDE8F00770472DE9F0419C4F144634
:10D660008C4601467A7806981D468A4218BFBDE866
:10D67000F08101213971012802D0022824D029E04B
:10D68000387840F2DB1148439049BE6901EB8001D4
:10D69000A64234BF32462246F869A84238BF054642
:10D6A0000023002D16D90020002A06D91CF800708E
:10D6B00021F81070401C8242F8D85B1C01EB460137
:10D6C000A444AB42EFD305E000232A46214660463E
:10D6D000FFF77DFFBDE8F04100F09FBC7C4A0128C8
:10D6E0001146D072497808BF242004D0002806BF14
:10D6F0002429FF207047507070477548C07A7047E2
:10D7000070B4DFF8D4C1DCF800C0DCF818C01CF03D
:10D71000040F1ABF012424EA0C060CF00106056868
:10D720000C68002E1CBF1B1B5C1E1CF0020F1CBFD4
:10D73000521B551E1CF0040F19BF04600D600560DC
:10D740000C6070BC7047002808BF70476049634B8D
:10D750004A7863491B78002A097818BF022A05D045
:10D76000042A18BF092A01D0012230E75D4A127845
:10D77000012A84BF5C4A1378012200F068BC2DE9BD
:10D78000F04FDFF84C9193B0012189F8041057490C
:10D79000544C554E0D785149DFF830B10F7899F857
:10D7A0000110122934D00DDC092921D005DC002913
:10D7B0001CBF0229042911D11AE0102918BF112910
:10D7C0000CD125E022297CD004DC132920D021298A
:10D7D00077D003E0242975D0512919D0002800F012
:10D7E000548100233A462946FFF7F1FE00F04DB977
:10D7F0002178012902D93E4937780D78002800F0B8
:10D80000448100233A46294600F021FC00F03DB94E
:10D81000F5F74AFAF5F750F90090002818BFF5F728
:10D82000E1FB2078012888BF3778F5F75BFB10F023
:10D83000020F18BF7F1CDFF8BC8099F8016099F8CF
:10D84000000040F2DB114143D9F818000BEB8104D2
:10D85000A84238BF0546D9F81C00B84238BF074671
:10D86000F5F76DFC01900020F6F7C8F84FF0000ABC
:10D87000002F4FDD4FF00009002DC4BF0AEB4A0016
:10D8800000EB0A1B3EDD019810F90900262824BF91
:10D89000002024F8190031D200F0010108EB813199
:10D8A00000EBD07001EB8B014010102E51F82000DE
:10D8B00036D0112E3BD0122E0CBFC0B2F6F7A4F812
:10D8C0001AE03AE041E00000DCBB001004AD0010BB
:10D8D000F88500104AFCFFFF748700106585001072
:10D8E0006B85001066850010688500106485001047
:10D8F000678500100000013024F8190009F10109C2
:10D90000A945C0DBF7480AF1010ABA45806904EB72
:10D910004004AFDB0098002818BFF5F766FBB4E0C1
:10D9200010F4003FC0F34230CAD04042C8E710F4C0
:10D93000803FC0F30420F8D1C2E700287DD0002347
:10D94000BA1C2946FFF743FE9FE0002875D0064623
:10D95000E5480068007E10F0040F07BF2C46BA4669
:10D960003C46AA46032300934FEA5A0261080993F2
:10D97000201F0A930B930C92CDE901100D920E9289
:10D98000CDE90331AAF104020F921092CDE905030B
:10D990001192CDE907105346224609A96846FFF7C0
:10D9A000AFFE5346224609AF0AA9E84601A8FFF791
:10D9B000A7FE5346224607F1080108F10800FFF7C9
:10D9C0009FFE5346224607F10C0108F10C00FFF7B9
:10D9D00097FE5346224607F1100108F11000FFF7A9
:10D9E0008FFE5346224607F1140108F11400FFF799
:10D9F00087FE5346224607F1180108F11800FFF789
:10DA00007FFE5346224607F11C0108F11C00FFF778
:10DA100077FE5346224607F1200108F12000FFF768
:10DA20006FFE99F8000040F2DB11414300220BEB3E
:10DA30008100914620F8129000E026E058F822106C
:10DA4000A1F1010C491C61451CD357F822104B1E53
:10DA5000491C99420FD303FB05C136F9114030F937
:10DA600012108C42C8BF20F8124057F822105B1CDD
:10DA7000491C9942EFD258F822100CF1010C491CB4
:10DA80006145E2D2521C092AD4D313B0BDE8F04F4D
:10DA900000F0C3BA934801218172807980F00100BF
:10DAA00000EB4001C1EB4010904901EB8000704752
:10DAB0008C48027A002132B1427A22B9827982F00E
:10DAC0000102827101728172704786491E28CA79EB
:10DAD000C87108BF002003D01F2808BF012000D153
:10DAE0008871104670477F48807980F0010000EB14
:10DAF0004001C1EB40107D4901EB800070472DE9EA
:10DB0000F04F7B49DFF8DC8185B00F7879490E78DA
:10DB1000012188F8091098F80710744C4FF000099B
:10DB2000102918BF11293AD0122918BF132936D04D
:10DB3000F0B198F8061001EB4102C2EB411104EB81
:10DB40008102002116EB070C18BF674C10D0236828
:10DB5000002E5B8A03BF30F811500B4422F813509B
:10DB600030F8113018BF22F81130491C8C45EED81E
:10DB7000F6F75AFE00F008040820F6F750FE98F871
:10DB80000A0000281CBF012188F808107CD020461C
:10DB9000F6F740FE88F8099005B0BDE8F08FF5F77C
:10DBA00083F8F4F789FF0290002818BFF5F71AFAF6
:10DBB00098F80750D8F82400009098F8060000EB79
:10DBC0004001C1EB401004EB800BF4F701F8002892
:10DBD0006AD01120F2F7A9FF00280CBF12201120F3
:10DBE00060F3070A0120F2F7A0FF002814BF01200C
:10DBF000022060F30F2A0AF0FF000190F5F7FEFE05
:10DC0000F5F79BFA00240390002E1FD903980257C2
:10DC1000142AA8BF143A02DA0A2AA8BF1232262A06
:10DC200028BF2BF814900ED2DDE90010F4F7C9FDDF
:10DC3000102D4AD0112D4FD0122D0CBFC0B2F5F7C8
:10DC4000E3FE2BF81400641CB442DFD30BEB460652
:10DC5000CAF3072B5846F5F7D1FEF5F770FA002402
:10DC60008246002F1AD91AF90420262A28BF26F83E
:10DC7000149010D258460099F4F7A3FD102D3BD014
:10DC8000112D40D0122D00E043E00CBFC0B2F5F7DB
:10DC9000BBFE26F81400641CBC42E4D302980028A2
:10DCA00018BFF5F7A2F963E70120F2F73EFF00285D
:10DCB00014BF0120022060F3070A1120F2F735FF9C
:10DCC000002814BF1120122093E710F4003FC0F386
:10DCD0004230B6D04042B4E710F4803FC0F3042095
:10DCE000F8D1AEE7F885001074870010DCBB001097
:10DCF000698500106A85001010F4003FC0F34230BF
:10DD0000C7D04042C5E710F4803FC0F30420F8D1EB
:10DD1000BFE798F8060080F0010088F8060088F850
:10DD2000089034E770B50D46EB4901220A71EB4AC1
:10DD300049781678EA4A212914781EBF2229232916
:10DD400070BD002818BF002D11D000232246314697
:10DD5000FFF73DFC631C012221462846FFF737FCF4
:10DD600005EB4400A31C01223146FFF730FCBDE85F
:10DD7000704000F052B970B50446C068D64D68B125
:10DD8000697859B9D749097801298CBFD649D4494E
:10DD90000B78D6490122097800F059F9A06820B122
:10DDA0006978002908BFFFF7EAFC6878102804BFEB
:10DDB0000020FFF7E4FC6878112804BF0020FFF77B
:10DDC000DEFC6878122804BF0020FFF7D8FC6878D2
:10DDD000132804BF0020FFF7D2FC206920B1E979A5
:10DDE000002908BFFFF78BFEE879102804BF002048
:10DDF000FFF785FEE879112804BF0020FFF77FFEBA
:10DE0000E879122804BF0020FFF779FEE87913288B
:10DE100018BF70BD0020BDE8704070E62DE9F74FD7
:10DE20008046AE480D46002690F800A0AC48AA49AE
:10DE3000344690F80090BAFBF5F000FB09F701209A
:10DE40000871487B0978DFF8A8B288420ED0A24A50
:10DE500040F2DB1148430BEB8001107840F2DB12FB
:10DE600050430BEB8000920013F085FC02980028D1
:10DE700088BFDFF864B22DD99BF80EC00022BCFB2E
:10DE8000F9F009FB10C101FB0AF100FB0510002DA0
:10DE900012D938F814309BF8001040F2DB1E01FB59
:10DEA0000EFE9349641C01EB8E0100EB020E521C26
:10DEB00021F81E309542ECD80CF10100C0B28BF86D
:10DEC0000E00B84224BF00208BF80E00761C02988A
:10DED0008642D1D38049887B401EC0B28873874276
:10DEE0009CBF781E88730878487303B0BDE8F04F74
:10DEF00000F093B87848017800F1280281F0010120
:10DF000032F81110002918BF7047017881F0010123
:10DF1000017000210182037822F81310754A0078FD
:10DF2000115470476C49087370476B48007B704709
:10DF300070B5694C0025257025732582658240F6F1
:10DF4000D8616B4813F00DFCA562A58270BD6249D3
:10DF5000087800224A8280F001001431095C69B11E
:10DF600040F2DB11624A414332F82110A1F55062C0
:10DF7000B63A02BF604931F8100070470020704780
:10DF8000554B187803F1140C80F001014FF6FF7027
:10DF90001CF80120012A18BF704740F2DB104843EB
:10DFA000534A02EB80005A8A30F81200521C5A82FF
:10DFB000514B33F81120521E1204120C23F8112079
:10DFC00004BF00220CF8012070474B49A1F1280240
:10DFD000137801EB43010B8803440B8092F800C0D7
:10DFE000012102F1140303F80C10118A0844108275
:10DFF0007047394A138A03EB5000404B01445B18C9
:10E0000024BF00207047117840F2DB125143384A98
:10E0100002EB810101EB4000704770B5F6F704FC9C
:10E0200000F008060820F6F7FAFB2B4C6079002573
:10E03000002801BF207880F001002070E5701CBF2F
:10E040000120E0703046F6F7E5FB257170BD2DE943
:10E05000F047994616460D460446F5F775F85FEA0F
:10E06000000C1CD01C49087840F2DB125043204AB7
:10E07000D1F8188002EB800009FB08F200EB4200A7
:10E08000454594BF2F464746C969A1EB0901B142F6
:10E0900038BF0E460021002E09D8BDE8F0874B4658
:10E0A000324629462046BDE8F047FFF790BA0023E4
:10E0B000002F08D91CF9032034F8122020F813206F
:10E0C0005B1C9F42F6D8491C00EB480004EB45045A
:10E0D000B142ECD3BDE8F087F885001064850010EC
:10E0E0006585001066850010688500106B8500103E
:10E0F00004AD00100C860010208600104AFCFFFFC3
:10E100004249002814BF00200120087070473F4892
:10E11000007800280CBF01200020704701203B49F7
:10E1200048707047394800214170017800291ABFB2
:10E130004068002870473648016821F001010160FD
:10E1400070473248017821B131490A6842F0010232
:10E150000A60002141608160C160016170472B4805
:10E16000017821B12A490A6842F001020A600021BF
:10E1700041608160C1600161704700B501784278FB
:10E1800085B0890141EA82018DF8001041880909B2
:10E190008DF80110818809098DF80210817801F04D
:10E1A0000F02017962F31F118DF80310017A8DF8C7
:10E1B0000410417A8DF805108179C27901F03F0190
:10E1C00002F00C0241EA02118DF80610C179827A40
:10E1D000890102F0010241EA42118DF80710C17B6A
:10E1E0008DF80810017C8DF80910817C407C01F0CD
:10E1F000030161F31F108DF80A0000208DF80B0059
:10E200000390684613F02FFB05B000BD2486001074
:10E21000144C0040002818BF47484849886370479D
:10E220004648806B444988420CBF0120002070475B
:10E2300042487047424B4FF0000C1C681B1F1D6882
:10E240003E4B19605A603F49D963DC6214F0804F3D
:10E2500022D0290C5985290A83F8291083F82850DF
:10E26000598D19B1598D012242EA014C93F82910B8
:10E2700039B193F82910022242EA014C32490C6864
:10E280001C6393F8281039B193F82810032242EA4E
:10E29000014C2E490C685C632D490C60091DC1F8C6
:10E2A00000C02C4A81691160B0E816109960DA60EC
:10E2B0001C61C3F814C090E807109861D9611A6214
:10E2C000C3F824C0986B1C49884202D123492248D4
:10E2D0000860FEE72249012804BF09607047022850
:10E2E00018BF704708471548D0F8EC201C498A42EF
:10E2F00004BFD0F8F0208A4208D1D0F8F4208A4236
:10E3000001BFD0F8F8208A4201207047C0F8EC1015
:10E31000C0F8F010C0F8F410C0F8F81000207047F2
:10E3200006480F49C0F8EC10C0F8F010C0F8F4101F
:10E33000C0F8F81070470000504D5544005F0110C0
:10E340002CED00E0544C414638ED00E034ED00E0A7
:10E35000344C00403C4C0040AD2007B0304C0040F5
:10E36000ADDEADDE70B50E460446F9F791FA04282D
:10E3700011D1A4F5C07080280DD2A019A0F281108F
:10E38000802808D265020024002E04D92846F5F71B
:10E39000E7FD012801D0002070BD641C05F5007563
:10E3A000B442F3D3012070BD70B50D460446F9F7B1
:10E3B0006FFA04280AD1A4F5C070802806D2600242
:10E3C0002946F5F76FFE012808BF70BD002070BD1B
:10E3D00010B5074CFEF7A7FF012808BF10BD206845
:10E3E00000F091FE002818BFF9F7C3FAF2E7000029
:10E3F00074870010FE4A0028916814BF41F00100A4
:10E4000021F0010090607047F94B99680A0E1207DD
:10E4100021F07F4142EA006211439960022818BF4F
:10E420007047F2F71CBAF2488068C0F30360704787
:10E43000EF488068000F7047ED483221006948437B
:10E44000EC49A1FB001080087047E948406970471B
:10E45000E748406A7047E649012048627047E4494E
:10E46000002048627047E24800787047002818BFD3
:10E470000120DF4908707047DD48806A7047DC483A
:10E480000021816201707047D949C8627047D8483D
:10E49000C06A70472DE9F04387B040F20F31F9F7B9
:10E4A000C1FB002804BF07B0BDE8F08313F0E0F91A
:10E4B00013F0E3F9F7F750FB5FEA00097ED1F7F7B5
:10E4C000A9FC0020F3F75DF8CB48F4F740FB0120EE
:10E4D000F4F730FBF2F782FDC84DC54EC84F10F07F
:10E4E000010FC84615D00020F2F781FDFEF737FE78
:10E4F000C5F800802020F5F792FCC248F5F795FC9E
:10E500002020F5F77EFC33202860386890F81F0142
:10E510002BE0F6F7ABF9BC48F6F75DFAF6F744FAEC
:10E52000F6F76DFA41003868B0F80E21B1FBF2F150
:10E53000491CC1F34F01718090F8100110F0FF00E9
:10E5400070700AD0F6F75BFA39684000B1F80C1128
:10E55000B0FBF1F0401CC0F34F010846F6F7BFF9DD
:10E5600017202860386890F81E01F060F4F79CFBD3
:10E57000F4F7A2FA002808BFF4F719FD707838B153
:10E58000401E10F0FF00707004BF7088F6F7A7F906
:10E59000B068C0F3036421460520F1F7A2FEFEF740
:10E5A000C2FE012807D0B068C0F30360A04208BFD4
:10E5B000B9F1000F27D0F5F715F800E01AE0C5F81B
:10E5C00000802020F5F72BFC0020F5F72EFCF6F755
:10E5D000D6F940B1F6F7BBF9F6F7F1F90020F6F7F6
:10E5E000FAF9F6F750F9F4F75FFBF4F767FA002051
:10E5F000F4F7ADFA13F041F913F044F9F9F7A9FC77
:10E6000007B0BDE8F0836846F4F79BFF98B1684611
:10E61000FFF7B1FBF9F73CF92146009A08F04EF8F4
:10E62000684613F034F9814608F0BEF8F4F7DAFFD3
:10E63000F9F7B5F9B3E73868D0F8B00010F0704FCB
:10E6400002D0F9F796F9AAE7F9F7B0F9A7E7042895
:10E650003CBF67494860704765484068704770B57F
:10E66000054600240DF003FA022801D0204670BDB3
:10E67000664800EB0510C1685D48C26B91421CBF43
:10E68000012101640124F1E770B50546002404F07E
:10E69000C0FE70B10DF0DFF908280AD05B4800EB2E
:10E6A0000510C1685248C26B91421CBF0121016430
:10E6B0000124204670BD554A014602EB011100209D
:10E6C000CA684B49CB6B9A4208BF70470120086467
:10E6D000704770B505460024F7F7C8FA01280FD136
:10E6E0004348D0E90C1291420AD100F1440101EBF8
:10E6F0000511C26BC96891421CBF0121016401244C
:10E70000204670BD2DE9F0473D4F034600243A688E
:10E7100080002646D2F80011082B31BF21FA00F004
:10E72000D2F80421203822FA00F000F00F00DFF8C0
:10E73000C080C1F303229042C8E90C020FD001F05F
:10E740000F0181426FD1F7F791FA01286BD1386838
:10E7500090F8040100F00F00C8F8300063E00020DA
:10E76000DFF8A890C8F8400009EB041148680828B1
:10E7700008D23A688000D2F8002122FA00F000F0B6
:10E780000F0508E03A6880002038D2F8042122FA08
:10E7900000F000F00F050F2D04D08968204688474F
:10E7A000012807D0641C042CDED3D8F840000128CF
:10E7B0000CD103E02646C8F83050F6E709EB061006
:10E7C000C068C8F83C000020F7F71EFAD8F83810E7
:10E7D000D8F83000814226D0C8F83800F2F7FBFBA9
:10E7E0000446F2F7FBFBD8F83020D8F804100FE00D
:10E7F00038860010ABAAAAAA335C0010104800406B
:10E8000074870010E15200101B5300107C8600102A
:10E8100041EA022141EA044141EA006200238921E0
:10E82000072003F099FCD8F83000BDE8F0872DE907
:10E83000F0414F480068B0F91611B0F9140112F018
:10E84000F4FFF2F70CF80120F7F7DEF900200DF0E5
:10E850000BF910F0E9FA0420FFF754FFF7F7B9F9C4
:10E86000002004F064FF434D002601206E61AE617C
:10E87000C5E907606E6005F0B5F802200FF067FC8F
:10E8800000200FF083FC13F007F800202E61F8F74A
:10E89000C2FB002004F06FFDF8F7FAFF052830D125
:10E8A000A868010FC0F30364A14202D06E61AE619B
:10E8B000EE612046FFF726FF07462146052003F0BC
:10E8C0000FFD002C4CD0022C46D0042C4CD0A86854
:10E8D0000E2C4FEA106120F07F404FEA017104BF17
:10E8E0000843A86005D041F000710843A860F1F723
:10E8F000B6FFFEF718FD012803D0F8F7C9FF052879
:10E90000CED010F028F90020F8F773FB0020F1F7C3
:10E9100074FD0020F8F7D0FA174C6068C0F340206F
:10E9200004F029FDF7F76FF910F085FA606820F41C
:10E9300000706060F8F7ACFF062805D00020AE63D9
:10E94000F7F78EF90320686002200FF00FFCBDE896
:10E95000F04100200FF029BC3846FFF79BFDC8E7C7
:10E96000384612F09EFFC4E7384605F0DBF8C0E7F2
:10E97000748700103886001000100040704700288F
:10E9800008BF704780220146014812F0E5BE70477B
:10E99000C4C40010704705283CBFFE49087070478A
:10E9A0000020FC4988604860FB48006890F8CD0072
:10E9B000052838BF087070470020F6494860704746
:10E9C000F4480078704770B5F34D0024286890F83B
:10E9D000B80010F0020F0BD0F8F75AFF022807D149
:10E9E000EC482968007801EB8000B0F8D00084B2D0
:10E9F000204670BD70B5E84D4FF48054286890F8FB
:10EA0000B80010F0020F0DD0F8F742FF022809D12C
:10EA1000E0482968007801EB8000D0F8D000000CB5
:10EA2000C0F31304204670BDDA488078002818BF70
:10EA3000012070472DE9F041F8F72AFF022803D1A1
:10EA400004F0B7FB022803D04FF48050BDE8F081FA
:10EA50004FF480552E4604F077FCDFF83C830446E3
:10EA6000CC4FD8F8000090F8B81011F0010F0CD07E
:10EA7000B0F8C200B9684042814206DC2CB10020E7
:10EA8000641EB860204604F062FCD8F8001091F8CB
:10EA9000B80010F0040F18BF002C0AD0B1F8C8005D
:10EAA000621E9040B1F8CA20824238BF1046C0F3BF
:10EAB0001306D1F8F00010F0020F1CBFB97800293E
:10EAC00002D0000CC0F31305B54298BF3546284666
:10EAD000BDE8F0812DE9F04FDFF8BCA287B0DAF88D
:10EAE000001091F8B82012F0020F0DD0A94A91F849
:10EAF000CC90DFF8A8B21778002809DB484503D28C
:10EB0000B84218BF064643D107B00020BDE8F08FD9
:10EB10003E464FF0FF38F3F7D1FFF4F7EEFF002544
:10EB2000B9F1000F34D9DAF80000002400EB8500B9
:10EB3000B0F8D00081B22046F2F72BFEF4F737FA96
:10EB40006846F4F7FEFC002866D0029878B10146CA
:10EB500093489BF8002000785043421E07D331F9B8
:10EB6000020B0028B8BF40420444521EF7D2F4F70B
:10EB700039FDF3F7A3FF002322469221072003F07B
:10EB8000EBFAA04584BF2E46A0466D1C4D45CAD366
:10EB9000B74244D0052E3CBF7E490E70DAF8000023
:10EBA000B0F8CE1039B300EB870200EB8600B2F864
:10EBB000D020B0F8D00092B280B2801A484340F31F
:10EBC0000F34F6F76DFC774B9BF80020002193F88B
:10EBD00000C002FB0CF2002A0DD930F811202244AB
:10EBE00020F811209BF8002093F800C0491C02FB7C
:10EBF0000CF28A42F1D84FF4800004F04BFDDAF8B1
:10EC00000000002300EB86008021B0F8D00082B223
:10EC1000072003F0A1FA09E0F8F7ABFE90E704F053
:10EC200093FB03283CBF401C04F091FB012007B07C
:10EC3000BDE8F08F584857490068B0F8C20042421A
:10EC400088688242BCBF401E886070472DE9F04F43
:10EC500093B093460E4604464FF0000A04F074FB4E
:10EC6000DFF834814B4F0500D14610D112F01EFE63
:10EC7000D8F80010B1F8C410884208D30120C7F8B2
:10EC8000089004F064FB13B00120BDE8F08F002E63
:10EC90001FDDB8680028B8BFC7F8089007DBD8F8B0
:10ECA0000010B1F8C0108842BCBF401CB860D8F852
:10ECB0000000B968B0F8C000884215DC032D13D2FB
:10ECC000681CC7F8089004F042FB13B00120BDE8AF
:10ECD000F08F09D1D8F80000B0F8C2004142B868FE
:10ECE0008842C4BF401EB860B87850B1D8F8000060
:10ECF00090F8F00010F0040F1EBF002013B0BDE824
:10ED0000F08FD8F80000B0F9BE108C420EDD7968A3
:10ED100021447960B0F8BA00884210DC4FF0FF302F
:10ED2000C7F80490FFF7D6FE824608E0786800280E
:10ED300005DD002CD4BF01212146401A7860DFF8A0
:10ED4000689099F8000007283BD118485946007888
:10ED50004200684612F00FFDADF80040ADF80260C9
:10ED6000ADF804503889ADF80600B888ADF8080051
:10ED7000D8F80000B0F8BE10ADF80A10B0F8C01016
:10ED8000ADF80C10B0F8BA10ADF80E10B0F8C20023
:10ED90000EE000005C87001074870010648500108E
:10EDA0006885001065850010F98500106B850010DE
:10EDB000ADF8100099F80000072804BF6846FEF778
:10EDC000C2FC504613B0BDE8F08F474810B500684C
:10EDD000D0F8F00010F4807F06D0C0F3033001219A
:10EDE00001FA00F0F5F73EFA4049002048708870BB
:10EDF00010BD70B53D4D0024A878002814BF012631
:10EE00000026687828B904F0AEFA002808BF00216F
:10EE100000D001218E4227D00A1C18BF0122AA70FF
:10EE200031480068D0F8F03013F0040F0ED021B153
:10EE3000C3F30310052808D206E00021A960696029
:10EE400090F8CD00052800D22870012413F0020F9D
:10EE500018BF0124002A18BF0122002382210720A5
:10EE600003F07AF9F1F76DFA204670BD2DE9F04113
:10EE70001D4800270068D0F8F01011F4807F30D0D2
:10EE80001A4E7078051C18BF0125C1F30330184ACB
:10EE90005268012303FA00F0024011F4007F0AD007
:10EEA00092B10CF0D8FD042818BF08280AD002201F
:10EEB0000CF0CCFD06E03AB10CF0CDFD042818BFF3
:10EEC0000828F4D1012403E0002401200CF0BEFD49
:10EED000A54206D0201C18BF01207070FFF789FFE3
:10EEE00007463846BDE8F081748700105C87001043
:10EEF000001000407148007870477048406800F585
:10EF0000407070476D48406800F58070704770B57C
:10EF10006A4C4FF448306A4A60600168914204BF0D
:10EF20004168B1F50C7F3BD18168B1F5464F37D8C8
:10EF3000644AC568954223D04FF0000C03466246F0
:10EF4000BCEB910F0AD253F8046B521C86EA0C0CEE
:10EF5000B2EB910FF7D3BCF1000F21D1026A7AB165
:10EF60004FF0000C03466246BCEB910F06D253F8FB
:10EF7000046B521CB444B2EB910FF8D365450FD12A
:10EF8000012500F5807000F0BEF848B1606800F51A
:10EF9000407000F0C7F800281EBF2570012070BD2A
:10EFA000002070BD4549002008704FF44830F4F748
:10EFB000D7BF4248017841B14068414A0168914257
:10EFC00002BF4168B1F50C7F7047002070473B4B92
:10EFD0005B6803F580731844F5F7B8B8374B5B6886
:10EFE00003F540731844F5F7B1B83448406800F5AC
:10EFF000A0607047314B5B6803F5A0631844F5F7D8
:10F00000A5B82E484068006970472C4949680A69CC
:10F0100082429CBF0020704700EB400001EB0010D3
:10F0200000F5C0607047254A526802EB8000436AD1
:10F03000406E1A4400FB01207047204988607047E9
:10F040001E48806870472DE9F0011C4B0022012703
:10F05000D3E901469046831893F92030002B12DB48
:10F0600007FA02FC1CEA060F0DD002F0FF0C04EBBD
:10F070008C0CDCF82450DCF864C0254403FB0C53F2
:10F0800041F8223001E041F82280521C102AE2D3DC
:10F09000BDE8F00170470029B8BF704730B494460E
:10F0A000064A526802EB8000446A406E224401FB2B
:10F0B000002030BC1A466146F5F748B86887001052
:10F0C00054465053EFBEADDE10B5FFF720FFB0B190
:10F0D000FFF713FF01464FF4C472174812F03CFBD0
:10F0E000FFF710FF154C01464FF4E872206812F04C
:10F0F00033FB2068C06BBDE8104004F0A6B80220C6
:10F10000F8F79DFCE1E758B10D4A0168914207D13B
:10F11000406820F00F00B0F5407F04BF0120704729
:10F120000020704730B1006820F00F00802804BF35
:10F130000120704700207047D036011074870010FE
:10F1400041505352FE4840687047FD49486070473F
:10F15000FB4880687047FA4988707047F8488078A3
:10F1600070470200F7484FF008010068438A008AA0
:10F1700003FB00101CBFC01C20F0030070472DE9EA
:10F18000F04104460D460846F8F77CFB78B10126AD
:10F1900006FA04F010F0CA0F18BF002C07D0032C99
:10F1A00005D8E8494FF4403201200B6802E0002006
:10F1B000BDE8F081A04213D006FA00F111F0CA0FA9
:10F1C0000BD0598A1F8A4FF0080C01FB07C1C91CDC
:10F1D00021F0030C0CEB4C010A44401C0328E9D934
:10F1E0000120A8420CD0B3F812C01C8A08210CFBE5
:10F1F0000411C91C21F00301401C0A440328F0D962
:10F200001046BDE8F0812DE9F04F0E4690F821A0A0
:10F2100090F8209000F15005ADF20C4D17460124F6
:10F2200011463046FFF7ABFFA11E012E08BFC649AD
:10F2300006D0022E08BFC54902D0032E08BFC4491C
:10F240004FF0000830B102688A4204BF4068CDE93F
:10F25000002001D0CDE90018BE48022E01680CBF85
:10F26000B1F98A00B1F93A0086460CBFB1F988209D
:10F27000B1F93820934600230AFB09FCBCF1000FCA
:10F280000ED935F913107145D8BF8B4505DC914275
:10F29000C8BF0A468142B8BF08465B1C9C45F0D8EF
:10F2A000104400EBD07042100023BCF1000F88BF67
:10F2B000E94616D935F91300801A00EBD0704110D9
:10F2C0007F29C8BF7F2105DC11F1800FB8BF6FF027
:10F2D0007F0100DA002409EB03005B1C01729C45EE
:10F2E000E8D88DF804409DF80500FF283CBF401C7D
:10F2F0008DF80500ADF806206C4639463046FFF71C
:10F300003EFF78B18F49082209684B8A098A03FBBE
:10F3100001222146F4F71AFF01280CBF4FF0010823
:10F320004FF0000840460DF20C4DBDE8F08F2DE97E
:10F33000F047984615460E468146F8F7A0FAF8F7CA
:10F34000A1FA002808BFBDE8F0877D4F824C3878CD
:10F35000814588BFBDE8F0870CD287F800904FF058
:10F360000000F8704FF0FF024FF014017A4812F0DD
:10F3700016FA19E097F803C0BCF1050F28BFBDE8E5
:10F38000F087BCF1000F18BF00200DDD14F820102D
:10F39000B14206D104EB80014978A94208BFBDE81B
:10F3A000F087401C6045F1DBF87804EB800104F83D
:10F3B00020604D70A1F80280401CF870BDE8F08715
:10F3C00070B5054616460C460846F8F75BFA002865
:10F3D0001CBF681E032832BF022E002070BD04EB44
:10F3E000C400400105EB450100EB411006EB46016E
:10F3F00000EB011000F5403000F5686070BD2DE9AC
:10F40000F04F97B04FF0000816460D460746CDF86E
:10F410003080FF2230216846CDF8348012F0BFF9E9
:10F42000DFF838A14FF47F30CDF800A00168880ADA
:10F43000424211EB822218BF401C404201EB800087
:10F44000C01C20F0030000F500504549428A437C6F
:10F4500052BA007C63F31F4242EA006001900888C0
:10F46000A1F1040940BAADF80A003869039099F88F
:10F4700000008DF81800002231462846FFF7A0FF53
:10F480000446012231462846FFF79AFF4FF0010C4F
:10F49000012D04D0022D18BF032D40D083E000229F
:10F4A000114624B32368534521D1237A647A28B1C5
:10F4B000D0F800B0D34504BF027A417A181902EBA4
:10F4C000010A504583BFADF830C0ADF83430ADF817
:10F4D0003640ADF830809CBFADF83420ADF8361022
:10F4E000BDF83400BDF836100844ADF83200BDF860
:10F4F0003400BDF836109DF81820C0B28DF8080011
:10F50000C9B20CFA02F28DF8091012F00E0F19BFF1
:10F51000401C8DF80800481C8DF8090043E00021CC
:10F520006CB12268524524D1227A18B10368534540
:10F5300008BF017A8A4288BFADF830C012E018E0F7
:10F5400078870010748700104654525946544D3243
:10F5500046544D3394870010E4F300104646485358
:10F560007C8700108EBFADF83220ADF83080ADF84A
:10F570003210022D18BF032D15D1387C10F0300049
:10F5800004BF17B0BDE8F08FBDF832003146401C13
:10F590008DF808002846FFF7F2FD00280CBF404612
:10F5A00040798DF80900FE480DF1380A6B46B0E845
:10F5B00016108AE8161090E8071012AC84E80710BD
:10F5C0009DF81800082813D20EA951F82000B0F1B8
:10F5D000FF3F0DD007EBC000D0E90A10CDE90410C1
:10F5E00099F80300EF49820003F11C0012F0C3F800
:10F5F000BDF830106C46CAB231462846FFF7E0FE2F
:10F6000048B130222146F4F7A1FD01280CBF4FF08C
:10F6100001084FF00008404617B0BDE8F08F0146E2
:10F62000012200208A4012F0CA0F08BF7047082943
:10F6300028BF7047DFE801F00B0404040B0B040C37
:10F640000821D9480068428A008A02FB00107047EE
:10F650004FF490707047012310B50022834013F0DF
:10F66000CA0F14D0082812D2DFE800F011040404F5
:10F6700011110D07FFF783FD03E000220120FFF7C2
:10F680009FFE024603E04FF4443000EB8122104617
:10F6900010BD2DE9F04106460127F8F7F0F8804645
:10F6A000F8F7F0F8002808BFBDE8F081BF4D6868A2
:10F6B00010F4807F18BF02240DD00120A04010F06C
:10F6C000CA0F05D0424621463046FFF79CFD07464B
:10F6D000306978B90BE010F4007F18BF0324ECD137
:10F6E00010F0070018BF0124E7D1BDE8F0812878A9
:10F6F000112805D2424621463046FFF780FE0746D4
:10F700003846BDE8F081A949C8607047A74810B4E1
:10F71000C068002808BF4FF47C30A54A01689142B8
:10F720001CD14168B1F5007F18D38368002284465C
:10F73000B3F5056F88BF4FF405630021B1EB930F5C
:10F7400024BF10BC70475CF82140491C2244B1EB37
:10F75000930FF8D3002A04BF10BC7047002010BCE0
:10F76000704770B50022C260D0F808C0012113466E
:10F770000446BCF5056F88BF4FF4056C0022B2EB60
:10F780009C0F06D254F82250521C2B44B2EB9C0F13
:10F79000F8D35A42C260854A127912F0800F07D11D
:10F7A0004FF47C304FF405622146F4F7CFFC01465C
:10F7B00001290CBF0120002070BDFF2270B500257B
:10F7C000044605614FF40061503011F0E8FFA58454
:10F7D000E584E562A56265632563E563A563656409
:10F7E0002564E5640120A56470BD2DE9F0414FF466
:10F7F0007C3104466E4E0868B04218D14868B0F5B6
:10F80000007F14D38A6800230D46B2F5056F94BFBC
:10F8100094464FF4056C0020B0EB9C0F26D255F8AF
:10F820002070401C3B44B0EB9C0FF8D3F3B1FF2297
:10F830004FF40561204611F0B2FF4FF40870C4E99F
:10F8400000604FF40560A0600020E06084F82000B4
:10F8500084F8210084F8220084F82300206160618C
:10F86000A061E0612046FFF7A8FF07E0B2F5056F51
:10F8700088BF4FF40562204611F06EFF0120BDE8FD
:10F88000F08170B402684FF408715160016801F1B1
:10F89000500291F821C091F820300CFB03F102EBEB
:10F8A00041010022BCF1000F08D900EB4204521CB8
:10F8B000B4F8DE4021F8024B9445F6D80022002B24
:10F8C00008D900EB4204521CB4F8064121F8024B5F
:10F8D0009342F6D80022BCF1000F08D900EB420495
:10F8E000521CB4F8644021F8024B9445F6D800222B
:10F8F000002B08D900EB4204521CB4F88C4021F8CC
:10F90000024B9342F6D8B0F8DA2021F8022BB0F877
:10F91000DC2021F8022BB0F8D82021F8022B00249B
:10F920000022BCF1000F0ED904EB440505EB0415D1
:10F9300000EB850505EB4206521CB6F8526121F832
:10F94000026B6245F6D30022002B0ED904EB44056E
:10F9500005EB041500EB850505EB4206521CB6F8D5
:10F96000826221F8026B9A42F6D3641C042CD7D32E
:10F9700070BC70472DE9F74F88B000250A992C46D6
:10F980002E460968049101F150030999002984BFAA
:10F990000849D1F800802AD9002200280CE0000094
:10F9A000D86F0200E4F3001074870010788700100D
:10F9B00053454C469487001088BFB8F93A700DD96A
:10F9C00033F9021B0029B4BFC1F1000C8C46BC45C1
:10F9D000BCBF0D44641C521C8242F1D30999761CB1
:10F9E0008E42D9D3002CC8BF95FBF4FA08DC490835
:10F9F000414301EB5002049901EB4201B1F950A0DF
:10FA0000002102910191049950310091002103914C
:10FA10000999002969D9FA49009E069609684FF0AC
:10FA2000000B4FF00109B1F81CE091F824105F467B
:10FA3000D846CDF814B00791002829D9B6F900208E
:10FA40004FF0000C06999344634600280DD9B1F994
:10FA50000040A51A48BF151B7545B8BF0CF1010C35
:10FA600001EB49015B1C8342F1D307998C4503D319
:10FA700005997F1C1144059108F1010806EB490620
:10FA80008045DBD3002FC4BF059991FBF7F101DC62
:10FA90009BFBF0F1039B0A9A09B202EB4302A2F826
:10FAA0006410D74A1268538BAAEB0303994209DD0D
:10FAB000128B52448A4205DD019A11440191029948
:10FAC000491C02910099099A01EB400100910399A8
:10FAD000491C039191429ED30299002905DDDDE97D
:10FAE000011291FBF2F1019102E05146CDF804A020
:10FAF0000A9AA2F8DA100021029103910499503178
:10FB0000009100210491002865D9BD49009F069706
:10FB100009684FF0000B099EB1F820E091F825101C
:10FB2000D846D946CDF814B00791002E2BD9B7F995
:10FB300000204FF0000C069993446346002E0DD927
:10FB4000B1F90040A51A48BF151B7545B8BF0CF1A7
:10FB5000010C01EB40015B1CB342F1D307998C45CA
:10FB600004D3059908F101081144059109F101092F
:10FB700007EB4007B145DAD3B8F1000FC4BF0599D0
:10FB800091FBF8F101DC9BFBF6F1049B0A9A09B2A8
:10FB900002EB4302A2F88C10994A1268538BAAEB2D
:10FBA0000303994209DD128B52448A4205DD039A10
:10FBB000114403910299491C02910099891C0091FA
:10FBC0000499491C049181429FD302980028C4BF24
:10FBD000039991FBF0FA0A98A0F8DCA001980A9921
:10FBE000504400B200EBD0704010A1F8D8000BB028
:10FBF000BDE8F08F2DE9F74F8CB004460E980E99B2
:10FC0000DFF8FCA10668002008620E990746A4F1FF
:10FC10000108C8610E9988610E9948610D98A0F19C
:10FC20000109002866D90025002C5FD9F81707EBD9
:10FC3000D06020F01F01791A012202FA01F101912E
:10FC400041110E9800EB810000F11C0B009007FBA6
:10FC5000045006EB4000082FB0F950000CD1222DC3
:10FC60000ADB232D08DCDAF80010222D14BFB1F9CD
:10FC7000BA10B1F9B8100FE0002F18BF4F4507D1E7
:10FC8000002D12BF4545DAF80010B1F9B21003D0CB
:10FC9000DAF80010B1F9B010002904BFDAF800104A
:10FCA000B1F9B01088421EDD00994FF0010CCA690D
:10FCB00001991143CBF80010E91705EBD1635A11F4
:10FCC0000E9923F01F0301EB820101F1140249692F
:10FCD000EB1A0CFA03F31943116083B2EAB2F9B2DA
:10FCE0000720FFF724FB6D1CA542B0D30D987F1CA5
:10FCF000874298D3DAF8000090F8D11000291CBF91
:10FD000090F8D000002800F010820D9800270028FD
:10FD100040F20B82801E0590A01E04900025002C4E
:10FD200040F2FE81781E0021039000FB041006EBD8
:10FD300040000A90781C029000FB041006EB400083
:10FD40000990F81707EBD06020F01F01791A012203
:10FD500002FA01F1089141110E9800EB8100079021
:10FD60001C30069007FB045006EB40000190B0F9F0
:10FD700050200023082F3ED1222D3CDB232D3BDCDD
:10FD8000222D19BF0623B0F94E000523B0F9520009
:10FD90008242CCBF11460146E1B1111A4FF0640C0A
:10FDA00001FB0CF100290BDB8242D4BF8446944650
:10FDB0006144A1F1010100DD104691FBF0FC0BE074
:10FDC0008242CCBF94468446A1EB0C0101F10101B3
:10FDD000F3DDF1E74FF0FF0C4FF000000146002B80
:10FDE00000F04C81072B80F06B81DFE803F0FEFD13
:10FDF000FEFCFBFAF9000DB1454503D1032319E0E0
:10FE000094870010012D1CBF0498854211D03FB18A
:10FE1000012F08D04F4509D1142D0AD0012309E044
:10FE2000142DFBDD05E0142D03DDF7E7059887426F
:10FE300000D10423A5F12200012898BF092F08BF93
:10FE4000009707D000210091012898BF072F08BF15
:10FE5000BA4602D00D98A0F1010A082F0ABF212D41
:10FE6000A4F1010CAC460020DDF800B001465F456E
:10FE700009D0012F1DD00399012001FB045106EB8D
:10FE80004101B1F9501057452DD0DDF814B05F4550
:10FE90001FD1002D14BF4FF0000B4FF0010B454553
:10FEA0000CBF4FF0010E4FF0000E5BEA0E0B1AD1A3
:10FEB0000FE0002D14BF4FF0000B4FF0010B454534
:10FEC0000CBF4FF0010E4FF0000E5BEA0E0BDAD1C3
:10FED000D1E7DDF808B0401C0BFB045B06EB4B0BD5
:10FEE000BBF950B059443DB1012D1BD0DDF804B031
:10FEF000401CBBF94EB05944654529D0DDF810B01F
:10FF00005D451FD1002F14BF4FF0000B4FF0010BC8
:10FF10004F450CBF4FF0010E4FF0000E5BEA0E0B89
:10FF200016D10FE0002F14BF4FF0000B4FF0010B64
:10FF30004F450CBF4FF0010E4FF0000E5BEA0E0B69
:10FF4000DAD1D3E7DDF804B0401CBBF952B0594414
:10FF5000DDF800B05F4516D14DB1DDF808B0401CAA
:10FF60000BFB045B06EB4B0BBBF94EB059446545EC
:10FF700009D0DDF808B0401C0BFB045B06EB4B0B13
:10FF8000BBF952B05944574516D14DB1DDF80CB00C
:10FF9000401C0BFB045B06EB4B0BBBF94EB059440A
:10FFA000654509D0DDF80CB0401C0BFB045B06EB8B
:10FFB0004B0BBBF952B0594485B9DDF800B05F4531
:10FFC00018BF57450AD0DDF828B0801CBBF952B0E5
:10FFD0005944DDF824B0BBF952B05944654505E0F9
:10FFE0003EE036E043E05EE064E069E018D1DDF831
:10FFF00000C0674518BF574512D0DDF80CC0801C03
:020000021000EC
:100000000CFB045C06EB4C0CBCF94EC06144DDF803
:1000100008C00CFB045C06EB4C0CBCF94EC0614400
:10002000002818BF002A3FF4D5AE4FF0640C01FB46
:100030000CF191FBF0F002EBC20101EB0211D0EBED
:10004000810059BF1044401E801A401C90FBF2FCF6
:10005000C2E6FE48006890F9D51090F9D4002FE070
:10006000FA48006890F9D71090F9D60028E0F748D0
:10007000006890F9DF1090F9DE0021E0002F18BF32
:100080004F450BD1002D18BF454506D1EF480068FC
:1000900090F9D31090F9D20012E027B14F451CBF60
:1000A000002D454506D1E948006890F9DD1090F92A
:1000B000DC0005E0E548006890F9D11090F9D00027
:1000C00051EA000305D1E148006890F9D11090F998
:1000D000D0008C4501DC84451EDA07984FF0010CF6
:1000E000C1690898014306980160E81705EBD060E4
:1000F00043110E9920F01F0001EB830101F114035D
:100100004969281A0CFA00F00843186093B2EAB261
:10011000F9B20720FFF70BF96D1CA542FFF422AEE0
:100120000D987F1C8742FFF4F9AD0FB00120BDE8A8
:10013000F08F2DE9F04F146887B015460E468046C3
:10014000A1F12009202928BF4FF0FF3B05D24FF035
:10015000010000FA06F0A0F1010B31BF00200120E0
:1001600000FA09F0401E0290B8F1200F3DBF0120B7
:1001700000FA08F0401E4FF0FF3038BF002207D3CE
:10018000A8F120024FF0010101FA02F1A1F10102F0
:10019000C6F1200A202E34BF20FA0AF100FA09F134
:1001A000B2401143B040CDE90001206920F4FE6067
:1001B0002061A748406810F0010F79D010F4807FCB
:1001C00005D02A463146404601F07AFA8AE010F41A
:1001D000007F2A463146404602D0FFF70BFD81E002
:1001E00001F04EF90020A86107466861B8F1000FE0
:1001F00022D905EB4700B0F98C000028B8BF404277
:1002000000B292490968B1F93810814211DD7A09CA
:1002100005EB820C07F01F0301219940DCF8142044
:1002200083B21143CCF81410FAB2FF210420FFF777
:100230007EF87F1C4745DCD30027B8F1010F1CBFB7
:10024000A8F1010003904DD005EB4700B0F98E30C6
:10025000B0F98C20991A48BFD11A09B2DFF8ECC165
:10026000DCF800C0BCF932C08C4537DAB5F9DC10D7
:10027000B2EB010C48BFA1EB020C0FFA8CFC5A1A2E
:1002800048BFCA1A11B28C4513DB7A0905EB82010B
:1002900007F01F0C01224B6902FA0CF21A434A6163
:1002A000B0F88C30FAB2FF210420FFF740F815E0D7
:1002B0002BE0791C4B0905EB830E01F01F0C01228A
:1002C000DEF8143002FA0CF21A43CEF81420B0F81B
:1002D0008E30CAB2FF210420FFF729F803987F1C53
:1002E0008742B1D36969E869B14008432063A969CD
:1002F000286AB140084360636969202E34BF21FA3F
:100300000AF101FA09F1084360635149087910F0D4
:10031000040F00F0088200202863E8620846407855
:1003200028BB0027002E22D9484905EB4700096861
:10033000B0F95201B1F95C20824203DCB1F95E10E0
:10034000814211DA7A0905EB820C07F01F030121C3
:100350009940DCF82C2083B21143CCF82C10F9B270
:10036000FF220220FEF7E3FF7F1CB742DCD3002010
:10037000A86268623648407830BB0027B8F1000FA9
:1003800022D9324905EB47000968B0F98202B1F978
:100390005C20824203DCB1F95E10814211DA7A09F5
:1003A00005EB820C07F01F0301219940DCF82420A3
:1003B00083B21143CCF82410FAB2FF210220FEF7D9
:1003C000B6FF7F1C4745DCD300202864E863204843
:1003D000407890BB0027002E2FD91C4905EB470021
:1003E0000968B0F99E01B1F960208242DCBFB1F921
:1003F0006220904210DD7A0905EB820C07F01F03A2
:1004000001219940DCF83C2083B21143CCF83C1028
:10041000FF22F9B201200BE0B1F96C208242DCBF6F
:10042000B1F96E10884205DD83B2F9B2FF221020C7
:10043000FEF77DFF7F1CB742CFD30020A86368631F
:1004400003484078C8BB002704E0000094870010F0
:1004500078870010B8F1000F2FD905EB4700B0F9ED
:10046000CE02FE490968B1F960208242DCBFB1F9D1
:100470006220904210DD7A0905EB820C07F01F0321
:1004800001219940DCF8342083B21143CCF83410B8
:10049000FF21FAB201200BE0B1F96C208242DCBFEF
:1004A000B1F96E10884205DD83B2FAB2FF21102047
:1004B000FEF73DFF7F1C4745CFD300202865E86449
:1004C000A8646864E6484078F0BB0027002E22D973
:1004D000E24905EB47000968B0F9EA01B1F9642087
:1004E000824203DCB1F96610814211DA7A0905EB28
:1004F000820C07F01F0301219940DCF84C2083B2E5
:100500001143CCF84C10F9B2FF220320FEF70FFF85
:100510007F1CB742DCD30027B8F1000F24D9CF49A4
:1005200005EB47000968B0F91A03B1F9642082426B
:1005300003DCB1F96610814213DA7A0905EB820C0B
:1005400007F01F03012100E00EE09940DCF8442091
:1005500083B21143CCF84410FAB2FF210320FEF716
:10056000E6FE7F1C4745DAD3696AE86AB14040EA93
:10057000010EC4F838E0A96A286BB1400843E06373
:10058000696A202E34BF21FA0AF101FA09F141EA21
:100590000007E763696BE86B01FA06F140EA0102C4
:1005A0002264A96B286C01FA06F140EA010060643C
:1005B000696B34BF21FA0AF101FA09F141EA00003E
:1005C00060646B6CE96C03FA06F341EA0301A16411
:1005D0000391AB6C296D03FA06F341EA0301E16470
:1005E0006B6C34BF23FA0AF303FA09F343EA0101FF
:1005F000E164059132EA0E054EEA0501256420EA20
:10060000070C049147EA0C00C4F844C006EB08014B
:10061000069008BFBCF1000F45D000231A461846CB
:10062000002988BF4FF001083DD94FEA501904EB6B
:10063000890900F01F0AD9F8409008FA0AFA19EA65
:100640000A0F03D0864294BF521C5B1C401C81429F
:10065000EBD8012B10D105EA0B0040EA0E00A06395
:1006600002980CEA00003843E06325EA0B0020649E
:1006700002982CEA00006064012A14D1206C009AD0
:10068000A36B02401A43A263626C019BD4F83CC086
:10069000134043EA0C03E363009B984320640198F2
:1006A00022EA00006064DDE903208243A26404982A
:1006B00040EA020CDDE9050320EA0300E064069B42
:1006C00043EA000508BF002821D000231A46184637
:1006D000002988BF012717D94FEA501804EB880872
:1006E00000F01F09D8F8488007FA09F918EA090F3D
:1006F00003D0864294BF521C5B1C401C8142EBD845
:10070000002B18BF002A02D10020A064E0645448E6
:10071000007910F0010F06D0206B20EA0C00206356
:10072000606BA8436063206B0099084203D1626B41
:1007300001990A4203D0216941F01001216110EAB8
:100740000B0F03D1616B0298014203D0206940F086
:1007500020002061A06B0099084203D1E26B01994F
:100760000A4203D0216941F04001216110EA0B0FD8
:1007700003D1E16B0298014203D0206940F0800070
:100780002061206C0099084203D1626C01990A42F1
:1007900003D0216941F48071216110EA0B0F03D16C
:1007A000616C0298014203D0206940F4007020611E
:1007B000A06C002804BFE06C002803D0206940F43E
:1007C0008060206107B00120BDE8F08F2DE9F04F77
:1007D000CBB017460D460446F2F770F90120F0F74A
:1007E000A4F906461120F0F7A0F9304314BF012008
:1007F00002208DF8180014BF112012208DF8190066
:10080000F1F7E6F938B19DF818009DF819108DF848
:1008100018108DF819009DF81800F0F786F90028D7
:1008200018BF284604909DF81900F0F77EF90028BB
:1008300018BF20460590F2F780FC0022002D88BFEB
:1008400024A910D98356142BA8BF143B02DA0A2B13
:10085000A8BF12338B54521CAA4203E094870010A5
:1008600078870010EED3F2F76AFC0021002C88BFD5
:1008700024AA07D9435C02EB010C491C8CF82630F2
:100880008C42F7D8F2F72EFB0390FE480DF1180AC0
:10089000007910F0200F55D007F1DE0000902830CD
:1008A0000025E9460DF1100B01905BF825601AF860
:1008B0000500F3F7A3F80024002E1AD905EB450034
:1008C00000EB051024A901EB400818F90420262AA2
:1008D00028BF002006D21AF805000021F1F771FFA9
:1008E000F3F792F859F8251021F81400641CB4426B
:1008F000EBD36D1C022DD8D3E34C26781D2E21D1CD
:1009000000210A460DF11C085BF822500020002D42
:1009100088BF59F822C007D93CF8103028F81130A8
:10092000401C491C8542F7D8521C022AECD31D2ECC
:1009300008D14046FDF7E3F820781D2804BF07A83A
:10094000FDF7DDF8CF4D287910F00C0F00F0AF83E4
:10095000039800F0F000F2F77DF99DF81800F0F729
:1009600004FF07909DF81800F0F7A5FF00243790CA
:100970001AF80400F1F768FE44A941F824001AF8B7
:100980000400F0F7D5FF0EA941F824001AF804007E
:10099000F1F721F920A941F824001AF80400F1F731
:1009A00052F922A941F824001AF80400F0F7FCF8E3
:1009B00046A918AA41F824001CA81AA902EB84022F
:1009C00000EB840001EB84010092CDE9011016A830
:1009D00000EB840314A800EB840212A800EB84014E
:1009E0001AF80400F1F70EFC1AF80400F1F73DFDC7
:1009F0001EA941F824001AF80400F1F775FE10A9A9
:100A000041F82400641C022CB2D3A04E3068B0F828
:100A100048109DF81800F0F7BCFE002400211AF8D9
:100A20000400F1F7F7FD994E306890F84A101AF873
:100A30000400F0F791FF1AF804000021F1F7E5F83F
:100A40001AF804000021F1F718F91AF8040001213E
:100A5000F0F790F83068B0F84C101AF80400F1F78D
:100A600097FC1AF804000021F1F706FE641C022C22
:100A7000D4D384484FF00009007910F0040F00F03F
:100A8000DD813446206890F84B3090F85920B0F85A
:100A900050100091CDE9012390F84F3090F84E208E
:100AA00090F858109DF81800F1F7F3F9206890F8C5
:100AB0004B3090F85920B0F850100091CDE9012347
:100AC00090F84F3090F84E2090F858109DF819008B
:100AD000F1F7DFF99DF818000021F1F7CDFD9DF841
:100AE00019000021F1F7C8FD3AADF2F760FAFCF702
:100AF0001AFC012806D02846F2F723FD00287DD0F5
:100B0000F2F770FDF1F7DAFF3E99002204AD002004
:100B100055F82230002B0ED902EB420C0CEB021CD4
:100B200007EB0C1C31F8026B0CEB4008401CA8F8DA
:100B300052618342F6D8521C022AE8D35448D0E9C5
:100B40000010CDE90C109DF81800EFF7EEFF48906B
:100B50009DF81900EFF7E9FF49909DF8180040A9AA
:100B6000F0F797FF9DF8190042A9F0F792FF9DF862
:100B7000180008A9F1F70AF89DF819000AA9F1F779
:100B800005F8424C206890F84B3090F85920B0F8A6
:100B900052100091CDE9012390F84F3090F84E208B
:100BA00090F858109DF81800F1F773F9206890F844
:100BB0004B3090F85920B0F852100091CDE9012344
:100BC00090F84F3090F84E2090F858109DF819008A
:100BD000F1F75FF99DF818000CA9F0F7B5FF9DF843
:100BE00019000CA9F0F7B0FF00249DF818000021AF
:100BF000F1F742FD9DF81900002100E017E0F1F740
:100C00003BFD9DF818000021EFF775FF9DF81900D6
:100C10000021EFF770FF1AF804000121EFF76BFFD6
:100C20001AF80400C0F3011001280AD102E0F6F717
:100C3000A0FE5CE784F0010001211AF80000EFF744
:100C40005AFFCDF8E090CDF8E4909DF8180038A94F
:100C5000F0F7FFFE9DF8190038A9F0F7FAFE04A896
:100C6000002150F824801AF80400F1F750FE002506
:100C70000190B8F1000F55D904EB440024A900EB12
:100C8000041007E078870010FF850010948700109B
:100C9000D06F020001EB400107EB001B00910098B0
:100CA00038AA00214657CDF8E090CDF8E4901AF824
:100CB0000400F1F744FD202E06DBA6F120010120FF
:100CC0008840CDE9389003E00120B040CDE93809F3
:100CD0001AF8040038A9F0F7BCFE389838AAC043C7
:100CE000389039980921C04339901AF80400F1F777
:100CF00026FD3AAEF2F75BF9FCF715FB012806D0AA
:100D00003046F2F71EFC00287ED0F2F76BFCF1F7BC
:100D1000D5FE019800880BEB45016D1CA1F89E01E2
:100D20004545BCD3CDF8E090CDF8E4901AF8040026
:100D300038AA0021F1F703FD641C022CFFF455AF23
:100D40009DF8180008A9F0F7FFFE9DF819000AA900
:100D5000F0F7FAFE9DF818004899EFF7CCFE9DF8E1
:100D600019004999EFF7C7FE9DF8180040A9F0F760
:100D700070FE9DF8190042A9F0F76BFEFE4C20684A
:100D800090F84B3090F85920B0F854100091CDE90C
:100D9000012390F84F3090F84E2090F858109DF8AD
:100DA0001800F1F776F8206890F84B3090F8592049
:100DB000B0F854100091CDE9012390F84F3090F82D
:100DC0004E2090F858109DF81900F1F762F89DF840
:100DD00018000121F1F750FC9DF819000121F1F7ED
:100DE0004BFC3AACF2F7E3F8FCF79DFA012806D089
:100DF0002046F2F7A6FB00287DD0F2F7F3FBF1F7CF
:100E00005DFE002204AC00E081E03E9954F822C06F
:100E10000020BCF1000F0ED902EB420303EB0213DA
:100E200007EB031331F8025B03EB4006401CA6F806
:100E3000EA518445F6D8521C022AE7D3CF480079FC
:100E400010F0080F7ED0CC4C206890F84B3090F812
:100E50005920B0F856100091CDE9012390F84F3099
:100E600090F84E2090F858109DF81800F1F711F8FE
:100E7000206890F84B3090F85920B0F85610009147
:100E8000CDE9012390F84F3090F84E2090F858109B
:100E90009DF81900F0F7FDFF00210DF1100C002066
:100EA0005CF82120002A0CD901EB410303EB01136C
:100EB00007EB031303EB4005401CA5F83692824272
:100EC000F8D8491C0229EAD32068002590F8680068
:100ED000B5EB400F36DA206890F86800A842D4BF1E
:100EE000012100219DF81800F1F7C6FB206890F859
:100EF0006800A84200E00DE0D4BF012100219DF868
:100F00001900F1F7B9FB3AAEF2F751F805E0F6F740
:100F100030FDF1E6F6F72DFD66E7FCF704FA01284F
:100F200005D03046F2F70DFBD8B3F2F75BFBF1F7D3
:100F3000C5FD3E994FF0000904AB0022104653F85E
:100F4000296000E058E0002E05D931F91030401C2E
:100F50001A448642F9D8B2FBF6F2701E3DD009EB76
:100F6000490303EB091307EB031B31F9103001EBC5
:100F7000400C3CF9028CB3EB080348BF5B4231F9EB
:100F80001080B8EB020831F910804CBFA2EB0808C2
:100F9000A8EB02083CF902EC3CF902CCBEEB020ED5
:100FA00000E00FE04CBFA2EB0C0CACEB020CE045F8
:100FB0000BEB400C09DDBCF936824345C8BFACF8E9
:100FC000363208E0F6F7D5FCA7E7BCF9348298453D
:100FD000B8BFACF83432401EC7D109F1010901EBAA
:100FE0004601B9F1020FA7D320686D1C90F8680084
:100FF000B5EB400FFFF66FAF9DF818000799F0F7BB
:10100000C8FB9DF818003799F0F764FC00241CAD6C
:101010001EAE20AF0DF188080DF588790DF58C7B9B
:1010200059F824101AF80400F1F7F4FA0EA850F851
:1010300024101AF80400F0F78FFC57F824101AF85F
:101040000400F0F7E2FD58F824101AF80400F0F755
:1010500014FE5BF824101AF80400EFF78BFD1AA9B0
:1010600018A851F8241055F8242050F82400CDE990
:10107000000116A8029250F8243014A850F8242039
:1010800012A850F824101AF80400F0F702FF56F8DE
:1010900024101AF80400F1F77BF910A850F8241076
:1010A0001AF80400F1F7E8FA641C022CB8D303988C
:1010B000F1F7D0FD4BB0BDE8F08F304801218160E1
:1010C000112101700021C170FDF73BB82B490020B0
:1010D000886070472DE9F04F284DADF56F7D0127F1
:1010E0001120AF604FF00008287085F80380FDF7ED
:1010F00028F868684FF4407131EA000008BF002604
:1011000000F099811D20FCF747FAED901D20FCF7B7
:10111000DCFCDFF868A0EE904FF46D716846DAF8F9
:101120000C4010F01EFB0094BAF8040010F4804F3D
:101130001CBF2046FEF741FB02F06BF930B10AF00C
:101140008AFC082818BF8AF8017001D18AF801804A
:1011500000986A4690F8203090F821C050300CFB7F
:1011600003F100EB41000021BCF1000F0DD930F874
:10117000025B02EB410603E09487001078870010C1
:10118000491CA6F8DE508C45F1D80021002B08D967
:1011900002EB410630F8025B491CA6F806518B426F
:1011A000F6D80021BCF1000F08D902EB410630F857
:1011B000025B491CA6F864508C45F6D80021002B30
:1011C00008D902EB410630F8025B491CA6F88C50A6
:1011D0008B42F6D830F8021BA2F8DA1030F8021B66
:1011E000A2F8DC1030F8021BA2F8D810002500216C
:1011F000BCF1000F0ED905EB450606EB051602EB18
:10120000860606EB410B30F8029B491CABF8529165
:101210006145F6D30021002B0ED905EB450606EB00
:10122000051602EB860606EB410B30F8029B491CC3
:10123000ABF882929942F6D36D1C042DD7D3614648
:101240001846FEF797FBDAF804003E4610F4004F0C
:1012500003D1694600F0ACFD0646ED98FCF79CF919
:10126000EE98FCF732FC94F8209094F82150002E70
:101270001CBFB9F1000F002D00F0DD809AF80400CA
:1012800010F0020F04D06A462946484600F032FCAE
:101290009AF8040010F0050F04D06A462946484623
:1012A000FEF747FF9AF80400D64610F0080F7DD0ED
:1012B000009A6846116921F4C0511161CDF860802F
:1012C000CDF85C809EF801B0BBF1000F1ED100216B
:1012D000002D1BD9DFF880C500EB4103DCF800C00E
:1012E000B3F93632BCF96AC09C450CDA4B0900EB05
:1012F000830301F01F0AD3F85CC007FA0AFA4CEA2C
:101300000A0CC3F85CC0491CA942E3D3C0F858805A
:10131000C0F85480BBF1000F21D10021B9F1000FBA
:1013200088BFDFF834B51AD9DBF800C000EB410301
:10133000B3F96633BCF96AC09C450DDA4FEA511C1B
:1013400000EB8C0301F01F0AD3F854C007FA0AFA25
:101350004CEA0A0CC3F854C0491C4945E4D3916BCC
:10136000C36D1943436DAB4019439163D16B036E59
:101370001943836DAB400B43D363416D202D39BFBF
:10138000C5F1200C21FA0CF1A5F1200C01FA0CF1A9
:101390001943D163416D002904BF816D002903D039
:1013A000116941F400611161C16D00E008E000299C
:1013B00004BF006E002803D0106940F48050106113
:1013C0009EF80400754610F0400F0FD16069401C74
:1013D00060612069002814BFE069A06900F1010084
:1013E00014BFE061A0616846FEF74BFAC4F80C80B8
:1013F000A36800222146A446B3F5056F88BF4FF4C9
:1014000005630020B0EB930F06D25CF82090401CDF
:101410004A44B0EB930FF8D35042C860287910F0DB
:10142000800F05D14FF47C304FF40562F2F78EFE49
:101430002046FEF72EF941208DF8B403C6B1207C7A
:101440008DF8B503607C8DF8B603A07C8DF8B703EA
:10145000E07C8DF8B80300230522EDA9072000F0F9
:1014600008FFFE48C0F808800DF56F7DBDE8F08FDD
:10147000FF208DF8B5038DF8B6038DF8B703E8E7C4
:101480002DE9F74F84B04FF0000AC2F820A00646BD
:10149000C2F81CA00598DFF8C083174654464FF0E9
:1014A0000109002821D907EB4400B0F964000028A5
:1014B000B8BF404200B2D8F80010B1F938108142EC
:1014C0000FDD610907EB810104F01F03CA6909FA06
:1014D00003F31A43CA6183B2E1B2FF220420FDF78D
:1014E00026FF0598641C8442DDD3002401281CBF1C
:1014F0000598451E46D007EB4403B3F96620B3F9BF
:101500006410501A48BF881A00B2D8F800C0BCF95D
:1015100030C0844533DAB7F9DA00B1EB000C48BFCC
:10152000A0EB010C0FFA8CFC111A48BF811A08B20B
:10153000844511DB600907EB800004F01F02C169DC
:1015400009FA02F21143C161B3F86430E1B2FF223B
:101550000420FDF7ECFE12E0601C410907EB81015D
:1015600000F01F0CCA6909FA0CFC42EA0C02CA61BD
:10157000C1B2B3F86630FF220420FDF7D8FE641C28
:10158000AC42B8D3D8F8000090F8361000297DD0CE
:1015900090F837003D68814288BF084600240599CD
:1015A000002984BF401C009070D94FF0010E0098B4
:1015B0004FF000090121CA46012852D9A648006807
:1015C0000390B0F93A3004FB066002900EFB06600F
:1015D000019004FB061005EB4000B0F950C0BCF1CF
:1015E000000FB4BFCCF100006046834239DB0EFB34
:1015F000061005EB4000B0F950000028B4BF42428D
:10160000024693422DDB029A521A05EB4202B2F9CE
:101610004E80B8F1000FB4BFC8F1000242469342B9
:101620001FDB019A521A05EB4202B2F94E20002A42
:10163000B4BFC2F1000B93469B4512DCA0EB0C0C2F
:101640000398B0F934006045B8BF09F10109A2EB75
:1016500008028242C8BF0AF1010A491C009881426F
:10166000B7D3BAEB090048BFA9EB0A007A49096869
:1016700091F83610884214DB600907EB800004F013
:101680001F030121C2699940114300E014E0C161C8
:1016900007EB4400E1B2B0F86430FF220420FDF70C
:1016A00046FE0598641C844206D2002C18BFA4F1A3
:1016B000010E7FF47CAF78E707B00120BDE8F08F22
:1016C0002DE9F74F064688B0002017681062D061F8
:1016D0009061506162480490002000900190029057
:1016E000824603900998154647F6FF7BA0F1010951
:1016F000A6F10108002871D90024002E69D94FEA0B
:10170000EA700AEBD06020F01F01AAEB0101012270
:1017100002FA01F1401105EB8000CDE906011C3011
:1017200005900AFB064007EB4000BAF1000FB0F944
:10173000500018BFCA450BD1002C18BF444507D133
:1017400045490968B1F99220B1F99010B2B911E098
:101750004149049B09689842B1F98A20B1F988107F
:10176000C4BF0294CDE903A05845BCBF8346CDE970
:10177000004AEBE7384A1268B2F98A2019B93649AB
:101780000968B1F98810904201DC88421EDA069996
:101790004FF0010CCA6907990A4305990A60E117DD
:1017A00004EBD1614A1105EB820303F1140221F02D
:1017B0001F015B69611A0CFA01F11943116083B2D0
:1017C000E2B20AF0FF010620FDF7B1FD641CB4424D
:1017D000A7D309980AF1010A82458DD31E4C2068CF
:1017E000B0F88E0000284DD00499A1EB0B01814286
:1017F00048DD03980399400905EB800001F01F03C1
:10180000C269012101FA03F31A43C2610198019AE6
:10181000400905EB800002F01F02C36901FA02F2E1
:101820001A43C2610298029A400905EB800002F057
:101830001F02436901FA02F21A4342610098009ABA
:10184000400905EB800002F01F02436991401943F3
:101850004161049883B205E09487001078870010F6
:101860000080FFFF0298C2B20398C1B20620FDF7C4
:101870005EFD00981FFA8BF3C2B20198C1B2062038
:10188000FDF755FDFE48006890F88C00002800F038
:101890002D814FF0000A002E7DD90998801E0090FE
:1018A00007EB4A000999B0F950000024012973D0D0
:1018B0004FEAEA710AEBD16121F01F02AAEB0202A2
:1018C000012303FA02F2491105EB8101CDE903126C
:1018D00014310291611C019101FB06A107EB41014A
:1018E000B1F950B0BBF1000FC8BF00285EDDBBEB03
:1018F000000148BFA0EB0B018345CCBF5A4602460E
:101900004FF44843594391FBF2F101F2FF114A0AA7
:10191000002C1CBF00998C420AD1BAF1000F18BFED
:10192000C24504D1D649096891F88D100CE014B174
:1019300000998C4204D1D249096891F8991003E0CA
:10194000CF49096891F88C1019B9CD49096891F807
:101950008C108A422ADDE11704EBD1614A1105EBB4
:10196000820221F01F0102F11C03A4EB010CD269D9
:10197000012101FA0CF111431960039983B2062089
:101980004A6904990A4302990A600AF0FF02E1B227
:10199000FDF7CDFC01E012E00CE001981FFA8BF39B
:1019A000C1B20AF0FF020620FDF7C1FC641C5846D4
:1019B0004C458FD30AF1010AB245FFF471AF099883
:1019C0004FF0000A002884BFB01E00907DD90AFBAA
:1019D00006F007EB40000024B0F95000012E7FD044
:1019E0004FEAEA710AEBD16121F01F02AAEB020271
:1019F000012303FA02F2491105EB8101CDE902123C
:101A00001C3101910AFB064107EB4101B1F952B0CB
:101A1000BBF1000FC8BF00285EDDBBEB000148BF73
:101A2000A0EB0B018345CCBF5A4602464FF4484316
:101A3000594391FBF2F101F2FF114A0ABAF1000F8A
:101A400018BFCA4509D1002C1CBF00998C4205D192
:101A50008B49096891F88D100CE014B100998C4203
:101A600004D18749096891F8981003E0844909680E
:101A700091F88C1019B98249096891F88C108A4242
:101A80002ADD02994FF0010CCA6903990A430199B2
:101A90000A60E11704EBD1614A1105EB820303F1FF
:101AA000140221F01F015B69611A0CFA01F119435C
:101AB000116083B2E2B20AF0FF010620FDF737FCA5
:101AC000601C1FFA8BF3C2B201E00FE008E00AF0DD
:101AD000FF010620FDF72BFC641C5846444591D3BA
:101AE00009980AF1010A8245FFF471AF0BB0012099
:101AF000BDE8F08F2DE9F04FD2F80090804689B014
:101B0000D9F81000164620F00F00C9F8100047F66B
:101B1000FF7003906FEA000002904FF0FF00049006
:101B200005904FF000001061F060B0605FEA010ABC
:101B300009F1500B0546706067D005FB08F04FF0C7
:101B4000000E3BF91010CDE9005E0A460120174651
:101B50007346B8F1010F19D905FB080C3BF91C407D
:101B60008C42C4BF21468646BC42BCBF274601907A
:101B7000B4EB020C48BFA2EB040C0FFA8CF29A42B1
:101B8000C8BF13462246401C4045E5D30298814217
:101B900002DDCDE9045E02910398874203DA0198E1
:101BA000039707950690C81B48BF781A02B23448BD
:101BB0000068B0F91CC0944503DBB0F91E008342F5
:101BC00020DDEA1705EBD262531106EB830C22F0FD
:101BD0001F020CF10C03AA1A0120DCF80CC0904083
:101BE0004CEA000018608BB20EF0FF02E9B205204B
:101BF000FDF79DFB0198BBB2C2B20098C1B20520AF
:101C0000FDF795FB6D1C554597D30025B8F1000FE6
